:020000040000FA
:040000006FD00400B9
:101000006F00907E00000000000000009020002093
:10101000AA220020A9BDF9F56C23002000000000E1
:10102000000000006C230020902000200000000041
:101030000000000090200020000000009020002010
:101040000000000090200020902000209020002030
:101050009020002090200020582F00209424002071
:101060000000000090200020902000201E2400207E
:1010700090200020D22300209020002090200020EB
:101080009020002090200020902000209020002020
:101090009020002001A04111B7170040985F3AC688
:1010A000945F3247E39CE6FE3245410182800111A4
:1010B00013078008F337078093F787083EC20100C3
:1010C0000100B7170040930570052380B70413068D
:1010D00080FA2380C7040100010083C6B70493F699
:1010E000F60DA385D704238007049246F3A6068055
:1010F0000100010093760502D5CEF336078093F602
:10110000860836C4010001002380B7042380C70489
:1011100001000100B70614007D89558D88C70100C4
:1011200001000100010023800704A246F3A6068007
:101130000100010073370780137787083AC6010062
:1011400001002380B7042380C704010001000100CF
:1011500001003727004093061005A303D7802380A2
:101160000704B247F3A70780010001009307800836
:10117000F3B7078093F787083ECE01000100B71749
:101180000040130770052380E704130780FA2380CB
:10119000E7040100010003C7B70413670708A3852C
:1011A000E70423800704F247F3A70780010001004A
:1011B0000561828093760504BDC6F336078093F6F9
:1011C000860836C8010001002380B7042380C704C5
:1011D00001000100B7061400938606047D89558D31
:1011E00088C7010001000100010023800704C246F6
:1011F000F3A6068001000100733707801377870884
:101200003ACA010001002380B7042380C70401000B
:1012100001003727004093062005A303D7802380D1
:101220000704D24781B773370780137787083ACC12
:10123000010001002380B7042380C70401000100DE
:1012400098471367070C98C723800704E24719BF24
:101250000111814601468145114506CE97000000E7
:10126000E780605893078008F3B7078093F78708F3
:101270003EC601000100B717004013077005238028
:10128000E704130780FA2380E7040100010003C785
:101290006704136717002383E70423800704B2471A
:1012A000F3A7078001000100F2400561828041112F
:1012B000814601468145114597000000E780A05214
:1012C00013078008F337078093F787083EC40100AF
:1012D0000100B7170040130670052380C70493066A
:1012E00080FA2380D70401000100FD552396B70240
:1012F00023800704A245F3A5058001000100733790
:101300000780137787083AC6010001002380C704CD
:101310002380D7040100010003C767041367170087
:101320002383E70423800704B247F3A70780010063
:10133000010001A0BD473305F50201007D1575FDD3
:101340008280411122C426C206C6AA8401446317C2
:101350009400B24022449244410182800504130566
:10136000803E420497000000E78000FD4180C5B741
:101370009305000273A04580824573901534924016
:101380002242B2424243D2436244F2440255925551
:101390002256B2564257D2576258F25806499649D9
:1013A000264AB64A464BD64B664CF64C065D965DD1
:1013B000265EB65E465FD65F09617300203041113C
:1013C000B7170040985F3AC6945F3247E39CE6FE49
:1013D000324541018280B71700401307000323887C
:1013E000E702854717170000232EF74673002030C9
:1013F000411122C42D6426C24AC006C637190040D6
:101400001304A4AAB704002023208900977000E0E9
:10141000E780E0A99C408297977000E0E78020A9D0
:10142000E5B737370040834747009146BD8B639E41
:10143000D702B73600401306F00F973500009385AA
:10144000E5219737000083D7673103C7A6001377DC
:10145000F70F1DE3B7E70400BC4F09468945171590
:1014600000000345A5F7829731A099466394D70001
:10147000834757007300203003C786001377F70FA8
:10148000E365F6FC13851700AE97173800002317A5
:10149000A82C2380E70075B7B787004003C7670013
:1014A000098B6309071003C77700930600031377BE
:1014B0000703630DD708173800000348787B1736F9
:1014C00000001306E6770547B30606012380E60011
:1014D00083C577001737000013078778429793F585
:1014E000F50F2300B70003C58700973500009385EB
:1014F0002576C2951375F50F2380A50003470700D5
:1015000089451377F703630CB70C63E7E50A6306B5
:10151000071A8545630CB7129737000083C75775C4
:101520003307F600034707001377F70F19CB85073A
:1015300093F7F70F3D476363F71A17370000A309C6
:10154000F772B787004009472383E700B787004059
:1015500083C77700E207E18763DE0704973700005F
:1015600083C71771173700001307876D3E978546AD
:101570002300D700173700001307876E3E979306A6
:1015800000032300D700173700001307676C3E974E
:10159000A14685072300D70093F7F70F3D47636403
:1015A000F71417370000A305F76CB7870040094709
:1015B0002383E70073002030930610026300D70EE8
:1015C000930620026305D70693060002E316D7F4BC
:1015D00003C727021377C70F13672700D5A803C7D0
:1015E00067001377070465CB03C7A702173800000D
:1015F00013088846173500001305C53D1347070833
:101600002385E70203C7A7021377370F1367870005
:101610002385E702814713070004B305F5008C41D9
:10162000B306F80091078CC2E399E7FEF5B503C74E
:10163000A702134707042385E70203C7A70213770E
:10164000C70F136727002385E702F9B503C76700B3
:101650001377070449C303C767021738000013084C
:101660006833173500001305A52A1347070823839D
:10167000E70203C767021377370F136787002383D7
:10168000E702814713070004B305F5008C41B30658
:10169000F80091078CC2E399E7FEBDBD03C767025E
:1016A000134707042383E70203C767021377C70FB3
:1016B000136727002383E70285B503C76700137705
:1016C000070411CB03C727021377370F136787006F
:1016D0002381E70291B5238006003DBD97370000C6
:1016E000A3880758B9BD97370000A383075875BD75
:1016F0002303048015472303E48001002302A48010
:10170000828083076480E3CE07FE23030480828007
:1017100083076480E3CE07FE03454480828083070D
:101720006480E3CE07FE2302A4808280411126C498
:101730004AC24EC006C61377F50BAD47AA892E895B
:101740009544630CF700194597000000E78080FA84
:1017500097000000E78020FB8D444E859700000035
:10176000E78040F9FD59FD1463983401B240A2446A
:101770001249824941018280135509011375F50F01
:1017800097000000E780E0F92209F1BF011126CCA3
:1017900006CEB704080097000000E780C0F61545A4
:1017A00097000000E78000F597000000E78080F6D2
:1017B00097000000E78000F62AC697000000E78047
:1017C00080F432459377150089EB13651500137586
:1017D000F50FF240E24405618280FD14E9F0014515
:1017E000CDBF397126DC4ADA4ED852D656D45AD2F9
:1017F0005ED006DE62CE66CCB7E700E07D5783AAF6
:10180000070022C603AA470023A0E71823A2E7186F
:10181000B7170040130770052380E704130780FA09
:101820002380E70483C74704930B75FFB684E20760
:1018300093FBFB0F8546AA892E8B32893724004003
:10184000E187015763FA76016308D50089461307DB
:1018500000026313D5000157D98F93F7F70FB71C18
:1018600000402382FC0411472303E4801305F00F9A
:1018700097000000E78000E8094C97000000E7802F
:1018800080E863657C15B7050700DA9537870700A0
:10189000795563FEE504B3879500636AF704370B57
:1018A0000800A94733EB65016395F90881E8814495
:1018B00097000000E78020E5268515A8DA85094510
:1018C00097000000E780C0E605090345F9FFFD1415
:1018D000050B97000000E780C0E481C49377FB0FFD
:1018E000E5F797000000E780A0EA69F17D55B7179A
:1018F0000040130770052380E704130780FA238054
:10190000E70403C74704418B2382E704F250B7E79B
:1019100000E023A0571123A24711E2543244525948
:10192000C259325AA25A125B825B724CE24C21615C
:101930008280A547639BF90685691309F00FB306FA
:101940009900B3742B01B6941349F9FFB37499004D
:10195000856B33796901416B9387F9FFB3F72701F1
:1019600099E363FC340193D94900C147E3E637FFAB
:101970003DBF0569C1697D19D9B71305800D63881D
:101980006901130500026384790113051008CA85F3
:1019900097000000E780C0D997000000E78040DF93
:1019A00031D54E99B38434416DBFDA852D4597000A
:1019B0000000E780E0D7CA94E30B99EE0509970091
:1019C0000000E78020D5A30FA9FEFDB79387F9FF9C
:1019D00093F7F70F636DFC0C83C71C0413073008E3
:1019E0006315F706370708006361EB06B3079B0032
:1019F000B706100063FBD704334BEB0089476399AC
:101A0000F9068980D549E38404EADA850945970017
:101A10000000E780E0D111090327C9FF9147232087
:101A2000E48003076480E34E07FE23033481FD173F
:101A3000EDFBFD14110B81C49377FB0FE9FF9700B9
:101A40000000E780E0D461F155B5B717004003C747
:101A50005704B70708001377070219E3B787070091
:101A60007955E376FBE833079B00E3F9E7F841B5E6
:101A70008547E380F9F0DA852D4597000000E7807F
:101A800020CB9389F4FFE38404E297000000E78011
:101A900060C893F7390091EB83260480032709007F
:101AA00093074900E396E6E03E89CE84D9BFB54767
:101AB0006399F9001305900B97000000E78080C33D
:101AC000FDB3B1471305B00AE388F9FE9947639760
:101AD000F904B7050800B365BB002D459700000069
:101AE000E78000C581448D4BA14997000000E78045
:101AF00060C263967401832704802320F900850463
:101B0000E39534FF8327048013172B0163550700E7
:101B10002312F90069BB2322F90051BB9D47639F43
:101B2000F90281451305B00497000000E78040C02A
:101B3000BD442320090023220900FD59970000001D
:101B4000E78040BD93F77400CA9703C70700FD14F0
:101B5000398D2380A700E39334FF91BBA14763979E
:101B6000F90697000000E780A0C28144630D0B00D6
:101B70008D479304C0036308FB00930400056304CE
:101B80008B01930440041375C507E30295D21945F0
:101B900097000000E78000B697000000E780A0B63D
:101BA000054597000000E780E0B426859700000017
:101BB000E78020B7094597000000E78080B69700CE
:101BC0000000E780E0BCE31405CE0DB39147639FAE
:101BD000F9001305600697000000E780A0B19700A8
:101BE0000000E78040B213059009F9B5E38109CC04
:101BF000F1547DB9BD6601471736000013068633E0
:101C0000938606A685458347060093F7F70F91C391
:101C100082800507E3F9E6FE97370000238CB73092
:101C2000DDB77D166206618693178601E18763D46E
:101C3000070001458280931726003307F500AE9711
:101C400018439C4363E7E7007D16E37FF7FC7D556F
:101C5000828005458280FD15E205E18513978501A7
:101C6000618793F7F50F63480700FD15139725006B
:101C70002A97584365D713851700620561858280CE
:101C80003308B5021C4283A80600B335B502C297DB
:101C900033B50701AE98469585486367B5006394F0
:101CA000A50063E3070181480C43C6950CC388C2B5
:101CB0001CC2828081471397870161876343B70005
:101CC0008280139727002A97232007008507E5B70E
:101CD0008147014793968701E18663C5B6001335B6
:101CE0001700828093962700AA9694428507558F05
:101CF000D5B793D755408A07AA979C430545331516
:101D0000B5007D8D828017F3FFDFE702833D2A84D3
:101D100097000000E78060F405C5931725003E9406
:101D20000327C4FF814711EB7D1516053E9542053B
:101D3000418517F3FFDF6700033D05838507E5B79E
:101D40000145C5BF81471397870161876343C7007A
:101D5000828013972700B386E50094422A9785076F
:101D600014C3D5B77D1662066186014793178601B5
:101D7000E18763D50700133517008280931726008B
:101D8000B306F500AE9794429C437D16B58F5D8FE8
:101D9000F1BF8A05AA9501476363B500828083A6D7
:101DA000C5FFF11593D71600D98F9CC11397F60183
:101DB000E5B72A830148014701456343D700828084
:101DC000B387050183A80700B30706019C43C697A4
:101DD000AA976384F80033B517010507B308030118
:101DE000620723A0F80061871108C1BF2A83014759
:101DF0008147014563C3D70082803388E50083288B
:101E00000800330EE600032E0E003388A840330886
:101E1000C8416384080133B508018507B308E300AE
:101E2000E20723A00801E1871107E9B717F3FFDFF5
:101E3000E702232B0111B286B2842E86AA850A8579
:101E400097000000E780C0FA2A84A6850A859700DB
:101E50000000E78020E833348000060413351500C5
:101E6000018D056117F3FFDF6700E32917F3FFDF3B
:101E7000E702A3244111AA89AE8A328BB68402C23A
:101E800002C402C60144131C8401135C8C416349E3
:101E90009C02939B1400FD1B0549138CF4FFF15C1D
:101EA00033048901620461846340740792478E049D
:101EB000CE9423AEF4FE410117F3FFDF67006323E6
:101EC00013192400B30B2B01014A93172A00D6974C
:101ED00083A50B0088437800340050009700000071
:101EE000E78040DA050A93178A01E187F11BE35E78
:101EF000FCFC92474E9905042320F900A2473EC2FC
:101F0000B24702C63EC441B7131A8901135A8A4127
:101F1000131D240093178A01E18763CF970092472E
:101F20000A044E941CC0A24705091379F90F3EC25A
:101F3000B24702C63EC4ADB7B3079A0313152A00D1
:101F400056950841780034005000050AEA97DA9760
:101F50008C4397000000E780E0D26DBF197106C284
:101F600012C416C61AC81ECA22CC26CE2AD02ED219
:101F700032D436D63AD83EDA42DC46DECAC0CEC2C9
:101F8000D2C4D6C6DAC8DECAE2CCE6CEEAD0EED2F9
:101F9000F2D4F6D6FAD8FEDA971500009385058CB0
:101FA0008841E700050092402242B2424243D243B8
:101FB0006244F244025592552256B2564257D257C5
:101FC0006258F25806499649264AB64A464BD64BBD
:101FD000664CF64C065D965D265EB65E465FD65F45
:101FE0000961730020300000972100209381810156
:101FF000175100201301018117F5FFFF1305C500DC
:102000009705002093850500171600201306C6FDCE
:1020100063FAC5008322050023A055001105910530
:10202000E3EAC5FE170502001305856D971500202C
:102030009385C5FB171600201306C66563FAC50015
:102040008322050023A0550011059105E3EAC5FE92
:1020500017150020130505649745002093858539E1
:102060006377B500232005001105E36DB5FEFD4241
:10207000739002BC8D4273904280B722000093821D
:10208000828873900230970200209382A2F793E235
:1020900032007390523097520000938262D1739055
:1020A00012346FB0F47573002030397101436EC67D
:1020B00019A0397141536AC866CA62CC5ECE19A0B4
:1020C000397101535AD056D252D44ED64AD826DA54
:1020D00022DC06DE33016140828241114AC026C201
:1020E00022C406C68282B24D4101024D924C224C5E
:1020F000B24B4101024B924A224AB2494101024984
:1021000092442244B240410182803D432A87637356
:10211000C3029377F700BDEFADE5937606FF3D8AE6
:10212000BA960CC34CC30CC74CC74107E36BD7FE30
:1021300011E28280B306C3408A0697020000969699
:102140006780A6002307B700A306B7002306B700E1
:10215000A305B7002305B700A304B7002304B70005
:10216000A303B7002303B700A302B7002302B700FD
:10217000A301B7002301B700A300B7002300B700F5
:10218000828093F5F50F93968500D58D9396050182
:10219000D58D61B7939627009702000096968682A8
:1021A000E78086FA9680C1171D8F3E96E374C3F8C8
:1021B000A5B73367B500FD530D8B79E7B7877F7FF0
:1021C0009387F7F710419441B372F6003363F6003A
:1021D000BE92B3E262006397720C6318D606504158
:1021E000D441B372F6003363F600BE92B3E26200EC
:1021F0006398720A631BD60410459445B372F600C7
:102200003363F600BE92B3E262006391720A631E0A
:10221000D6025045D445B372F6003363F600BE9241
:10222000B3E26200639A72086311D60210499449BE
:10223000B372F6003363F600BE92B3E262006393BA
:1022400072085105D105E30FD6F6131706019397CF
:102250000601631CF7001357060193D706013305E7
:10226000F7409375F50F91E982804183C18333056F
:10227000F7409375F50F91E182801377F70F93F78D
:10228000F70F3305F74082800346050083C605003B
:10229000050585056313D60065FA3305D6408280AF
:1022A00011059105E312D6FE014582802105A105A5
:1022B000E31CD6FC014582803105B105E316D6FC4E
:1022C000014582804105C105E310D6FC01458280AD
:1022D000B717004003C777051377E70FA38BE70411
:1022E000130700F8A38DE7043D47238CE704130789
:1022F0005003A38CE70403C7A7051377D70F238DDB
:10230000E7048280B717004003C7E7020D89411137
:102310001377C70F498F93068008F3B6068093F6AC
:10232000860836C601000100930670052380D70495
:10233000930680FA2380D704010001002387E70277
:1023400023800704B247F3A7078001000100410181
:10235000828041112A83014E930E407E130F001993
:10236000930F400663E56E129308001913034006AD
:10237000B3781503854E0D4FA14F337365020D8958
:102380001335150063EFBE121308F6FF79467298F5
:102390004208135808013307C70213D61700BE07B7
:1023A00032976146B3F6C60213068070B386C60242
:1023B0003697A166F58F42075D8FB716004083C739
:1023C000F60293F70708A303F1000346710083C7E1
:1023D000F60293F70708E394C7FE83477100B71628
:1023E000004093F7F70F6388071293078008F3B74D
:1023F000078093F787083EC401000100B71700402B
:10240000930670052380D704930680FA2380D704AF
:102410000100010023AA070383C6170393E60608F9
:10242000A388D70223800704A247F3A707800100EF
:1024300001001166B71700407D16D45BC85F938515
:102440004703A98EF18EF5FA93068008F3B606804D
:1024500093F6860836C601000100930670052380B6
:10246000D704930680FA2380D7040100010098C1A5
:1024700003C7170313670704A388E7022380070431
:10248000B247F3A7078001000100410182807D135C
:102490003368E3039308E016630E08003368F30320
:1024A0009308D016630808009378330093B8180097
:1024B0009388D81633081E01131E0801135E0E01FF
:1024C00055B56393E5030548638608000148630337
:1024D00003002A8871087298FD15131E0801C205B1
:1024E000135E0E01C18179BD13F8150063F4BF00BE
:1024F0007908D5B713381800E5BF83C7F60293F7FC
:102500000708A303F1000346710083C7F60293F79F
:102510000708E394C7FE8347710093F7F70FF1DFD5
:10252000E9B531714AD966CB06DF22DD26DB4ED70D
:1025300052D556D35AD15ECF62CD6AC96EC7AA8C26
:1025400002D897100000E78020B12A8993078008FD
:10255000F3B7078093F787083EDA01000100B71749
:102560000040130770052380E704130780FA2380D7
:10257000E7040100010003C7F7021377770FA38771
:10258000E70203C7F70213678700A387E7022380E8
:102590000704D257F3A70780010001000545970003
:1025A0000000E78060D6130780C13347E902116A53
:1025B00093070AE893065002BD69930BA004814A71
:1025C000014B13048008930470057D1AB347F90288
:1025D0003307D7023EC0FD873ECC938709A69309F7
:1025E000803E3347F7023AC27D873AC43347390306
:1025F0008549B399990193D93940B306D702B30BF2
:102600007703B3C6F602B3CBFB0236C6FD8636C8E7
:1026100093D6FB4136CEB7460F0093860624334946
:10262000D9028566938606FAB3969601B389E902C4
:10263000130760553309D90293060010B389E902E4
:102640003349D902B3C9F9029316390036CA37198A
:102650000040FD8636D0930D090493D7F9413ED250
:10266000F336048093F6860836DC010001009307F8
:1026700070052380FD00930680FA2380DD000100B1
:1026800001008346390593F6860FA309D9048346D2
:10269000390593E61600A309D90423800D00E256FC
:1026A000F3A6068001000100130C80FA116DF336C9
:1026B000048093F6860836DE01000100930770055A
:1026C0002380FD0023808D01010001008346390530
:1026D000216693E60602A309D90483560905B3E6E9
:1026E000A6012318D90483560905D18E2318D904CD
:1026F00023800D00F256F3A60680010001008346F8
:10270000390593F606026381061A03463905218AC4
:102710006DDE081897100000E7800098733604807B
:1027200013768608B2C20100010023809D00238039
:102730008D0101000100B717004003C6370513766D
:10274000F60DA389C70403C6370513660602A389DD
:10275000C704835609052166B3E6A6012318D904E8
:1027600083560905D18E2318D90423800D0096467F
:10277000F3A60680010001008346390593F60602A0
:10278000638B061483463905A18AEDFE970000206D
:10279000E7806090AA8636D497000020E780A08F5B
:1027A000A256E30AD5FE835609054255B3E6A601B3
:1027B0002318D90497100000E780C08F834639059D
:1027C000A18AEDDE03560905834629058247337643
:1027D000CA00B306DA0293D5F641B296B388F64042
:1027E000E24733B8C6002E983308F840A247B3B684
:1027F00016013308D84063C70701631DF8009247EC
:1028000063FA1701C247634FF80E63950701B24799
:1028100063EAF80E894663E9660FF24693151800DD
:1028200013D3F8015E8613951800B365B30042D642
:1028300046D497C00100E78040493258050B137B0E
:10284000FB0F63470001631A0838A25863870838F2
:1028500013081500B336A800B69513D6F5013298C3
:10286000B336C800AE9613581800FE06B3E606014C
:102870007336048013768608B2C6010001002380F7
:102880009D0023808D01010001000356C902B2960C
:10289000C206C1822316D90223800D00B646F3A6D4
:1028A00006800100010021B5F336048093F6860806
:1028B000B6C00100010023809D0023808D0101002E
:1028C00001008346390593E60602A309D904238053
:1028D0000D0086460DB5F336048093F68608B6C41F
:1028E0000100010023809D0023808D010100010073
:1028F0008346390593E60602A309D90423800D0017
:10290000A646BDB5E30B0BF0F336048093F68608BC
:10291000B6C801000100930680FA23809D00238041
:10292000DD00010001008346390593F5FC0F93F6A5
:10293000860FA309D90483463905CD8EA309D9048E
:1029400023800D00C646F3A6068001000100130592
:1029500080FA03463905930639051D8A631C9629BA
:102960007336048013768608B2CC0100010013068A
:1029700080FA23809D002380CD000100010003C662
:1029800006001376F60D2380C60003C60600136604
:1029900006022380C600835609051166D18E2318CE
:1029A000D904835609052166D18E2318D9042380C2
:1029B0000D00E646F3A6068001000100130680FA2A
:1029C0008346390593F60602638006268346390559
:1029D000130C3905A18AFDDA081897000000E7807A
:1029E000A06BF336048093F68608B6D00100010090
:1029F000930680FA23809D002380DD000100010002
:102A000083460C00116693F6F60D2300DC00834626
:102A10000C0093E606022300DC0083560905D18EE4
:102A20002318D904835609052166D18E2318D904A9
:102A300023800D008656F3A60680010001001306D0
:102A400080FA8346390593F60602638A0620834698
:102A50003905A18AEDFE97F0FF1FE780C0632A8C3D
:102A600097F0FF1FE7802063E30C85FF835609057D
:102A700011664255D18E2318D90497000000E780D3
:102A800060638346390513063905A18AFDDAF336FA
:102A9000048093F68608B6D401000100930680FAFC
:102AA00023809D002380DD00010001008346060095
:102AB00093F6F60D2300D60023800D00A656F3A64C
:102AC0000680010001008356090503462905D24707
:102AD000B376DA003306CA021305800C9355F6412B
:102AE0003696330DF6408257333CD6002E9C333653
:102AF000A601330CFC40330CCC40330885039256BE
:102B00004E86B335A5033305A503C29597C00100D2
:102B1000E780A01B63468001631E0C16630C0D1634
:102B2000130615003335A6002E959356F5013696FB
:102B3000B335D600AA959396F50105828585D18E89
:102B40006346B000639D051A638B061A0356C902DB
:102B500015823305D6003336C500B2956348B00000
:102B6000639105241306F00F637DA622894663F363
:102B7000561593078008F3B7078093F78708BED6EA
:102B80000100010037170040930770052300F70488
:102B9000930780FA2300F704010001008356C7025F
:102BA00089678117D58FC207C1832316F7022300D7
:102BB0000704B657F3A7078001000100FA506A54D2
:102BC000DA544A59BA592A5A9A5A0A5BFA4B6A4C49
:102BD000DA4C4A4DBA4D296182801308F5FF33352E
:102BE000A800FD152E951356F5013298B336C8008E
:102BF000AA9695B9F336048093F68608B6CA010002
:102C0000010023809D002380AD0001000100834668
:102C10003905CD8EA309D90423800D00D646F3A62D
:102C200006800100010035B3F336048093F6860870
:102C3000B6CE0100010023809D002380CD0001005D
:102C400001008346390593E60602A309D9042380CF
:102C50000D00F646F3A606800100010095B3F33699
:102C6000048093F68608B6D20100010023809D00FF
:102C70002380CD00010001008346390593E606025A
:102C8000A309D90423800D009656F3A606800100FF
:102C9000010045BB9306F5FF33B5A600FD152E9543
:102CA0009355F501AE96B3B5B600AA951396F50106
:102CB000858269B5F336048093F68608B6D801009C
:102CC0000100930680FA23809D002380DD0001002F
:102CD00001008356C9020566011693F6F60FD18EE0
:102CE000C206C1822316D90223800D00C656F3A660
:102CF000068001000100850A93FAFA0F95B233E6C7
:102D0000B60045C20356C9023305D0403338A0008F
:102D1000B305B040B385054115826345B000D1E1EC
:102D20006371A608894663F0560593078008F3B7D8
:102D3000078093F78708BEDA01000100B71700404B
:102D4000130770052380E704130780FA2380E70444
:102D50000100010003D7C7027D8B2396E702238081
:102D60000704D65781BDF336048093F68608B6DC97
:102D700001000100930680FA23809D002380DD007E
:102D8000010001008356C9020566011693F6F60F8D
:102D9000D18EC206C1822316D90223800D00E656C9
:102DA000B9B793078008F3B7078093F78708BEDEAB
:102DB0000100010037170040930770052300F70456
:102DC000930780FA2300F704010001000356C702AD
:102DD00093975600B297C207C1832316F7022300C8
:102DE0000704F657C1BB914763EEB70217E701002E
:102DF0001307C78B8A05BA959C41BA978287B71784
:102E0000004003A7470B1345F5FF698F23AAE70A84
:102E100003A7070B698F23A8E70A03A7070A798D81
:102E200023A0A70A8280B717004083A6470B134749
:102E3000F5FFF98E23AAD70A83A6070B558D23A881
:102E4000A70A83A6070A758F23A0E70A8280B7170F
:102E5000004003A7470B498F23AAE70A03A7070BE4
:102E60001345F5FF45BFB717004083A6470B13472F
:102E7000F5FF758F23AAE70A03A7070A598D4DB7F7
:102E8000B717004003A7470B498FEDB7914763EE93
:102E9000B70217E701001307A7828A05BA959C417C
:102EA000BA978287B717004003A7470D1345F5FF70
:102EB000698F23AAE70C03A7070D698F23A8E70CE6
:102EC00003A7070C798D23A0A70C8280B7170040B9
:102ED00083A6470D1347F5FFF98E23AAD70C83A6C7
:102EE000070D558D23A8A70C83A6070C758F23A06B
:102EF000E70C8280B717004003A7470D498F23AA2C
:102F0000E70C03A7070D1345F5FF45BFB7170040B2
:102F100083A6470D1347F5FF758F23AAE70C03A778
:102F2000070C598D4DB7B717004003A7470D498FC0
:102F3000EDB7797122D43714004026D24AD0035914
:102F400024028354040206D64209C2044ECE52CC57
:102F500056CA13590901C1802DE11379F9F793F489
:102F6000F49F4209C20413590901C18093078008E4
:102F7000F3B7078093F787083EC401000100930769
:102F800070052300F404930780FA2300F404010081
:102F90000100231124032310940223000404A247F8
:102FA000F3A7078001000100B25022549254025945
:102FB000F249624AD24A45618280B7F507008146EC
:102FC0003000B105194597000020E7808081A247B5
:102FD00013972701E34A07FC1369090893E40440A7
:102FE00093098008F3B7098093F787083EC0010072
:102FF0000100930A700523005405130A80FA230088
:10300000440501000100231124032310940223002E
:1030100004048247F3A7078001000100294597F0C7
:10302000FF1FE7802031F3B9098093F989084EC268
:1030300001000100230054052300440501000100A4
:103040008357040293E707202310F40223000404AB
:103050009247B9B7B7170040884742054181937737
:10306000050491EB9377F5013755E80113050580C9
:103070003345F50282809377050C130700046397AC
:10308000E7009377F50137459C1CCDB72165130503
:1030900005D0828037E700E01C435443A183E20659
:1030A000D58F1CC1FD572320F7182322F7188280E3
:1030B00013178500B7E700E023A0E710618123A282
:1030C000A7108280B7F700E08847CC47828081470D
:1030D00037370040A14663C4C7003285828003456C
:1030E000B740E38EA6FE3385F5000345050085074E
:1030F0002304A740CDB797070020938727EF9C4371
:10310000173700201307072F3E95636EE50017372A
:1031100000201307273F6368A70017070020232715
:10312000A7EC3E858280FD57EDBF8280411122C40D
:1031300006C62A8497000000E78000F22947B307FB
:10314000E502B2408D83B3D7870222449507B3D7F7
:10315000E70237370040C207C1832316F700410159
:103160008280411137150E0006C697000000E780E7
:1031700020FCB7370040130770F82381E7000D47A4
:10318000A381E70013070004A380E7000547238716
:10319000E700B24041018280373700408347270073
:1031A0001A0593F7F703C98F93F7F70F2301F70079
:1031B0008280B737004003C7170019C9D98DA38093
:1031C000B70003C70700136787002380E7008280EA
:1031D00093C5F5FFF98DA380B7008280AE872A875B
:1031E000B736004021463738004089E71703000012
:1031F0006700E3F383C8B600E30916FF05078348B9
:10320000F7FFFD17C20723041801C183F9BF41115D
:1032100022C406C62A8497000000E780E0E329471D
:10322000B307E502B2408D83B3D7870222449507E6
:10323000B3D7E70237370040C207C1832316F740F0
:1032400041018280716541111305052006C6970072
:103250000000E78000FCB7370040130770F82381B7
:10326000E7400D47A381E74013070004A380E74030
:1032700005472387E740B24041018280CC4141119C
:1032800006C6328503C6150083C5050022064D8E8D
:1032900042068D654186138875A2630C0611634B47
:1032A000C804138845A26300060D634AC8009385CD
:1032B00035A26301B6082390060029464DA0138865
:1032C00055A26305060D938565A2E316B6FE8D45EE
:1032D0001D4663E6E5081146198E63F3C7003E8676
:1032E000B7E704002390C600FC4797D501009385FB
:1032F000653F9DA0138895A263030611634E060DDA
:103300001388A5A263000613938505A5E315B6FAF5
:1033100099451D4663E5E504198E63F3C7003E86B3
:10332000B7E704002390C600FC479705002093856B
:1033300025D61DA09D451D4663E3E5022146198E55
:1033400063F3C7003E86B7E70400FC472390C6003E
:103350009705002093858534BA9582970146B2403F
:10336000328541018280AD451D46E3EAE5FE3146E6
:10337000198E63F3C7003E86B7E704002390C600AA
:10338000FC4797D5010093856538F9B7B1451D46CF
:10339000E3E7E5FC3546198E63F3C7003E86B7E7E1
:1033A00004002390C600FC4797D50100938505379C
:1033B00065B78D451D46E3E4E5FA1146198E63F3C2
:1033C000C7003E86B7E704002390C600FC4797D5A8
:1033D00001009385E53149B78D451D46E3E1E5F8E8
:1033E0001146198E63F3C7003E86B7E704002390A9
:1033F000C600FC4797D5010093850534B1BFA545AC
:103400001D46E3EEE5F42946198E63F3C7003E86B8
:10341000B7E704002390C600FC4797D501009385C9
:10342000E52D1DBFB5451D46E3EBE5F23946198E86
:1034300063F3C7003E86B7E704002390C600FC474D
:1034400097D501009385052901BFB7E7040003A3C1
:103450000713970600209386A6C24146A545170587
:1034600000201305E5B802832D455DE703C505007F
:103470000947631FE50803A84500411106C6034735
:10348000180032850346080022074168518F9308CF
:1034900028FE6307170563E9E800051863030703BF
:1034A00023900600294591A8130648FE630AC70425
:1034B0001518E31707FF15463E87637BF60015478F
:1034C00001A8130600023E876374F600130700028A
:1034D000B7E704002390E600FC471316070111A884
:1034E0003E8691C30546B7E70400FC472390C6001B
:1034F0004206CC45418282970145B240410182801B
:10350000130600083E87E375F6FC13070008C9B7E9
:103510002390060005458280828041677917630405
:10352000E504411122C406C685472A84639FF5003D
:10353000B7E7040022852244B24003A3871397050E
:1035400000209385E52F4101028389476399F500A7
:10355000B7E7040083A7070B8545829771D9B2406E
:103560002244410182808280797126D252CCAE847D
:103570002A8A97D501009385251E17D501001305CA
:10358000252006D63AC622D44AD0368432894ECE79
:1035900097C00100E780A0BEA28517D501001305E2
:1035A000251F97C00100E78080BD294597C0010015
:1035B000E780C0C183C7840093F70702F9E383C99A
:1035C00004008947054532476396F908D44083C70C
:1035D000160083C60600A207D58FC166138616FEA5
:1035E000638CC7028D16638FD7068D6693862690EF
:1035F00029456391D706B7E70400A286225403A3A6
:103600004714B250F2494A86A6850259925452850F
:10361000624A8547456102832D450DEF93070002FD
:10362000354563E98702B7E70400FC47C844130641
:103630000002CA8582978149970700209387072156
:103640009C43014581CB9C4391C74E852286CA8508
:1036500082970145B250225492540259F249624A6B
:10366000456182802D457DF79307700F3545E3E373
:1036700087FEB7E70400FC47C8442286CA858297C4
:1036800065BF2145C1BF411122C437E4040083272F
:10369000841326C2AA84416506C697050020938537
:1036A000251A7D1582978327C40A17050000130584
:1036B00005E78588829795C0032304132244B2400E
:1036C000924497060020938626AE4146C5451705CD
:1036D00000201305659C41010283B24022449244BC
:1036E00001454101828019C59707002023A0A71634
:1036F00001458280454582801147636AA70A97D6B3
:103700000100938626040A0536951841411106C624
:103710003697AE87B2850287130700026145639D25
:10372000E700B7E70400FC47130600021705002076
:10373000130545F782970145B24041018280054754
:103740006145E39BE7FEB7E70400FC470546170524
:103750000020130525F7F9BF1307700F6145E39D9E
:10376000E7FCB7E70400FC471306700F17050020BD
:10377000130585F5C1B7130700086145E39EE7FA15
:10378000B7E70400FC4713060008170500201305DF
:1037900025034DB715476145E390E7FAB7E7040005
:1037A000FC471546170500201305C50961B70945F3
:1037B0008280411126C2B7E4040083A7C41322C447
:1037C0004AC006C62E8497050020938565072A897E
:1037D0008297058905C5970700209387E78B83D7D4
:1037E000A70BA28503A3440D2310F4002244B2408A
:1037F00092444A850249014641010283B240224473
:103800009244024949454101828097070020238163
:1038100007049707002023AF0702B717004003A74C
:10382000070CB706C0FFFD16758F23A0E70C03A792
:10383000070DB7064000558F23A8E70C03A7070C18
:103840003D9B23A0E70C03A7070D1367070123A8DF
:10385000E70C8280B717004003A5470C83A7470CED
:10386000598113451500C18B058999E3136525001E
:103870009707002083C7C7FD6380A7029707002032
:103880002388A7FC11C9970700209387A7FC03A3EF
:1038900007006303030002838280114517F3FFFFD3
:1038A000670063C8011122CC06CE3714004026CA37
:1038B0004AC84EC652C483447405034AB4058349BA
:1038C00084050349940597F0FFFFE780A0A0834794
:1038D000A40593F4F40F137AFA0F93E71700230D5E
:1038E000F40493F9F90F1379F90FB717004003C7E0
:1038F000A705058B6DFF03D5C705A38D4705238C51
:103900003705A38C2705A38B9704F2406244D24469
:103910004249B249224A05618280411193970501CB
:1039200022C406C626C2C1872E8463DC0700B7E422
:103930000400FC54829719C1BC5482972165218DE3
:1039400015A893F7150013C515008DE793F725000B
:103950009DC797000000E78020F0B7E70400BC4F48
:103960001306000A894517050020034525EF8297B5
:1039700013452400B240224492444101828093972F
:10398000250163D80702B7E4040083A7C41E829709
:1039900097000000E780A0F0BC4C375607001306E4
:1039A0000630896517050020034545EB82970965B8
:1039B00079B7939715010145E3DE07FA17D50100A2
:1039C000130505E597C00100E7804093B7E70400C1
:1039D000BC4F13060064916517050020034505E8F8
:1039E00082971165A9BF1D71A2CC37E404005C5C0D
:1039F000485886CE494697D501009385E5DC8297E5
:103A000011E917D50100130565DD97C00100E780B6
:103A1000E08E01A0B7F600E0795798CAFD57DCCADE
:103A20000567B7E700E023A0E7101306F00290C295
:103A300023A0E718010001003707002018471306EC
:103A4000000481459706002023A8E6E04157A38A99
:103A5000E7403C4408088297970700209387877FB8
:103A60003EC8856713870740938757D1231AE10023
:103A70002312F1021307B00F97F7FFFF9387C76474
:103A80002310E1023ED81547970700009387C7E14E
:103A9000B7F50700A30FE1003EDC054797070000DC
:103AA0009387E7DF81463000E10519452301E102F4
:103AB0003EDE97F0FF1FE780C0D218088147994685
:103AC00030003E960346060085070507A30BC70096
:103AD000E398D7FEC24791C70357410185676373D7
:103AE000F70001A0B7E7040083A7470A08088297F8
:103AF000AA8511C917D50100130585CF97B001001C
:103B0000E780E06701A0F6406644256182804111AC
:103B100026C2B7E4040083A7040806C622C417051A
:103B200000001305C5DF829717040020130404D397
:103B30002300A40097000000E780800297000000A7
:103B4000E780E0CC03450400224403A38405B2408F
:103B5000924413060032896541010283797106D6C9
:103B600022D413078008F337078093F787083EC2F3
:103B700001000100B7170040930570052380B704CA
:103B8000130680FA2380C7040100010083C6F702F0
:103B900093F6A60FA387D702238007049246F3A6C5
:103BA00006800100010073370780137787083AC445
:103BB000010001002380B7042380C7040100010035
:103BC00003C7F70213672700A387E70223800704D0
:103BD000A247F3A7078001000100054597E0FFFF1A
:103BE000E780807297000000E78060CB0147814644
:103BF0008147054685451305407E97E0FFFFE78036
:103C0000807537E404003C44680051468145829742
:103C1000B707C0A83EC8B787E803938707D03ECA56
:103C200097E7FF1F9387A7793EC67C586800829765
:103C3000B250225445618280411197D5010093858D
:103C4000A52217D501001305A5B306C697B001003C
:103C5000E780E05217D501001305C53897B0010081
:103C6000E780E051B2402945410117B301006700E8
:103C7000E355411197D501009385452017D50100E3
:103C8000130505B006C697B00100E780404F17D571
:103C900001001305E53397B00100E780404EB240C4
:103CA0002945410117B3010067004352411122C465
:103CB00006C6834705002A849DC797D501009385D2
:103CC000A52117D501001305A5AB97B00100E7802A
:103CD000004B4C4017D501001305454697B0010035
:103CE000E780E0493DA058410DEF97D5010093854D
:103CF000A51E17D501001305A5A897B00100E78000
:103D0000004817D501001305E54497B00100E7808E
:103D100000472244B2402945410117B30100670022
:103D2000E34AA1679386D7036313D70297D50100AF
:103D30009385851A17D50100130585A497B0010056
:103D4000E780E04317D501001305C5417DBFED07AE
:103D500097D501009385451817D50100130545A295
:103D6000631BF70097B00100E780604117D50100A1
:103D70001305854059BF97B00100E78040404C4093
:103D800017D501001305454191BF411197D5010099
:103D90009385051017D501001305859E06C697B0BB
:103DA0000100E780C03DB2402945410117B3010041
:103DB0006700C341797122D426D24AD02E842A8941
:103DC000B28481457146480006D697E0FFFFE78040
:103DD000003497F7FF1F9387275EDC4783D70700E0
:103DE000231421012313F10097500000E780405570
:103DF0008547A305F1009307401F2305A1003EC698
:103E00002686FD57A2854800230AF100975000003E
:103E1000E780E055B25022549254025945618280A5
:103E20004111814617F6FF1F1306465685451705B3
:103E300000200355252406C697D00000E780E0A5A2
:103E400015C997D501009385E50717D5010013051E
:103E5000259397B00100E780803217D50100130544
:103E6000E52997B00100E7808031294597B001002E
:103E7000E780C03597D501009385C50417D50100AB
:103E80001305059097B00100E780602F17D501005A
:103E90001305052897B00100E780602E294597B0EB
:103EA0000100E780A03297F7FF1F9387E750DC47B8
:103EB000054797D501009385E5002390E70017D5C6
:103EC00001001305E58B97B00100E780402B17D563
:103ED00001001305252597B00100E780402AB24074
:103EE0002945410117B301006700432E411122C447
:103EF00097D50100938585FF2A8417D50100130506
:103F0000258806C697B00100E78060274C4017D58A
:103F100001001305251C97B00100E78040262945C4
:103F200097B00100E780802A034704009307F00F51
:103F3000631FF70297D50100938545FB17D5010054
:103F40001305058497B00100E78060234C4017D526
:103F500001001305251997B00100E7804022224493
:103F6000B2402945410117B3010067002326B24042
:103F7000224441018280411122C426C22A84AE8497
:103F800017C501001305C57F97D501009385C5F1BD
:103F900006C697B00100E780801E17D50100130503
:103FA000652497B00100E780801D294597B0010086
:103FB000E780C02197D50100938505EF9707002082
:103FC000239A870A17C501001305857B05449707C7
:103FD0000020239F970897070020239C87089717A6
:103FE0000020239C977697B00100E7804019971531
:103FF000002083D5857617D501001305251F97B0BE
:104000000100E780C017294597B00100E780001C38
:10401000971700202380876497F7FF1F9387C7397E
:10402000DC47170500200345E58303D70700C16778
:10403000FD17631EF700B7E7040003A38705130607
:10404000000A85452244B240924441010283B7E709
:10405000040003A387051306001493050010DDB7C1
:10406000B1C1411122C417C50100130565712E8429
:1040700097D50100938585E206C697B00100E780D9
:104080000010A28517D501001305051597B0010092
:10409000E780E00E2244B2402945410117B30100F8
:1040A0006700C3128280011122CC26CA4AC836C6D4
:1040B00006CE2A84AE84328997000000E780C0CF04
:1040C000F157B246631EF50089CE97500000E78095
:1040D000203E4A86A685228597000000E780C0CD55
:1040E00005C59707002083D747FC850717070020E1
:1040F000231DF7FA97070020239AA7FAF24062449B
:10410000D2444249056182809707002083D727FA6D
:10411000850717070020231CF7F8CDB797F7FF1F77
:1041200083C7B77417F5FF1F034545743D8D2205FE
:1041300097F7FF1F83C797733D8D4605458111C5CE
:10414000D1476315F50055458280054582804111B0
:10415000971700202393076097170020238C074EA2
:1041600006C617070020034727FF9307F00A6315C9
:10417000F7029307F0F88945170500201305C5FDE0
:1041800017070020230AF7FC97070020A38607FCE7
:1041900097600000E78000DC97600000E780C008BF
:1041A00097600000E780000A814537050400970703
:1041B000002023A907F897070020238307F8970713
:1041C0000020239907EC97070020239707EA970719
:1041D0000020239C07F297070020239707F69730CB
:1041E0000000E780C06D014597600000E78080DF38
:1041F00097000000E780C0F2970700202391A7F402
:10420000B7E70400BC4F13060014894517F5FF1FDC
:1042100003454565829797D501009385E5C917C584
:1042200001001305E55597B00100E78040F59705BB
:10423000002083D5C5F017D50100130525FC97B0E4
:104240000100E780C0F3B2402945410117B30100E6
:104250006700C3F7011122CC37E404005C5C06CE92
:1042600026CA354697D50100938505D917E5010083
:104270001305C5AE829711E917C501001305055650
:1042800097B00100E780800701A097F7FF1F938791
:10429000275E3EC4B7F50700856793870780814690
:1042A00017F6FF1F1306465CE10519453EC697E069
:1042B000FF1FE78000537C44194697F5FF1F938545
:1042C000A55A17050020130525DD8297340017F63F
:1042D000FF1F1306665997D501009385E51D17D575
:1042E00001001305E51E97700000E780804CAA844A
:1042F00021C197D501009385A5C217C501001305FB
:10430000254897B00100E78080E7A68517D5010012
:10431000130585CF97B00100E78060E6294597B087
:104320000100E780A0EAF2406244D2440561828045
:1043300097F00000E780A0B117D501001305C5C3B1
:1043400097600000E780A04097600100E780E06A86
:1043500017F5FF1F1305C50297600100E780805322
:1043600017D50100130545C297600100E780606B17
:10437000AA8497700000E78060A797100100E7808B
:10438000C04297900100E780E0DB97800000E78063
:10439000400397700000E780601D97400100E780B0
:1043A000200497D501009385A5B717C50100130513
:1043B000253D99C897B00100E78060DCA68517D538
:1043C00001001305A5C6B9B797B00100E78020DB4F
:1043D00017D501001305C5C797B00100E78020DAA3
:1043E000294597B00100E78060DE97400100E78033
:1043F00000E097000100E780C0FE6DC585453705E8
:10440000040097300000E780804B97D5010093852A
:1044100025B117C501001305A53697B00100E78047
:1044200000D617D50100130525C497B00100E78019
:1044300000D5294597B00100E78040D997F7FF1FC5
:10444000938707E783D70700171700202317F73054
:10445000854717170020230FF71E97F7FF1F938735
:10446000A7F5DC4703D70700C167FD176316F70000
:1044700097000000E780009B97700000E780807E37
:104480008567938707E33E9597700000E780407E3D
:1044900097200000E780A038171500200355E52B72
:1044A00097600000E7808080054597600000E78006
:1044B00060B397600000E780E0D897D5010093854E
:1044C00025A617C501001305A52B97B00100E780AD
:1044D00000CB17D501001305A5BE97B00100E780FA
:1044E00000CA2DBD97000000E78080C39707002019
:1044F0002397A7C497D50100938585A217C501000E
:104500001305052897B00100E78060C717D60100A2
:104510001306C6B79705002083D565C217D50100DD
:10452000130545B797B00100E78060C5294597B0EE
:104530000100E780A0C93C4C1306000A894517F525
:10454000FF1F034525328297014597600000E780F1
:1045500060A9A5B7411122C437E404008327041AD7
:1045600006C6829797500000E780007883270408EA
:104570001715000013058542829797F7FF1F2383C5
:10458000A72E17F5FF1F130525E397500000E780BE
:10459000E0282244B2404101170300006700C3CB6A
:1045A000B7E70400FC471171A2DDCAD986DFA6DB9C
:1045B000CED72E8432892E86AA85170500201305B2
:1045C000A5B9829717070020130707B9834707008B
:1045D000930680029387E70793F7F70FE3ECF61053
:1045E000BA898A0717C701001307C722BA979C43E5
:1045F000BA9782878D4797D501009385A59417C5F3
:1046000001001305E517630FF40097B00100E78080
:1046100000B717C501001305A55197B00100E78049
:1046200000B6BDA497B00100E78060B517C50100D2
:104630001305855197B00100E78060B4294597B014
:104640000100E780A0B8930720F8114697050020E5
:10465000938585B04A8517070020230FF7AE97078B
:104660000020A38C07AE97F0FFFFE780E0742A8458
:104670001DC997D501009385E58C17C50100130569
:10468000251097B00100E78080AFA28517C5010013
:104690001305454F97B00100E78060AE294597B0FC
:1046A0000100E780A0B297D501009385A58917C5C1
:1046B00001001305E50C97B00100E78040AC17C579
:1046C00001001305654D97B00100E78040AB294517
:1046D00097B00100E78080AF4165930730FA054647
:1046E00097050020938545A77D1517070020230512
:1046F000F7A697F0FFFFE780206C2A841DC997D5A5
:1047000001009385258417C501001305650797B03F
:104710000100E780C0A6A28517C5010013058546E4
:1047200097B00100E780A0A5294597B00100E78078
:10473000E0A9B7E70400BC4F0566130606C8A1450B
:1047400017F5FF1F034505128297FE506E54DE5485
:104750004E59BE591161828091476303F40297C597
:1047600001009385257E17C501001305650197B0EB
:104770000100E780C0A017C501001305254571BDE4
:10478000B7E70400FC4F914517F5FF1F0345850D62
:10479000829797C501009385E57A17C50100130537
:1047A00025FE97B00100E780809D17C50100130525
:1047B000A54397B00100E780809C294597B0010090
:1047C000E780C0A097500000E78080CE914535A4D7
:1047D00085476303F40297C501009385A57617C545
:1047E00001001305E5F997B00100E780409917C56E
:1047F00001001305E54015B597070020239C278984
:10480000B7E704000566BC4F130606C8C1450DBFD7
:104810008D476303F40297C501009385A57217C500
:1048200001001305E5F597B00100E780409517C535
:1048300001001305A53ED5B3930740F8114697052F
:104840000020938565914A85170700202306F7907D
:1048500097070020A383079097F0FFFFE780C055DC
:104860002A84E30405EE97C501009385A56D17C55D
:1048700001001305E5F097B00100E7804090A285A4
:1048800017C501001305053097B00100E780208FA0
:10489000294597B00100E780609345BD9147E31C2F
:1048A000F4F6B7E70400FC4F9305000217F5FF1F6D
:1048B000034545FB829797C501009385A56817C5F9
:1048C00001001305E5EB97B00100E780408B17C5A9
:1048D000010013052536F1BD894763E3870297C5BB
:1048E00001009385256617C50100130565E997B09A
:1048F0000100E780C08817C501001305E53431BB0E
:104900009704002083C464859707002083C7D78459
:1049100097C5010093850563A20417C5010013051F
:1049200025E6DD8C97B00100E7806085A28517C57C
:1049300001001305A53297B00100E7804084C2044E
:10494000294597B00100E7806088C1849305D4FFB2
:1049500093960401C1824A8693F5F50F17F5FF1F60
:104960001305B57F97300000E78020F9E35F90DC06
:10497000930750F817F7FF1F2300F77E83C739000E
:10498000228697F5FF1F9385257D85074A8517F7B2
:10499000FF1FA304F77C97F0FFFFE780E0412A8424
:1049A000E30505DA97C501009385C55917C50100D0
:1049B000130505DD97A00100E780607CA28517D56F
:1049C000010013056580C9B5894763E3870297C570
:1049D00001009385255717C50100130565DA97A0D7
:1049E0000100E780C07917C501001305E52835B13E
:1049F00097500000E780C0ABA28517F5FF1F130595
:104A0000A57597500000E780E05481B38D4763039C
:104A1000F40297C501009385E55217C501001305FF
:104A200025D697A00100E780807517C50100130502
:104A30006526E5B6B76602000146B7750200054572
:104A400097E0FF1FE780E0D9930760F817F7FF1F93
:104A50002304F77097F7FF1FA381077093070006E1
:104A600017F7FF1F230CF76E894717F7FF1FA307E0
:104A7000F76E97F7FF1F2384076E97F7FF1FA3803A
:104A8000076EC14717F7FF1F230CF76C930720F938
:104A900017F7FF1FA306F76C314697F7FF1FA38296
:104AA000A76C97F5FF1F9385256B4A8597F7FF1F26
:104AB0002389076A97F0FFFFE78000302A84E30626
:104AC00005C897C501009385E54717C50100130583
:104AD00025CB97A00100E780806AA28517C5010059
:104AE0001305C51C55B3B1476303F40297C5010014
:104AF0009385454517C50100130585C897A001009A
:104B0000E780E06717C501001305051C39B6B7E754
:104B10000400FC4F9305000417F5FF1F034585D4DF
:104B2000829797500000E780A098B145F9B591476A
:104B300063E3870297C501009385C54017C501004F
:104B4000130505C497A00100E780606317C5010045
:104B500013054519D9B497F4FF1F83C4246097F750
:104B6000FF1F83C7975FA204DD8C8E04B777020016
:104B70006D14BE942286A68517C501001305C517BE
:104B800097A00100E780A05FB7E70400FC472286FA
:104B900097F5FF1F9385955C280082979316040173
:104BA000C1823000A685094597E0FF1FE78060C3FA
:104BB0002A8409C917C501001305C51597A001006E
:104BC000E780C073930770F8194697F5FF1F938528
:104BD000A5584A8517F7FF1F2300F75897F7FF1FBF
:104BE000A38E875697F0FFFFE780001D2A84E30E0F
:104BF00005B497C501009385E53417C50100130579
:104C000025B897A00100E7808057A28517C501004D
:104C10001305451195B99947630BF41297C5010027
:104C20009385453217C50100130585B597A001008E
:104C3000E780E05417C5010013054510F9BA914704
:104C400063E3870297C501009385C52F17C501004F
:104C5000130505B397A00100E780605217C5010056
:104C60001305450F5DBA97F4FF1F83C4244F97F7D0
:104C7000FF1F83C7974EA204DD8C8E04B777020016
:104C80006D14BE942286A68517C501001305C50DB7
:104C900097A00100E780A04EB7E70400FC472286FA
:104CA00097F5FF1F9385954B280082979316040173
:104CB000C1823000A6850D4597E0FF1FE78060B2F6
:104CC0002A8409C917C501001305C50B97A0010067
:104CD000E780C062930780F8194697F5FF1F938518
:104CE000A5474A8517F7FF1F2308F74697F7FF1FC9
:104CF000A386874697F0FFFFE780000C2A84E3062F
:104D000005A497C501009385E52317C50100130588
:104D100025A797A00100E7808046A28517C501005E
:104D20001305850795B699476303F40297C50100FB
:104D30009385452117C50100130585A497A001009F
:104D4000E780E04317C5010013058506F9B0B7E712
:104D50000400FC4F9305000417F5FF1F034585B0C1
:104D6000829797400000E780A074994579B18D47FC
:104D70006303F40297C501009385C51C17C50100A4
:104D8000130505A097A00100E780603F17C501004B
:104D90001305850359B017C501001305E50397A056
:104DA0000100E780A0551305C01297D0FF1FE780D0
:104DB0004059014597E0FFFFE780002E0D45971011
:104DC0000000E780E01E294597D0FF1FE78060576D
:104DD00097D0FF1FE780C0478DBA99476303F4025D
:104DE00097C501009385051617C501001305459960
:104DF00097A00100E780A03817C50100130585FEC4
:104E000029B817F7FF1F0347773597F7FF1F83C7A9
:104E1000E73422075D8F9166BA96C2061166C18299
:104E20001306F6EF8D476365D60297E7FF1F93875A
:104E3000A7589C4B17F6FF1F034636329386C700D0
:104E40002DC203D6070069CA8907E39CD7FE8947AC
:104E50001307A0F8114697F5FF1F9385E52F4A85A4
:104E600097F6FF1F238AE62E17F7FF1FA307F72EDB
:104E700097F0FFFFE78040F42A84E308058C97C58C
:104E800001009385250C17C501001305658F97A0B8
:104E90000100E780C02EA28517C501001305C5F5E6
:104EA000E5B203D60700630EE60A8907E39BF6FE28
:104EB0008D4779BF91476304F40297C5010093853C
:104EC000650817C501001305A58B97A00100E780B1
:104ED000002B17C501001305A5F36FF00FF4B7E71A
:104EE0000400FC4F9305000817F5FF1F0345859745
:104EF0008297C9B897C501009385C50417C50100FD
:104F00001305058897A00100E780602717C50100F9
:104F1000130585F16FF06FF02390E70017E5FF1F91
:104F20001305854997300100E780E05197C50100DE
:104F30009385450117C501001305858497A00100DD
:104F4000E780E02317C50100130505EF97A00100D6
:104F5000E780E022294597A00100E78020278147CC
:104F6000C5BD2390070017E5FF1F1305E5449730E3
:104F70000100E780404D97C501009385A5FC17B55A
:104F800001001305E57F97A00100E780401F17C5CA
:104F900001001305E5EB5DBFB7E70400FC474111D5
:104FA0002E8606C622C426C24AC02E842A89AA8515
:104FB00017F5FF1F1305451A829797C501009385C2
:104FC00025FA17B501001305A57B97A00100E7801E
:104FD000001B97F5FF1F83C5251817C50100130592
:104FE00025A097A00100E7808019294597A001001E
:104FF000E780C01D97F4FF1F9384041683C7040045
:1050000041479387070693F7F70F636FF75A17C760
:1050100001001307678A8A07BA979C43BA97828769
:105020009D476307F40297C50100938565F317B5A3
:1050300001001305E57497A00100E780401417C52F
:1050400001001305659A97A00100E780401395A41D
:1050500097F7FF1F83C75710DDCB17F7FF1F0347D5
:10506000D70F97F7FF1F83C7470F22075D8F97F76B
:10507000FF1F83C7A70EC2075D8F97F7FF1F83C768
:10508000F70DE207D98F17F7FF1F232DF70A83C704
:10509000640097C501009385A5EC17B501001305C1
:1050A000256E17F7FF1F230DF70897A00100E78073
:1050B000000D97F7FF1F9387E7088C4317F6FF1F34
:1050C0000346060817C501001305C59397A0010004
:1050D000E780E00A294597A00100E780200F97F7B5
:1050E000FF1FA38B07062244B24092440249930754
:1050F00000F817F7FF1F2301F7069D4517F5FF1F5F
:10510000130585054101175300006700A3E497705C
:105110000000E78060B497F7FF1F2380A704935730
:10512000850017F7FF1FA30AF702935705012A848A
:1051300017F7FF1F2304F70293578501014517F75F
:10514000FF1FA30DF70097700000E78040B597F7A9
:10515000FF1F2386A70097C50100938565E017B55B
:1051600001001305E56197A00100E780400117F6F3
:10517000FF1F0346C6FEA28517C501001305058A59
:10518000B1B7CD476303F40297C50100938545DDB0
:1051900017B501001305C55E97A00100E78020FE4A
:1051A00017C501001305058979BD97F7FF1F83C750
:1051B000C7FB17F7FF1F034737FBA207D98FC207AB
:1051C000C18717F7FF1F231CF7F6634AF00097F01B
:1051D000FFFFE780E0F497F7FF1F2392A7F6B7E7FA
:1051E000040003A387051306000A89452244B24040
:1051F0009244024917E5FF1F0345C566410102833A
:105200008D476303F40297C50100938565D517B5F3
:1052100001001305E55697A00100E78040F617C589
:1052200001001305E59005B517F4FF1F0344E4F2F0
:1052300097F7FF1F83C757F297C50100938545D2A3
:10524000220417B501001305A5535D8C97A001003A
:10525000E780E0F2A28517B501001305257F97A02E
:105260000100E780C0F1294597A00100E78000F622
:105270000D4697F5FF1F938525EE228597F0FFFFDA
:10528000E78080B3AA8421C197C50100938545CDED
:1052900017B501001305C54E97A00100E78020EE69
:1052A000A68517B501001305A57B97A00100E7802F
:1052B00000ED2244B240924402492945410117A31E
:1052C00001006700A3F097F7FF1F239587DCB7E77E
:1052D0000400116603A38705130606E8914539B754
:1052E0008D476303F40297C50100938565C717B521
:1052F00001001305E54897A00100E78040E817C5C5
:1053000001001305A59181B317F4FF1F0344E4E4E2
:1053100097F7FF1F83C757E497C50100938545C4DE
:10532000220417B501001305A5455D8C97A0010067
:10533000E780E0E4A28517B501001305A57397A0E7
:105340000100E780C0E3294597A00100E78000E85D
:105350000D4697F5FF1F938525E0228597F0FFFF07
:10536000E78080A5AA841DC197C50100938545BF2C
:1053700017B501001305C54097A00100E78020E0A4
:10538000A68517B501001305257005B797F7FF1F10
:10539000239487CEB7E70400116603A3870513069D
:1053A00006E89305000299B5894763E3870297C52C
:1053B00001009385E5BA17B501001305653C97A078
:1053C0000100E780C0DB17C501001305E587A5B91B
:1053D00097F4FF1F83C464D897F7FF1F83C7D7D7FD
:1053E00097C501009385C5B7A20417B50100130541
:1053F0002539DD8C97A00100E78060D8A68517B518
:1054000001001305E56997A00100E78040D7294511
:1054100097A00100E78080DB228697F5FF1F938528
:10542000A5D3268597F0FFFFE78000992A84630EB5
:10543000051A97C501009385A5B217B5010013059C
:10544000253497A00100E78080D3A28517B501001D
:105450001305456699BD854763F98718834519008B
:105460002244B24092440249B335B00097F7FF1F7F
:10547000238CB7C217B5010013050565410117A3B9
:1054800001006700C3CFA2852244B24092444A85FE
:1054900002494101171300006700C3B7994763032E
:1054A000F40297C501009385A5AB17B5010013055C
:1054B000252D97A00100E78080CC17C501001305BA
:1054C000659251B617F4FF1F034424C997F7FF1FD5
:1054D00083C797C897C50100938585A8220417B58F
:1054E00001001305E5295D8C97A00100E78020C924
:1054F000A28517B501001305A55E97A00100E780FE
:1055000000C8294597A00100E78040CC194697F5CF
:10551000FF1F938565C4228597F0FFFFE780C08950
:10552000AA841DC197C50100938585A317B5010005
:105530001305052597A00100E78060C4A68517B56F
:1055400001001305E55A95B397F7FF1F239E87BE09
:10555000B7E70400116603A38705130606E8930561
:10556000000869B1854797C501009385659F17B508
:1055700001001305E520630BF40097A00100E7800C
:1055800000C017B501001305E55775BC97A00100D1
:10559000E780E0BE17B501001305455897A001004C
:1055A000E780E0BD294597A00100E78020C22244A2
:1055B000B2409244024997F7FF1F239207B8410176
:1055C000176300006700C35997C50100938545998B
:1055D00017B501001305C51A97A00100E78020BA8E
:1055E00017C5010013054584B9BCB240224492445A
:1055F000024941018280411106C622C426C239C136
:105600002A8497F00000E780C0DDAA8411EDB7E797
:105610000400BC474146814522858297B24022441E
:10562000268592444101828041657D1597F00000F6
:10563000E78000DCB7E7040001E9BC47414681454B
:10564000228582978144D9BF0347E501FC47930532
:10565000900819E393050003AA9541462285829795
:1056600085446DBF93170501C1876359F00297F711
:10567000FF1F2395A7AC854717F7FF1FA30EF7AAB7
:10568000B7E7040003A387050566130606C893055C
:10569000002017E5FF1F0345E51C028382804111AE
:1056A00026C206C622C44AC083470500AA849DC7F5
:1056B00097C501009385C58417B501001305450CF6
:1056C00097A00100E780A0ABCC4017C501001305EF
:1056D000A5B697A00100E78080AA95AA5841B70710
:1056E000CF009387777D6313F7120359C500854771
:1056F00000458354E50063F3270F03470400034686
:105700001400F17693178700D18FC207C187938663
:10571000C6556393D7029707002083D70704638990
:10572000970A22852244B2409244CA850249410127
:1057300017E3FFFF6700C3AA954763F1270B9307A1
:105740003005631DF708930750046319F608834674
:105750002400930710046393F60883473400639F83
:10576000E706034744009307B0046319F7060347AD
:105770005400930790056313F706A947014563FF9B
:105780002701B7E70400DC5F2D4697C5010093852C
:1057900025AC228582977D151335150097F7FF1FDD
:1057A000238DA798268597000000E780E0EBB7E7F8
:1057B0000400BC4F130600059305004017E5FF1FCA
:1057C0000345450A829797F7FF1F83C70797B1DB09
:1057D000B24022449244024941018280970700204E
:1057E00083D7A7F763889700CA85228597E0FFFFD4
:1057F000E780009F22852244B2402686CA859244D3
:105800000249410117F3FFFF6700C3D9B707CC0076
:105810009387777D6317F70497B501009385456EED
:1058200017B501001305C5F597A00100E780209585
:105830009C4483D6E40083D5C40003C6070017C583
:1058400001001305A5A197A00100E7804093224421
:10585000B240924402492945410117A30100670063
:10586000E396B707CE009387777DE303F7F697B506
:1058700001009385E56817B50100130565F097A051
:105880000100E780C08FCC4017C501001305C5900B
:1058900089B597F7FF1F83C7378AB9C397F7FF1FEB
:1058A000A38C0788B7E70400FC4F411122C406C649
:1058B0002A849305002017E5FF1F0345A5FA829768
:1058C000854711C897F7FF1F9387478783D707003E
:1058D0002310F4008547B24022443E854101828076
:1058E0003E85828017F5FF1F03450585828097F767
:1058F000FF1F83C76784637BF50097F7FF1F9387BC
:10590000E78206053E9503550500828001458280A9
:105910000111854622CC4AC84EC652C406CE26CABC
:105920002A8A2E89328497E0FFFFE7800078AA89CF
:10593000630B09049307F4FFC207C1835D476364E7
:10594000F704B7E40400FC442286CA8517E5FF1F6C
:105950001305057C829797E7FF1F2398877C97E7BD
:10596000FF1F2395477B894717E7FF1F230EF77A11
:10597000BC4C8565130600329385058017E5FF1F33
:10598000034545EE8297F24062444E85D244424937
:10599000B249224A056182805D71A2C486C6A6C250
:1059A000CAC04EDE93F715002E84B5CB97E0FFFFFB
:1059B000E7804047930710F817E7FF1F230EF7789B
:1059C00097E7FF1F83D7C76A17E7FF1FA306F7787C
:1059D0009145A18317E5FF1F1305057817E7FF1F02
:1059E000230DF77697E7FF1FA389077697400000FE
:1059F000E7804056B7E70400BC4F13060014930538
:105A0000001017E5FF1F0345E5E5829713451400D5
:105A1000B640264496440649F25961618280856405
:105A200093840480B3F79500A5CB97E7FF1F83C746
:105A3000A76FA1CF17E6FF1F0356266F39C685460D
:105A400097E5FF1F9385C56C17E5FF1F0355056C90
:105A500097E0FFFFE780606597E7FF1F9387C76CBC
:105A600083C70700FD1793F7F70F17E7FF1F230DF5
:105A7000F76A81CFB7E70400BC4F13060032A68552
:105A800017E5FF1F034505DE8297056513050580B1
:105A9000218D42054181ADBF93F70540A5C397E72E
:105AA000FF1F83C7876997B60100938626E589E7BC
:105AB00097B60100938606E6814793053002338747
:105AC000F6000307070013960701418209C7639197
:105AD000B7021306300217E5FF1F0355256611C5EF
:105AE0006C0097000000E780E0E2134504400DB72A
:105AF00070003E962300E6008507D1B793F7052096
:105B000081CB97E7FF1FA389076213C5052009B75B
:105B100093F70510B1C3054597400000E780804C1E
:105B200017050020035565C397400000E780001863
:105B300097100000E780A0CE97E7FF1F83C757713B
:105B400089E797400000E780206E97400000E780DB
:105B5000606F134504106DBD93F72500E9CF17E77B
:105B6000FF1F0357C75D69C7AD64B7190040938431
:105B7000A4AA23A0990097E6FF1F9386A65C9442EF
:105B800097B701009387476917E6FF1F0346465BF7
:105B9000814517B501001305256997600000E7806E
:105BA00040EC23A0990097D7FF1F239BA7702A8959
:105BB00041C197B501009385A53717B501001305BD
:105BC00025BC97900100E780805BCA8517B501006E
:105BD000130505D697900100E780605A29459790F4
:105BE0000100E780A05E97E7FF1F239A0754930701
:105BF00010F817E7FF1F2301F75697E7FF1F83D71A
:105C0000274717E7FF1FA309F754A18317E7FF1FD3
:105C10002305F75491458D4717E5FF1F1305C5531D
:105C200017E7FF1FA30BF75297400000E780803271
:105C300013452400F1BB93F74500D1C397B501008C
:105C40009385052F17B50100130585B397900100C3
:105C5000E780E05217B50100130545CF979001008A
:105C6000E780E051294597900100E780205693078F
:105C700020F817E7FF1F2301F74E97E7FF1F83D791
:105C8000674117E7FF1FA309F74CA18317E7FF1F21
:105C90002305F74C854717E7FF1FA300F74C9740F4
:105CA0000000E780E08017E5FF1F1305E54A9145F6
:105CB00097400000E780002A1345440091BB93F70A
:105CC0008500A9C797B501009385852617B5010002
:105CD000130505AB97900100E780604A17B50100F6
:105CE000130505C897900100E78060492945979002
:105CF0000100E780A04D97E7FF1F239207449760BC
:105D00000000E780E0E51345840019B393F705012F
:105D1000D1C3854517E5FF1F0355C53797500100CF
:105D2000E780E09A97B501009385852017B50100BB
:105D3000130505A597900100E780604417B50100A1
:105D4000130545C397900100E7806043294597906C
:105D50000100E780A047930730F817E7FF1F230DE6
:105D6000F73E97E7FF1F83D7E73217E7FF1FA3052B
:105D7000F73E17E5FF1F1305253EA1838D4517E765
:105D8000FF1F230CF73C97400000E780A01C134541
:105D90000401BDB993F70502D1C797B501009385FA
:105DA000251917B501001305A59D97900100E780FF
:105DB000003D17B50100130525BE97900100E7804F
:105DC000003C294597900100E7804040930740F848
:105DD00017E7FF1F2302F73897E7FF1F83D7C7296D
:105DE00017E7FF1FA30AF736A18317E7FF1F230654
:105DF000F736854717E7FF1FA301F73697E7FF1F21
:105E0000239C072697300000E780806A17E5FF1F74
:105E100013058534914597400000E780A013134592
:105E20000402FDB693F70504FDC397B50100938501
:105E3000251017B501001305A59497900100E78080
:105E4000003417B501001305A5B697900100E7804F
:105E50000033294597900100E780403797E7FF1FFF
:105E600083C7872F1307700A6386E7061307800A24
:105E7000638CE7081307600A6393E704930760F8ED
:105E800017E7FF1F230AF72C97E7FF1F83D7E727A2
:105E900017E7FF1FA302F72CA18317E7FF1F230EAD
:105EA000F72A854717E7FF1FA30DF72AB14517E526
:105EB000FF1F1305652A97400000E780A00997306F
:105EC0000000E780E05E1345040497E7FF1F239E70
:105ED00007223DBE930770F817E7FF1F230EF72632
:105EE00097E7FF1F83D7672217E7FF1FA306F72651
:105EF000A18317E7FF1F2302F726854717E7FF1F38
:105F0000A30EF724994565B7930780F8F1B793F787
:105F100005080145E38E07AE97B50100938545015D
:105F200017B501001305C58597900100E78020256E
:105F300017B50100130545A997900100E7802024BB
:105F4000294597900100E78060289307A0F817E79C
:105F5000FF1F2303F72097E7FF1F83D7E71E17E7ED
:105F6000FF1FA30BF71EA18317E7FF1F2307F71ED1
:105F7000854717E7FF1FA302F71E97E7FF1F23952B
:105F8000071C97300000E780A05217E5FF1F13059C
:105F9000A51C914597400000E780C0FB134504080D
:105FA00085BC814617E3FFFF67002310411122C41F
:105FB00091462A8417E6FF1F130646289D652D4546
:105FC00006C697D0FF1FE780C081B7F7070003C759
:105FD0000701A5476313F70001A0930600100146CF
:105FE0009D65254597C0FF1FE780A07F97E7FF1FAE
:105FF000238687242244B240914617E6FF1F1306EA
:10600000E6239D652945410117C3FF1F6700637D96
:106010001171CED7B7E9040083A7C904CAD917E91B
:10602000FF1F13096913A2DD2E8686DFA6DB2E84EF
:10603000AA854A85829797E7FF1F83C7E711130751
:10604000700A6385E710636DF7001307600A6385C4
:10605000E704FE506E54DE544E59BE5911618280E1
:106060001307800A6385E7161307900AE393E7FE98
:106070008D476306F41C97B501009385A52917A5E4
:1060800001001305E56F97900100E780400F17B5F9
:1060900001001305652525A08D47630CF40297B513
:1060A00001009385252717A501001305656D9790BD
:1060B0000100E780C00C17B501001305251C97905F
:1060C0000100E780C00B294597900100E780001090
:1060D00049B7854717B501001305051C17E7FF1FD2
:1060E0002304F7FC97900100E7804021B775020078
:1060F000B76602000146054597C0FF1FE780606E46
:10610000930760F817E7FF1F2308F70497E7FF1FBF
:10611000A38507049307002617E7FF1F2320F70432
:10612000E5779387072117E7FF1F231BF702B14588
:1061300097E7FF1F2387070297E7FF1FA383A702A5
:106140004A8597000000E780E01621B7914763E396
:10615000870297B501009385E51B17A5010013057C
:10616000256297900100E780800117B501001305B3
:10617000A514B1B797E4FF1F83C444FE97E7FF1F40
:1061800083C7B7FDA204DD8C83A7C9046D142286E2
:1061900097E5FF1F938595FC280082978E04931640
:1061A0000401B7750200C1823000A695094597C069
:1061B000FF1FE7800063930770F817E7FF1F230DA9
:1061C000F7F8994597E7FF1FA38AA7F895BF91476E
:1061D00063E3870297B501009385C51317A50100F6
:1061E0001305055A97900100E78060F917B5010083
:1061F0001305050EE9B597E4FF1F83C424F697E75E
:10620000FF1F83C797F5A204DD8C83A7C9046D1413
:10621000228697E5FF1F938575F4280082978E04E8
:1062200093160401B7750200C1823000A6950D4592
:1062300097C0FF1FE780E05A930780F8BDBF17B5EE
:1062400001001305A50B97900100E780200B930731
:1062500090F82304F100834719008D452800A3041A
:10626000F100834729002305F10097000000E78033
:1062700060041305C01297C0FF1FE780800C014522
:1062800097D0FFFFE78040E10D4597000000E780D1
:1062900020D2294597C0FF1FE780A00A97C0FF1FA3
:1062A000E78000FB7DB397E7FF1F23A1A7FA828059
:1062B00097E7FF1F938787F903A307006303030092
:1062C0000283174300006700E3C841114AC097F6F4
:1062D000FF1F83D68648328917D6FF1F0356E60F65
:1062E00022C426C206C62A84AE8497000000E78036
:1062F000406829C921C8994763F697048347140069
:1063000003470400A207D98F13978700A183D98F71
:10631000C2073167C1831307C7556395E70297D753
:10632000FF1F83D7870BA301F400A1832302F4008E
:1063300097F7FF1F83D7674291C7A302F400A18399
:106340002303F40097F7FF1F83C7C730A1CB26862E
:10635000A28517D5FF1F0355450897000000E78069
:1063600080C4630F090297F7FF1F83C7A72E8DEB29
:1063700097E7FF1F83C7C7ED85C79DC097E7FF1F3E
:1063800083C787D291EF22852244B2400249A68575
:1063900092444101174300006700C3BBE31A09FCA4
:1063A000B240224492440249410182808347550011
:1063B0008345450017B50100130585F8A207DD8D5B
:1063C000179301006700A3DB17B50100130545F61D
:1063D00017930100670083F28D4763F6B708011138
:1063E00026CA06CE22CC0344350097E4FF1F83C49F
:1063F00034E697B501009385E5F5B337800017E7DC
:10640000FF1FA307F7E409C497B50100938545F57D
:1064100017B50100130545F597900100E78020D6D8
:1064200097E7FF1F83C7D7E26386970097000000B6
:10643000E780004397400000E780C0E099679387BA
:1064400057EE2316F100680085479145A3078100A8
:106450002307F10097000000E780C0E5F2406244A6
:10646000D244056182808280894763F7B7080111B1
:1064700022CC06CE26CA8344250085472A84639D04
:10648000F404914763F5B70403454500834734009E
:1064900022055D8D97D7FF1F2391A7F49700000079
:1064A000E78000569967938767EE2314F1008347CE
:1064B000340023059100A305F1008347440095456E
:1064C00028002306F10097000000E780A0DEF240DC
:1064D0006244D24405618280FDF89967938767EE34
:1064E0002314F10097D7FF1F83D727EFA305F100EF
:1064F00023050100A183E1B782800111996722CCB5
:10650000D51717F4FF1F1304E4142314F100834775
:10651000040026CA97F4FF1F938424242305F10066
:1065200083D7040028009545A305F100A18306CE7A
:106530002306F10097000000E780C0D703D60400CF
:106540008345040017B50100130505E3979001008A
:10655000E780E0C2F2406244D244056182809D67D8
:106560007971D9172316F10097F7FF1F9387870ECC
:1065700083C707001305F10006D62307F10097F043
:10658000FFFFE780800709E9B7E70400BC47414601
:1065900081451305F10082976800CD459700000002
:1065A000E78040D197F5FF1F83C5C50A17B50100E5
:1065B000130585DF97900100E78060BCB25045610C
:1065C000828063080516411126C206C622C44AC04D
:1065D00097E7FF1F83C7D7C797F4FF1F83C48407BC
:1065E00099C393E424002A8497100000E78020E3F5
:1065F00019C193E4040137E9040083278904228543
:106600001306200381458297930750FA2300F40074
:106610009307A005A300F4008D472301F4009147E0
:10662000A301F40093070005A302F40097F7FF1FEE
:1066300083D7A7122304F400A183A304F40097D7FF
:10664000FF1F83D787D9230394002305F400930405
:10665000C400A18323020400A305F400268597F05B
:10666000FFFFE78080F919E58327890441468145CA
:106670002685829797D7FF1F83D7C7D3230EF400B1
:10668000A183A30EF40093070002230FF4009307E5
:1066900010FAA30FF4009D472300F402A3000402A4
:1066A000B7E70400FC4713052402194697D5FF1FDE
:1066B0009385851B829797E7FF1F83D7479F230406
:1066C000F402A183A304F40297E7FF1F83D7E79D99
:1066D0002305F402A183A305F40297E7FF1F938724
:1066E000E79C839707002285930500032306F402A5
:1066F000C207C183A183A306F40297D7FF1F938724
:1067000027BC839707002307F402C207C183A18334
:10671000A307F40297000000E780A0212308A40249
:106720002181A308A402B2402244924402494101BB
:10673000828082805D71E17793C777FF1305E10066
:1067400086C62316F10097000000E780C0E76800C6
:106750009305400397000000E780C0B5B640616133
:1067600082805DC9411122C426C206C6930750FA31
:106770002300F5009307A005A300F5008947230136
:10678000F5009147A301F50093070005A302F5006A
:1067900097F7FF1F938707EC83C707009304C50093
:1067A0002A842303F50097E7FF1F938777AA83C7FF
:1067B000070023020500A303F50097F7FF1F83D707
:1067C000C7F92304F500A183A304F50097D7FF1FA1
:1067D00083D7A7C02305F500A183A305F50026856F
:1067E00097F0FFFFE78060E101E9B7E70400BC47ED
:1067F00041468145268582972285F1459700000014
:10680000E7802013230EA4002181A30EA400B24030
:10681000224492444101828082805D710A8586C64D
:10682000A2C497000000E78000F437E404007C4431
:106830008A850810794682973C441305E10309468E
:1068400081458297101093050002014597D0FFFF04
:10685000E780C0EAB6402644616182800111B7C773
:10686000A55A22CC9387C73317E4FF1F1304549E05
:106870003EC483470400856601469965254506CEDA
:106880003EC697C0FF1FE780C0F53000A14699655E
:10689000294597C0FF1FE780C0F48345040017B562
:1068A00001001305E5BA97900100E780408DF240A2
:1068B0006244056182800111A146300099652D4531
:1068C00022CC06CE97C0FF1FE780A0F1A24737C4B5
:1068D000A55A1304C43363958702B24517B5010066
:1068E0001305C5AEB335B00097E7FF1FA382B79677
:1068F00097900100E780A088F240624405618280A1
:106900009165A1463000938505F02D4597C0FF1F86
:10691000E78020EDA247E38287FC97E7FF1FA3896A
:106920000792814517B50100130585ACD1B7C16742
:1069300069768146FD170506139706014183636456
:10694000B7003E8582803307D50003470700B98F23
:10695000214713F81700858363050800B18FC2072C
:10696000C1837D171377F70F6DF78506F1B741C522
:10697000A547054763F2B70883471500034705009D
:106980003168A207D98F13978700A183D98FC207D7
:10699000C1831308C855054763900707411106C610
:1069A00022C426C203442500914763F0870493075D
:1069B000540063ECF502A301C50021822302C50047
:1069C0009304340091C6A302D500A1822303D5000D
:1069D0002A84A68597000000E780A0F5269423006E
:1069E000A4002181A300A4000147B24022449244A4
:1069F0003A854101828005473A8582800111B7C7F7
:106A0000A55A22CC9387E7342A842AC68566014694
:106A10009565254506CE3EC497C0FF1FE78060DC24
:106A20003000A1469565294597C0FF1FE78060DBD0
:106A3000A28517B501001305A5A397800100E78083
:106A4000007497000000E78080DDF2406244056139
:106A500082800111A146300095652D4522CC06CEDD
:106A600097C0FF1FE780E0D7A24737C4A55A130499
:106A7000E43463958702B24517B5010013054599C3
:106A800097D7FF1F239BB794C205C1819780010050
:106A9000E780E06EF2406244056182809165A14624
:106AA0003000938505EE2D4597C0FF1FE78060D32A
:106AB000A247E38287FCD14717D7FF1F231FF79018
:106AC000D14517B501001305A596C9B7011122CC10
:106AD0002A841305E10026CA06CEAE8497F0FFFF94
:106AE000E78060DB09C90355E1002686A28597F09F
:106AF000FFFFE78020E2A685228597100000E7804F
:106B0000A09297D7FF1F83C7A77499C7A685228530
:106B100097300000E7800044F2406244D2440561AF
:106B2000828001114EC606CE22CC26CA4AC893F7EF
:106B30001500AE899DCBAD67371700409387A7AA94
:106B40001CC3B7E70400BC4F13060019854517D5D1
:106B5000FF1F03456588829713C51900F240624400
:106B6000D2444249B2490561828093F7250001452C
:106B7000F5D717F7FF1F035727BE954763FAE70CB2
:106B8000014417F6FF1F130626AD930630051305C3
:106B90005004130810049308B004130390059307DE
:106BA00064006374F7043A847D5997F4FF1F83C42B
:106BB000A4AA97F7FF1F83C737AAA204DD8CAD678D
:106BC0009387B755638CF41463E4970AA967938796
:106BD000A755638FF414A28517F5FF1F1305C5A7EA
:106BE00097000000E780C0EEF1A0B307860083C5E0
:106BF0000700639BD50483C517006397A50483C56D
:106C000027006393050583C53700639FD50283C5BD
:106C10004700639B150383C7570063976702228968
:106C200015E897F5FF1F83D525B3B3852541C20528
:106C3000C181F1CD17F5FF1F130505A24A959700F5
:106C40000000E780E0E8E1A005044204418081BF44
:106C50003A847D598547E3EA87F45DC4854517F595
:106C6000FF1F1305659F97000000E78060E669A895
:106C7000B1679387C7556389F404B5679387D75580
:106C8000E39BF4F4A28517F5FF1F1305E59C9730ED
:106C90000000E780202C8947630EF4009305E4FF91
:106CA000C205C18117F5FF1F1305259B9700000042
:106CB000E7808077A68517A501001305257D9780BD
:106CC0000100E780C04B89A097200000E780E01D0D
:106CD00097000000E780A07411C9A28517F5FF1F77
:106CE0001305859797000000E78000740546A2858C
:106CF00017F5FF1F1305459697F0FFFFE780205D0E
:106D000097200000E780601AFD57E31CF9F097F721
:106D1000FF1F239307A413C5290089B5A28517F582
:106D2000FF1F1305659397F0FFFFE780606859B771
:106D3000A28517F5FF1F1305259297F0FFFFE78047
:106D4000E0688DBF411122C437E404005C5C06C6D4
:106D5000354697A501009385252A17B5010013052F
:106D6000E5FF829711E917A5010013056573978068
:106D70000100E780A05801A08327041C82972A8481
:106D8000054597C00000E780E00B97700100E780A1
:106D9000009197600100E780006697B00000E780EF
:106DA000601D2285B2402244410182804111054587
:106DB00006C622C426C297C0FFFFE780C01713058E
:106DC000A00497B0FF1FE780802E757585457D155F
:106DD00097C0FFFFE78060017D7585451305F53697
:106DE00097C0FFFFE780C00A371400408327840A5A
:106DF0008D451305002093E707202324F40A97C04C
:106E0000FFFFE78080FEB7E4040097C0FFFFE78044
:106E1000A043C85897800100E780404E17B5010095
:106E20001305C5F397800100E780404D8327840C4C
:106E30008545414593E707082324F40C97C0FFFFDD
:106E4000E78000058D451305000897C0FFFFE78028
:106E5000200497C0FFFFE780003137A50700130526
:106E6000051297C0FFFFE780A02C014597C0FFFFE8
:106E7000E780C03295450545894717F7FF1F230F67
:106E8000F78C97C0FFFFE7800033B7E700E01307F8
:106E90000006238DE7403707000423A0E71097D0B2
:106EA000FFFFE78080B497D0FFFFE78080C69700A0
:106EB0000000E78060E997000000E78000A09700ED
:106EC0000000E78040B997D0FFFFE780E0689700B7
:106ED0000000E780A05697000000E780801083A79D
:106EE000040817050000130505C4829797C7FF1F04
:106EF0002384A74EBC4C130600648545829797B047
:106F0000FF1FE780E04E01458280AD6737170040E4
:106F10009387A7AA1CC3B7E700E03707400023A068
:106F2000E71801000100B7F7070003C70701A547ED
:106F30006316F7009397450191C301A04111AE86F6
:106F40000146AA85254506C697C0FF1FE7806089D0
:106F5000B240B7E700E03707400023A0E710410147
:106F600082804111B2862E86AA852D4506C697C01D
:106F7000FF1FE7800087B2400145410182809307EF
:106F8000000463ECC7041D71A2CC2A840808A6CAB9
:106F9000CAC886CE32C697800100E780E012AD678E
:106FA000371700409387A7AA1CC3B7E400E037094E
:106FB000400023A0241901000100B2461008A28558
:106FC000294597C0FF1FE780C081F640664423A093
:106FD0002411D64446492561828039558280411169
:106FE0000D658D4506C697C0FFFFE78000E0B71727
:106FF00000408D6623A6D70A17E5FF1F13054576C7
:107000001387C70A9387870A1CC15CC58566896791
:107010005CC958C114C518C9B7E70400B24003A33E
:10702000871E410102838145B307B50083870700AE
:1070300089E7172300006700E3ED8505C205C181DC
:10704000E5B7011106CE2307010001ED17A50100E8
:107050001305456C97000000E78020FDF2400561B4
:1070600082805800A947BA8529462548B376C502CB
:10707000FD1793F7F70F93860603A304D700B356C3
:10708000C5026375A8007D173685EDF33385F500DD
:10709000D1B797A70100938727681357C5003E977C
:1070A00003470700011106CE2304E10013578500B2
:1070B0003D8B3E970347070023060100A304E10030
:1070C000135745003D8B3D893E97AA97034707001C
:1070D00083C7070028002305E100A305F1009700FE
:1070E0000000E78080F4F24005618280797117A585
:1070F00001001305655B06D622D426D24AD04ECEB7
:1071000097000000E78060F217E5FF1F0355E56474
:1071100097000000E78020F897E7FF1F83C7875399
:1071200017A501001305C55589C717A5010013054B
:10713000A55497000000E78040EF17A50100130554
:10714000E55697000000E78040EE17A50100130503
:10715000655697000000E78040ED1145970000005C
:10716000E78060EE17B50100130545B397000000F6
:10717000E780A0EB014597000000E780C0EC17B561
:1071800001001305A5B197000000E78000EA130590
:10719000000597000000E78000EB97D7FF1F83C72B
:1071A000370B17A501001305254E89E717A5010028
:1071B0001305054E97000000E78020E717A50100A2
:1071C0001305C54F97000000E78020E637A50700AC
:1071D0001305051297000000E780E0E617A50100FF
:1071E0001305454E97000000E78020E497E7FF1F56
:1071F00083C7875817A501001305054A89E717A516
:1072000001001305E54997000000E78000E217A59B
:1072100001001305E54B97000000E78000E117A58A
:1072200001001305654B97000000E78000E017A5FB
:1072300001001305E54A97000000E78000DF17C54D
:10724000FF1F0355251797000000E780C0E417A52E
:1072500001001305254997000000E78000DD17C5F0
:10726000FF1F0355851797000000E780C0E217A5B0
:1072700001001305A54797000000E78000DB17D544
:10728000FF1F0355C5E297000000E780C0E017A587
:1072900001001305254697000000E78000D917D5A7
:1072A000FF1F035585E097000000E780C0DE17A5AB
:1072B00001001305A54497000000E78000D717D50B
:1072C000FF1F0355A5DE97000000E780C0DC17A56F
:1072D00001001305E54297000000E78000D517C5BF
:1072E000FF1F0355E5FD97000000E780C0DA17A5F2
:1072F00001001305654197000000E78000D30144B9
:1073000097C9FF1F9389495697A401009384C440ED
:107310001949B307340183C707000A85050413D749
:107320004700BD8B2697A6970347070083C7070032
:10733000230101002300E100A300F10097000000F9
:10734000E780A0CEE31724FD17A501001305453CF7
:1073500097000000E78060CD0A8597E0FFFFE78097
:10736000C0290A8404088347040003451400090463
:10737000A2075D8D97000000E780E0D1E39584FED1
:10738000B250225492540259F2494561828041110F
:1073900026C2E97797E4FF1F9384044D22C49387A4
:1073A000A7552E842381B4002E86AA8517E5FF1FDA
:1073B0001305C54B06C62390F400A38104009780F3
:1073C0000100E78060D093052400C205C18117E564
:1073D000FF1F1305854997F0FFFFE7808055B387AE
:1073E00084002382A7002181A382A7009305640063
:1073F0002244B24026859244C205C181410117232F
:107400000000670023B109C99307000463E6B700D1
:10741000170300006700E3F7828017E5FF1F0345AD
:10742000A535828097E7FF1F83C7C74389E71723E6
:107430000000670023AE828097E7FF1F83C72747BE
:1074400099EF411106C697200000E78080A4B24062
:10745000854717E7FF1F230CF74441018280828094
:10746000630C0544638A05441D71CAC8CEC686CE26
:10747000A2CCA6CAD2C4D6C2DAC05EDE62DC66DAAC
:107480006AD86ED6B947AA892E8963F9B7063946F4
:1074900097A501009385050A97800100E78060C0E9
:1074A00031ED83C7E900130710036394E7028547B2
:1074B00017E7FF1F2308F73A17A5010013058508F2
:1074C00097E7FF1F239F073897000000E780E0B58C
:1074D000E5A01307000317A501001305A509E3950F
:1074E000E7FE97E7FF1F238F073697E7FF1F239AD3
:1074F000073617A5010013056506F9B797E4FF1FC6
:1075000083C44436639F0428B706400001475946A8
:10751000A50613140701418063792439338AE900F1
:1075200083470A00D91793F7F70F6367F600B3D7BD
:10753000F600858B0507F1FF330489404204418042
:10754000BD4763FE8726414697A501009385C50484
:10755000528597800100E780C0B46314052617A503
:1075600001001305A50497000000E78000AC970018
:107570000000E780E0B717A5010013056580A9B7F3
:10758000B387490183C6070097E7FF1F83D7672D9D
:10759000B9E39307A005639BF600854717E7FF1F34
:1075A0002311F72C97E7FF1F238AD71C050A93178F
:1075B0000A01C183E3E627FDF6406644D644464906
:1075C000B649264A964A064BF25B625CD25C425D43
:1075D000B25D25618280854D639BB7039307500A96
:1075E000639EF600894717E7FF1F231CF7269307C2
:1075F00050FA17E7FF1FA303F7184DBF9307A00525
:10760000E386F6FA97E7FF1F239D072445B7138704
:1076100017004207DA9741832380D70017E6FF1F40
:107620002311E6248D47E3F3E7F817E4FF1F034433
:10763000141597E7FF1F83C7871422045D8C9307F7
:10764000F4FFC207C1839306F00DE3EDF6FA93074A
:107650006400C207C183E31BF7F493052400C2054D
:10766000C18117E5FF1F1305851197F0FFFFE78024
:10767000402C33078B008347570003474700A2077E
:10768000D98F17E7FF1F231E071C6311F5108144D4
:10769000630CB40197E4FF1F83C4840EA20497E730
:1076A000FF1F83C7F70DDD8C170500001305E5D517
:1076B00097F0FFFFE78060BF6385740963EF9B026B
:1076C0006388A4059307EC656383F40697E7FF1FBF
:1076D00083C7070B05476380E70881CB1387A7059E
:1076E0001377F70F8D4663F9E6081307F0072300B9
:1076F000E100A300F100894595A86389940593876B
:10770000FA77E395F4FC97F0FFFFE780E00211A819
:10771000A28517E5FF1F1305A50697F0FFFFE78079
:10772000E0CB014597F0FFFFE78020B841B5A28587
:1077300017E5FF1F1305C50497F0FFFFE78000D38F
:10774000CDB797F0FFFFE78080DBE1BF97F0FFFF49
:10775000E78020E1F9B7930710F813051100230023
:10776000F10097F0FFFFE7800000FD450A859700D4
:107770000000E78000C275B7A28517E5FF1F13055B
:10778000250097F0FFFFE780E08861BF9307F007CF
:1077900089450A852310F10097000000E78060BF4B
:1077A00031B5BD6A396C014A17EBFF1F130B0BFD96
:1077B000938BFA55938CFA66130DEC55CDBB63167B
:1077C000F40E3D4697A50100938585DF528597808D
:1077D0000100E780008D11E517A50100130545DFC5
:1077E00059B3C14763F3870C454697A501009385BC
:1077F00065DF528597800100E780A08A39E997E02C
:10780000FFFFE780600E2A8417A501001305C5DE7F
:1078100097000000E7806081228597000000E780E4
:10782000808217B901001309E9E9E30694D44A8577
:1078300097F0FFFFE780607F268597E0FFFFE780F6
:10784000400B850497000000E780E08493F4F40F78
:10785000E9BF414697A50100938585DB5285978056
:107860000100E780008431E183470A011307100318
:10787000639CE700854717E7FF1F230FF7EE17A567
:107880000100130525DA89B11307000317A50100CC
:10789000130545DCE39AE7C297E7FF1F238E07EC49
:1078A00017A50100130585D905B1CA854E8597C076
:1078B000FFFFE780E09209B38280411126C2AE84C7
:1078C0008D4522C406C62A8497B0FFFFE780405C3E
:1078D000B717004099C803A5C70C418D23A6A70C74
:1078E000B240224492444101828003A5870C418D1D
:1078F00023A4A70CF5B78347050003471500A2078B
:10790000D98FC2076177C18713072720639AE700E1
:10791000834525003705040017030000670023FA9C
:10792000828017E6FF1F1306E6F88147B28613032D
:10793000F00FA9483308F6000348080013F7F70FC3
:107940006307A80C630668008507E39517FF2947BE
:10795000B387E6002380A70097E7FF1F938747F6CA
:107960005DA8411113D765001347170006C693F6AB
:107970003500058B954791CA054699476387C60030
:1079800009469D476383C600A14713F64500333679
:10799000C00093F68503050685C2A145638BB60436
:1079A000E145638AB604930580026388B6049305B3
:1079B00080036393B600914697E5FF1F2387F51672
:1079C00097E5FF1F2382C51697E5FF1FA38ED514E9
:1079D000BE8517A50100130525D897700100E78023
:1079E000007AB240854717E7FF1FA300F714410153
:1079F00082808546D1B78946C1B78D4675BF17A528
:107A000001001305E5D7177301006700437717E7F7
:107A1000FF1F1307E7EABA972380B700E147E302A5
:107A2000F5F493077002E30CF5FC82802A8723802B
:107A30000500814717E5FF1F1305C5E71308F00F81
:107A40002946B306F50083C606006396E60297E66C
:107A5000FF1F9386E6E6B69783C707000545238098
:107A6000F5009947636EF7029D4763FDE700E14724
:107A7000630DF7008280638506018507E393C7FCE9
:107A80000145C5B7238005008280B737004003C792
:107A9000370083C7050093F70704D98F2380F500CB
:107AA00082805D7152DC56DA5ED6716A97EBFF1FF9
:107AB000938BCB188D6AA6C24EDE62D486C6A2C452
:107AC000CAC05AD866D26AD06ECEC1495E8C97E4DD
:107AD000FF1F9384A4DF130A0A20938A7ADC17E934
:107AE000FF1F0349A918B3872B0183C7070093F72A
:107AF000F70FC9EFB787004003C76700058BE31096
:107B0000077C03C76700118BE30D077E83C757000F
:107B1000918B99E36F10200317E7FF1F0347271589
:107B200085476304F7006F10400197E7FF1FA38E9E
:107B3000E7FE97E7FF1F238B07E497E7FF1F2389E3
:107B400007F097E7FF1F238707FC97E7FF1F2384B2
:107B500007FC97E7FF1FA38B07E297E7FF1FA389A7
:107B600007EE97E7FF1FA38707FA97E7FF1FA38496
:107B700007FA97E7FF1FA38B07FA97E7FF1FA38872
:107B8000070EB787004011476F0070779307190001
:107B900093F7F70F3D476364F70617E7FF1F2307C7
:107BA000F70C97E7FF1F9387670BCA9783C70700F8
:107BB0001307100293F7F703638EE71E6366F7045B
:107BC00005446385871CE38C07620947638EE710D1
:107BD00013070002E384E74EB7E700E037074000F1
:107BE00023A0E71801000100629923000900FD1994
:107BF00023A0E71093F9F90FE39309EEE5BD97E7AA
:107C0000FF1F2385070671BF130730026388E70C47
:107C100063E8E71613074002638CE70A13070003C3
:107C2000E39CE7FA97E7FF1F93874702CA9703C7CA
:107C30000700A1471377F70FE31BF71483C764000E
:107C400097E6FF1F238AF6EC97E7FF1F83C777C8E5
:107C500091C7FD5797E6FF1F2380F6EC97E5FF1FBE
:107C600083C5D5C697E7FF1FA388B7EA97E7FF1F2D
:107C700083C7C7C513FB07089306000493F70706DD
:107C8000639FD74C9307A009638DF51663EAB7127B
:107C90009307F0056386F54A930750096384F52A34
:107CA000014497E7FF1F83C737E71547E392E7369D
:107CB000B7E700E03707400023A0E7180100010004
:107CC000B786004023808602130680FC6F00500EAA
:107CD000FD5717E7FF1F2300F7E4FDBDFD5717E72A
:107CE000FF1F2309F7E2CDBD17A501001305C5BA93
:107CF00097700100E780806097E7FF1F938707F583
:107D0000CA9703C40700014B97ECFF1F938C8CD4D8
:107D10001374F40F17AD0100130D8DB863478B0476
:107D2000294597700100E780604A854717E7FF1FE4
:107D3000A300F7D217E7FF1F230D87D017E7FF1F18
:107D40002306F7DE37E700E0B70640002320D71808
:107D500001000100378600408347A60293F7370FE2
:107D60002305F6022320D71085BDB3876C0183C598
:107D700007006A85050B97700100E780404079BFD6
:107D8000854717E7FF1F2305F7CCB9B517E7FF1F96
:107D90001307C7EB4A970347070097E6FF1FA38720
:107DA000F6BE97E6FF1F2384E6BE17E7FF1F230FEB
:107DB000F7D61DB5854717E7FF1F2309F7BC29BD77
:107DC0009307400A6389F5349307200B6384F536E3
:107DD0009307100AE396F5EC838724000144E3D26D
:107DE00007EC97E7FF1F83C797AE93F63700638AC8
:107DF000061A0546638AC62209466395C61A1D47B8
:107E000055A217E5FF1F034585ACC94797ECFF1F37
:107E100083CCFCAB97E5FF1F83C585AB17E4FF1F41
:107E2000034414AB6315F510CD476392FC10930720
:107E30007008639CF5021307300FB7170E00630834
:107E4000E4001307900DB7B704006314E40817E7C4
:107E5000FF1F2329F7CCBE8517A501001305C5A474
:107E600097700100E780A03125BD93078008639DCE
:107E7000F500B307804013F4F70FB77746009387F8
:107E800087CDB3D78702E1B793079008639AF500CF
:107E9000B307804013F4F70F91679387C766D5B790
:107EA0009307A008639BF500B307804013F4F70F16
:107EB000B7173D0093870790E9B79307B008639A17
:107EC000F500B307804013F4F70F9167938797D0BD
:107ED0004DBF93F5F5078D47639BF500B3078040D1
:107EE00013F4F70FB7975B00938707D859BF8947FB
:107EF000639BF500B307804013F4F70FB7770B00CF
:107F00009387071BBDBF8547639AF500B307804081
:107F100013F4F70FDD67938767E3A5B7D28785F979
:107F2000B307804093F7F70FB3D7FA020DB7970066
:107F30000000E780409FA285668597000000E780EB
:107F4000809EB9BB9305610017E5FF1F0345259887
:107F500017E4FF1F0344B49797000000E78040AD8B
:107F600093057100228597000000E78060AC3C001B
:107F700017E7FF1F2322F7CC834761002304F1009A
:107F800083477100A304F100894717E7FF1F23050A
:107F9000F7B88357810017E7FF1F2319F7920944A9
:107FA00009B3154793F64700B336D00093F787031C
:107FB000850685C32146638BC7066146638AC7066B
:107FC000130680026388C706130680036393C70005
:107FD000914717E6FF1F2309D6B497E6FF1FA38535
:107FE000F6B497E7FF1F2382E7B417E7FF1F0347A5
:107FF000278E9376070497E7FF1F83C7778D8DEE53
:108000001377770C93067008630CD7021377F70782
:108010008D466312D70CB307F040B7955B0093F71A
:10802000F70F938505D849A81947ADBF854755B7C0
:10803000894745B78D4771BF930670086311D70212
:108040001307300FB7150E006389E7021307900D71
:10805000B7B504006383E7021307700845BF9306B2
:10806000800C6311D702B307F040B775460013F7D1
:10807000F70F938785CDB3D5E70297E7FF1F23A3BB
:10808000B7AAD9BB9306900C631CD700B307F04086
:1080900093F5F70F91679387C766B3D5B702F1BF22
:1080A0009306A00C631DD700B307F040B7153D0041
:1080B00093F7F70F93850590B3D5F5027DBF93062F
:1080C000B00CE315D7F4B307F04093F5F70F9167C1
:1080D000938797D0D9B78946631BD700B307F04081
:1080E000B7750B0093F7F70F9385051BF1B785461E
:1080F000631AD700B307F040DD6593F7F70F938558
:1081000065E35DBFD28535FBB305F04093F5F50F10
:10811000B3D5BA029DB783C72400C18B99C78547E1
:1081200017E7FF1F230DF79EA5BE97E7FF1F2388C4
:10813000079EBDB6854717E7FF1FA308F79E8DB6BC
:108140003C0017E7FF1F2329F7AE094793070003F9
:108150002314F10097E6FF1F2380E69C2DBD639456
:108160000756A94763E5B742179701001307075C55
:108170008A05BA959C41BA97828717D4FF1F03449A
:108180001475894C6306940D63E68C06854763037A
:10819000F4089307F00F17E7FF1F0347E79763F60D
:1081A000E70017E7FF1F2309F79697ECFF1F83CC23
:1081B000AC969307000413F4FC0F63F497011304C7
:1081C000000497E7FF1F938727A703AD07002286C8
:1081D0002685EA85B38C8C40229D97700100E7804C
:1081E000A0EE97E7FF1F2389979397E7FF1F23A52B
:1081F000A7A545BC8D47630CF40A9947E31BF4F827
:10820000979701009387075917E7FF1F2326F7A2C7
:10821000A94751B717E7FF1F034767A597E7FF1F58
:10822000938787914946979501009385A55F6306DB
:108230008700979501009385E55A3E859770010068
:10824000E78080E817E7FF1F2328A79EC947A1B74B
:1082500097E6FF1F83C6A6A1054797E7FF1F9387F1
:10826000A78D6394E6023E85130670029795010080
:108270009385C55897700100E78000E517E7FF1F59
:10828000232CA79A9307700239B73E851306300452
:10829000979501009385C55097700100E780C0E273
:1082A00017E7FF1F232AA79893073004EDB597D54A
:1082B000FF1F83C5C56117950100130525609770E1
:1082C0000100E780C0EB054D97EDFF1F83CD2D9A90
:1082D00097D5FF1F83C5A55F179501001305055EA0
:1082E0006398AD0B97700100E78060E997D7FF1F97
:1082F00083C7E75DB5CBE36EF4E817940100130480
:10830000A456638CB7011794010013046456638666
:1083100097011794010013042457228597700100D8
:10832000E78000FF1375F50F93071500860717E721
:10833000FF1F2303F7808D4717D7FF1FA30EF77E7C
:1083400097D7FF1F9387477F0147BE861376F70FA6
:1083500089076365A60297E7FF1F23AFD78C97D7DE
:10836000FF1F83C7677D05BD979701009387C748A7
:1083700017E7FF1F2322F78C914731BD3306E40036
:1083800003460600A380070005072380C7007DBFC2
:1083900097700100E780A0DE97D7FF1F83C72753A0
:1083A000E1D7E368F4DE179401001304E448638C1A
:1083B000A701179401001304A4486386970117943A
:1083C000010013046449228597700100E78040F49E
:1083D0001375F50F93071500860717D7FF1F230D99
:1083E000F7748D4717D7FF1FA308F77497D7FF1FA0
:1083F000938787740147BE861376F70F8907E37C5E
:10840000A6F43306E40003460600A3800700050730
:108410002380C700D5B797D5FF1F83C5454B179558
:1084200001001305654A97700100E78040D597D792
:10843000FF1F83C7377093E7470017D7FF1FA30BB2
:10844000F76E83C7240017D7FF1FA303F76E89B801
:10845000179501001305854897700100E78000EA31
:1084600097D7FF1F9387C76C83C7070017D7FF1FD6
:10847000230EF74417D4FF1F0344046A33348000EB
:108480000DB0179501001305A54697700100E78010
:10849000E0E697D7FF1F83C7F76993E7070117D770
:1084A000FF1FA309F76883C7240017D7FF1F230105
:1084B000F7686FF0EFFE179501001305A54497705C
:1084C0000100E780A0E303C704007D8B51EFB7876D
:1084D000004003C767021377C70B13672700238386
:1084E000E70203C7A7021377C70B1367270023858B
:1084F000E70203C7E7021377C70B13672700238739
:10850000E70203C727031377C70B136727002389E5
:10851000E702854717D7FF1F230AF74617D7FF1F24
:108520002308F75217D7FF1F2306F75E17D7FF1F41
:108530002303F75E97D7FF1FA38A074497D7FF1F30
:10854000A388075097D7FF1FA386075C97D7FF1F05
:10855000A383075C97D7FF1FA38A075C97D7FF1FEA
:10856000A38707706FF0CFF389476312F70297D79D
:10857000FF1F83C7E7359146638CD70863E0F60495
:10858000638EE70C6369F70A05476380E70EFD57C2
:1085900017D7FF1FA302F75837074000B7E700E0DF
:1085A00023A0E71801000100B78600401306F0FC85
:1085B0002381C60223A0E7106FF00FE21307200803
:1085C0006382E7086362F70213071008E391E7FC90
:1085D000378700408347670293F7C70B93E727006D
:1085E0002303F7026FF0CFEB130730086389E7022C
:1085F00013074008E39DE7F83787004083472703C8
:1086000093F7C70B93E727002309F7026FF04FE9B1
:10861000378700408347270393F73707F5B7378736
:1086200000408347E70293F7C70B93E72700230730
:10863000F7026FF0EFE6378700408347E70293F7D2
:108640003707F5B7378700408347A70293F7C70B73
:1086500093E727002305F7026FF08FE43787004088
:108660008347A70293F73707F5B73787004083475B
:10867000670293F73707ADB71795010013058529F2
:1086800097700100E78080C797D7FF1F23800724DA
:10869000D5B3179501001305E52897700100E78011
:1086A000E0C597D7FF1F2393072297D7FF1F938714
:1086B000A74603C40700894763F38700094413747E
:1086C000F40F6FF00FDE13070002E392E7EC631B79
:1086D0000B0A638FF500930720026383F508179553
:1086E00001001305A52797700100E78040A945B553
:1086F000179501001305C52397700100E78000C09E
:108700000144179D0100130DED23A14CB387840094
:1087100083C507006A85050497700100E78020A6DD
:10872000E31694FF178501001305856B9770010010
:10873000E780C0BC17D4FF1F0344841901E897D712
:10874000FF1F23870716014B6FF0AFD58947E31052
:10875000F4E4854717D7FF1F230CF7146FF04FD4AD
:1087600017D6FF1F0346B61697D5FF1F83C52516DC
:10877000179501001305851D97700100E78020A063
:108780006FF00FD26380F50693071002E399F5F4BA
:1087900097D5FF1F83C5C513179501001305051D48
:1087A00097700100E780A09D97D7FF1F23A69748E9
:1087B00097D7FF1F93870737944383D7470017D76F
:1087C000FF1F0347873617D6FF1F2321D6101D44EE
:1087D00097D6FF1F239EF60E97D7FF1F238BE70E1A
:1087E0006FF02FCC97D5FF1F83C5850E179501001D
:1087F0001305451997700100E780609897D7FF1F10
:108800002388070A97D7FF1F2392070C6FF02FF9D1
:108810002547638FE7C89946378700406394D7029E
:1088200023008702B7E700E0B706400023A0D7186F
:1088300001000100130600FC2301C70223A0D7108A
:108840006FF08FB99306100A639FD7002300870249
:10885000B7E700E0B706400023A0D71801000100E9
:10886000130680FCD1BF9306A009E381D7FE9306CF
:10887000400AE38DD7FC93062002639DD700B7E73B
:1088800000E0B706400023A0D71801000100230034
:108890008702F9B78546E384D7FE93070008E30013
:1088A000FBFEB7E700E0B706400023A0D7180100A1
:1088B0000100130620FC23008702BDBF17D7FF1F4E
:1088C000034797256302F71E63E7E70295476300B6
:1088D000F7109947630AF704B78600402380060221
:1088E000B7E700E03707400023A0E71801000100C8
:1088F0001306A0FC75B99307F005630AF700930708
:1089000050096306F70093071002E317F7FCB7E777
:1089100000E03707400023A0E71801000100B786F8
:108920000040130620FC69B117DBFF1F034BCB1E71
:10893000930700045A8D63F46701130D000497D761
:10894000FF1F9387672F83AC07001374FD0F2286E8
:10895000E685268597600100E7800077B3078B40A6
:10896000669417D7FF1F2309F71A97D7FF1F23A570
:10897000872CB7870040630C0B022380A703B7E660
:1089800000E03706400023A0C6180100010003C71D
:108990002702134707042381E70203C7270213773F
:1089A000C70F2381E70223A0C6106FF0EFA2238038
:1089B000070237E700E0B70640002320D718010080
:1089C0000100130620FC2381C7026FF0AFB937877F
:1089D00000408347370097D6FF1F83C6761593F76D
:1089E0000708D58FA301F700B7064000B7E700E0FE
:1089F00023A0D718010001001306A0FC35BD97D7AE
:108A0000FF1F9387A724CA9783C7070093F7F70F21
:108A1000C1CF97D7FF1F83C78725D9E717D7FF1F78
:108A20000347970F930700026310F70883AD040014
:108A300017DDFF1F034DCDE997DCFF1F83CC5CE9F9
:108A400017DBFF1F034BEBE8E6876A87DA866E8643
:108A500097D5FF1F83C5C5E517950100130505F4DC
:108A600097600100E780A07197D7FF1F23ACB70B79
:108A700097D7FF1F238AA70B97D7FF1FA386970BB4
:108A800097D7FF1F2383670B97D7FF1FA38187E229
:108A9000B7E700E03707400023A0E7180100010016
:108AA000B78600406FF04FA2B7E700E037074000FD
:108AB00023A0E71801000100B786004015BD97D636
:108AC000FF1F83C6C61A0547639CE6042947238116
:108AD000E70209472383E7022385E70297D7FF1FB1
:108AE000A386070497D7FF1FA3830718B787004003
:108AF000A381070017D7FF1FA30C07020547238395
:108B0000E700B640264496440649F259625AD25AC2
:108B1000425BB25B225C925C025DF24D61618280DD
:108B200029472381E70209472383E7022385E702D8
:108B30002387E7022389E70255B717D7FF1FA3084A
:108B4000F7D66FE01FFF854717D7FF1F2300F7E415
:108B500017D7FF1F230EF7EE17D7FF1F230CF7FAC7
:108B600017D7FF1F2309F7FA6FE0BFFE854717D716
:108B7000FF1F230DF7E017D7FF1F230BF7EC17D7C5
:108B8000FF1F2309F7F817D7FF1F2306F7F817D79A
:108B9000FF1FA30D07DE17D7FF1FA30B07EA17D789
:108BA000FF1FA30907F697D7FF1FA38607F682804A
:108BB000411106C697000000E78080FBB7870040A0
:108BC00023800700130740FC2386E7001307C00437
:108BD000A386E70017D7FF1F130747CF2398E700A7
:108BE00017D7FF1F130787D2239AE70017D7FF1F56
:108BF000130707DE239CE70017D7FF1F130787E93A
:108C0000239EE70029472381E70209472383E702E0
:108C10002385E7022387E7022389E702A381070070
:108C2000930600F8A380D700930690022380D70014
:108C3000FD562383D7002381E7009306000537E71D
:108C400000E0230BD740B70640002320D71003C70E
:108C5000170013671700A380E700B24097D7FF1FE4
:108C6000239807EC41018280411106C6970000005D
:108C7000E78000F0B787004023800700130700FC5F
:108C80002386E7003147A386E70017D7FF1F1307A6
:108C9000E7C32398E70017D7FF1F130727C7239AB7
:108CA000E70017D7FF1F1307A7D2239CE700294728
:108CB0002381E70209472383E7022385E702A38193
:108CC0000700930600F8A380D70093069002238044
:108CD000D700FD562383D7002381E70093060005C4
:108CE00037E700E0230BD740B70640002320D7101A
:108CF00003C7170013671700A380E700B24097D798
:108D0000FF1F239707E241018280F16793870720C5
:108D100017D7FF1F2328F7E0854717D7FF1F231515
:108D2000F7E0A14717D7FF1F2301F7E097D7FF1FF1
:108D3000A38D07DE97D7FF1F238A07DE97D7FF1F74
:108D4000238807B697D7FF1FA38307B6814717D598
:108D5000FF1F130525B6FD5517D6FF1F130646B690
:108D60002947B306F5002380B600B306F60023803A
:108D700006008507E397E7FE97D7FF1FA38F07D865
:108D800097D7FF1FA38D07D897D7FF1F238807D832
:108D900097D7FF1F238307D897D7FF1F238207D8B2
:108DA00097D7FF1FA38C07D697D7FF1F238907D616
:108DB000814717D6FF1F130666E84147B306F60042
:108DC000238006008507E39BE7FE828017D7FF1FFD
:108DD0000347E7E985476316F700170300006700BC
:108DE000E3E8170300006700E3DC411122C406C674
:108DF00017D7FF1F0347A7E785472E8613F4F50F04
:108E0000AA856317F70417D5FF1F130565C0976080
:108E10000100E780602B97D7FF1F238B07C2B7871E
:108E2000004023848702B7E600E03706400023A015
:108E3000C6180100010003C7A7021377C70F2385D7
:108E4000E702B240224423A0C610014541018280BE
:108E500017D5FF1F130585AF97600100E780C02677
:108E600097D7FF1F238407B2B7870040238287026A
:108E7000B7E600E03706400023A0C6180100010055
:108E800003C767021377C70F2383E7025DBF411152
:108E900006C697000000E78080E7B2404101170353
:108EA00000006700E3F2411106C697F0FFFFE7807C
:108EB00080BF97D7FF1F83C777ADA1CB97D5FF1F83
:108EC00083C5E5AC89C917D5FF1F130565AC97E0CD
:108ED000FFFFE780205997D7FF1FA38907AA97D7DD
:108EE000FF1F238507C437E700E0B70640002320B3
:108EF000D71801000100378600408347660293F7C8
:108F0000370F2303F6022320D710B240410182809D
:108F100041C9D9C597D7FF1F83C787C1D1C30111E5
:108F200022CC4AC84EC656C25AC006CE26CA52C421
:108F30002E89AA890144930A0004371B0300637732
:108F40002403B3078940C207C183BE8463F4FA00D7
:108F500093040004C204C180130A1BD497D7FF1FD7
:108F600083C7C7A29DE37D1A631C0A00F2406244D6
:108F7000D2444249B249224A924A024B0561828058
:108F800097F0FFFFE78020B2D1BF33858900269498
:108F9000A685420497000000E78060E5418045B760
:108FA000828097D7FF1F9387E7DE18429C4383D6C2
:108FB00045000345070083C5C70003564600639676
:108FC000A50083D5E700638DD502011106CE238667
:108FD000A7002397D700B705CF00DC4B9385757D9D
:108FE00005077D162EC2230001003AC42316C100D6
:108FF0002317D10099C30A858297F24005618280C8
:109000008280411122C417A4FF1F1304643F5C4CEB
:1090100006C691CBC84B01C9B7E70400BC5782977D
:109020005C4C23AA0700B240224441018280DC4DFF
:10903000DC4B81CFB7E70400904503A3870591453A
:1090400017D5FF1F034545D502838280B7E704008B
:1090500003A30705A14517D5FF1F0345E5D30283E9
:109060006D713C083EC6B707E500232291103EC84B
:10907000AA843C083285232611103ECA232481107D
:10908000232021112E8997300000E780605A2A841E
:109090009795010093850594177501001305456E9A
:1090A00097600100E780A00DA285179501001305C8
:1090B000259F97600100E780800C2945976001009B
:1090C000E780C010B705CB009385757D68009710C9
:1090D0000000E780E05FA285680097300000E7802D
:1090E0008047014781467000CA8526859720000089
:1090F000E780608305CD2A84979501009385858D4F
:10910000177501001305C56797600100E780200708
:10911000A285179501001305659997600100E78006
:109120000006294597600100E780400A8320C110AE
:10913000032481108324411003290110516182808E
:1091400097D7FF1F938707C518429C43797122D494
:1091500006D60348070083C807012A8483D6450042
:10916000035546006396080183D82701638DD80212
:109170002388070105072399D7003708CC00DC4B6B
:109180001308787D3ACC1307F5FF42CA2308010083
:10919000231EE100231FD10099C7080832C62EC440
:1091A00082973246A245228597000000E78080EB37
:1091B000B250225445618280797131469775010021
:1091C0009385C54C280006D697600100E780C0EF64
:1091D00097A7FF1F83D7C722231B0100231C010071
:1091E000231D0100231E0100231F010099E3C16715
:1091F000FD17231AF10097A7FF1F83D7872091EB54
:1092000097D7FF1F938707B99C439C43DC4783D7BD
:10921000070097A6FF1F9386A61E231BF100D84EBA
:1092200083D74600231CF1005C4B91CB97A7FF1F0F
:1092300083C7771D81EB97000000E780C0DCB25048
:1092400045618280FD1717A6FF1FA30EF61A03566D
:10925000070183C706014C472800230FF100973010
:109260000000E780602C97D7FF1F9387A7B29C432D
:109270000147978601009386667F884330004C083B
:1092800097100000E780206A5DD975B799C9B7E7E4
:10929000040003A30705A14517D5FF1F0345C5AF6C
:1092A000028382805C4EDC4BB9CFB1CD411122C428
:1092B000177501001305C54C2E8497850100938511
:1092C000A57606C697600100E78060EBA28517854A
:1092D00001001305A57797600100E78040EA294562
:1092E00097600100E78080EEB7E704002244B240B7
:1092F00003A3870517D5FF1F034505AA13064006DC
:109300009145410102838280411122C417A4FF1FAD
:109310001304C40C1C4C06C689C7DC4399C34C48D3
:109320008297584CB7E70400BC57484B82975C4C77
:10933000B240224423AA07004101828017A7FF1FE1
:109340001307C70B834707009306F00B850793F7B6
:10935000F70F63E9F60097A6FF1F2381F60A03457E
:1093600007008280930700F8FDB78357450099E313
:109370007D558280011122CC17A4FF1F13044408DD
:109380005C4C4AC84EC6DC4B52C406CE26CA56C2F6
:10939000B2892E8A2A898DC7B7E70400FC5F8297BD
:1093A00097D7FF1F9387079D9C431307301FB30771
:1093B000F54071556375F70697000000E780A0C47B
:1093C0009307D00D7D5563EC3705B7E40400938710
:1093D0008900B858832AC401139507014181029777
:1093E00023AAAA00484C584921E797850100938594
:1093F000A561177501001305A53897600100E78086
:1094000000D8178501001305256D97600100E780DE
:1094100000D7294597600100E78040DB5D55F240A9
:109420006244D2444249B249224A924A056182804A
:1094300013874900B705CF002319E5009385757D93
:10944000310597100000E780A028484C834569004B
:10945000310597300000E7800010484C4E86D285D9
:10946000310597300000E780200C7146CA8517A5AA
:10947000FF1F1305E5F897600100E780E0C4FC5C7E
:1094800082970326C90097D7FF1F23A5A78E11CA6D
:10949000BC4C854517D5FF1F0345059082970145B4
:1094A000BDBF97000000E78060D1D5BF411106C65F
:1094B00022C426C217D4FF1F1304048E9700000095
:1094C000E78060B4B7E40400FC4C03450400854524
:1094D000829703450400224403A3C405B24092448A
:1094E000A14541010283411126C297D4FF1F9384F5
:1094F000648A9C4006C622C44AC0D5C3DC43C5C3A7
:109500005CC12300B5002A84978501009385054B33
:10951000177501001305C52697600100E78020C676
:10952000294597600100E78060CA9C4023A407009A
:1095300023A2070097A7FF1F938747EADC4FDC4B66
:1095400091C7295597000000E78040DC97A7FF1FCF
:10955000938707EBDC4FDC4B89C797000000E7805F
:1095600020F537E904008327C905894517D5FF1F72
:109570000345858282978327C905914517D5FF1F2B
:109580000345858182979C4003A34701630903003B
:1095900022852244B2409244024941010283B240F2
:1095A000224492440249410182800111328506CE53
:1095B00022CC26CA2E8497300000E7806007AA8458
:1095C000978501009385C542177501001305451B5A
:1095D00097600100E780A0BA030784000356640087
:1095E00083554400A686178501001305A54897609A
:1095F0000100E780C0B8294597600100E78000BD01
:1096000097A7FF1F83C7E7DD639D9700014597007C
:109610000000E780A0CF81450A8597000000E78021
:10962000C0ECF2406244D244056182806D71232413
:109630008110232611102322911093F745002E84C8
:10964000638707143C083EC0B707E5003EC23C08EC
:109650003EC4231701002318010023190100231A17
:109660000100231B010097A7FF1F83D727D799E38A
:10967000C167FD172316F10097A7FF1F83D727D6D1
:1096800091EB97C7FF1F9387E7709C439C43DC4790
:1096900083D7070017A7FF1F130747D42317F1002D
:1096A000544F835747002318F100DC4AA1E7978500
:1096B000010093852538177501001305650C976027
:1096C0000100E780C0AB178501001305654797606F
:1096D0000100E780C0AA294597600100E78000AF3C
:1096E000134544008320C1100324811083244110BA
:1096F0005161828097A7FF1F83C7B7CE2555D9C375
:10970000FD1717A6FF1FA30EF6CC03D6060183474D
:109710000701CC460A85230BF10097300000E78053
:10972000A0E097C7FF1F9387E7669C4317A7FF1F1B
:109730001307C7CA978601009386C63088430A86F6
:109740006C0097100000E780001EAA8451D997850D
:1097500001009385252E177501001305650297609A
:109760000100E780C0A1A685178501001305053E0D
:1097700097600100E780A0A0294597600100E7807D
:10978000E0A4268597000000E78040B891BF93F7DA
:1097900025009DC7B7E70400BC474146814528081E
:1097A0008297255597000000E78040B6280893056A
:1097B000F00F97000000E78040D3134524001DB749
:1097C00093F7150081CB97000000E780209F134599
:1097D000140009BF93F78500014589D717A7FF1F1C
:1097E000034777C297A7FF1F938787C10DC3D84F41
:1097F000584B11CF37E70400384F9047854517C5C0
:10980000FF1F03456559029713458400E1BD97F09A
:10981000FFFFE780407FCDBF5C4D411106C688C386
:1098200017C7FF1F2328F756B7E7040083A70708C9
:10983000170500001305C5DF8297B24097C7FF1FC9
:10984000238CA75401454101828001113335A000CA
:10985000A307A100B7E7040083A7471706CE1306A6
:10986000F1008545130550308297F24005618280F2
:109870008280411122C406C697B7FF1F83C7579D38
:10988000054489EF97C7FF1F83C7C7DC014499E7E9
:1098900017B4FF1F0344C49B134414002285970090
:1098A0000000E780C0FA178501001305E53009E4E0
:1098B00017850100130545312244B2404101176369
:1098C00001006700C38B797122D4A30F010037E434
:1098D00004008327841726D24AD006D6AA842E896C
:1098E000130550309305F10132C682973246834703
:1098F000F10193150601C18185CB01452EC6970064
:109900000000E780C0F483274417B2454A862685C5
:109910008297054597000000E78060F3B25022541B
:109920009254025945618280832744174A862685CE
:109930008297EDB741119397050122C406C626C24E
:10994000C1872E8463D40702B7E40400FC5417A532
:10995000FF1F0345E5AD829719C1BC54829721656D
:10996000218DB240224492444101828093F7150038
:109970008DC7B7E7040083A7471A17A6FF1F130672
:1099800026AA97C5FF1F9385E54117A5FF1F03452D
:1099900025AA829713451400E9B793F725000145DE
:1099A000E9D397C7FF1F83C7674185E7B7E704007F
:1099B00003A8871A1307401F97A7FF1F83C747A74E
:1099C000814613064006994517C5FF1F0355853E7E
:1099D00002981345240071B797C7FF1F83D7873DAF
:1099E0006398A70217C7FF1F2317B73C17C7FF1FAE
:1099F0002314C73C17C7FF1F2311D73C2E8617859A
:109A000001001305E522BE85175301006700237787
:109A10001785010013054523176301006700038EB6
:109A20000357450097C7FF1F83D7C7386318F7024E
:109A3000C167F91717C7FF1F232EF73697C7FF1FF8
:109A400023AC073697C7FF1F2384073697C7FF1F2E
:109A500023860736170300006700E3E1178501003E
:109A60001305851E17630100670043897D1595471F
:109A700063E2A71C17870100130787120A053A95AE
:109A80001C41011122CC06CEBA972E8482871785FD
:109A900001001305E51B97600100E7802086A1A265
:109AA00003C7250099476311F7022E859700000030
:109AB000E78040F783456400178501001305451AC8
:109AC00097500100E780A06B97A7FF1F23820778BC
:109AD000178501001305851A7DBF03C7250095472B
:109AE0006319F702C16717C7FF1F0357A72CF917A0
:109AF00003D5A5006309F702B7E7040083A7C717DA
:109B00008297178501001305651897500100E780BB
:109B1000E07E854717A7FF1F230CF772178501000A
:109B2000130545198DBF97C7FF1F2395A72883D716
:109B3000E50097C6FF1F2390F62883D7050197C637
:109B4000FF1F239BF62683D7250197C6FF1F239669
:109B5000F62697C7FF1F238D0724631BE502B7E78F
:109B60000400BC4F096613060690894517A5FF1F20
:109B70000345058C82970356E4008355A40017859E
:109B800001001305E51197500100E780405F51B7D0
:109B90009307700F2316F100B7E7040083A7870D22
:109BA00017A6FF1F0346C6886C0082974DF98547AC
:109BB00017C7FF1F230EF71E5DB71785010013059A
:109BC0002510D1BD83C5250091476392F502178505
:109BD00001001305651097500100E780207297007F
:109BE0000000E78040C9F2406244056182809947E5
:109BF0006392F502228597000000E780A0E283458A
:109C00006400178501001305A50597500100E78042
:109C10000057D1BF9547639AF50083471400E1F3DD
:109C2000178501001305850DBDB5178501001305C6
:109C3000650DE1BF82803757315F97A7FF1F93877C
:109C40006780130777D598C39356C500178701001F
:109C50001307C7FABA9683C5060093568500BD8AD6
:109C6000BA9603C6060093564500BD8A3D89BA964A
:109C70002A9783C60600034707002384070023832F
:109C8000D700A383E7002382B700A382C70097977A
:109C9000FF1F9387277C2383B700A383C7002384F8
:109CA000D700A384E7008280411106C69700000018
:109CB000E780A0F8B7E7040083A787141796FF1F73
:109CC00013064678D54501458297B2404D46979593
:109CD000FF1F93852578130570304101170300009D
:109CE0006700A3BE61712324811A37E4040083272F
:109CF00004082326111A2322911A2320211B232E24
:109D0000311917050000130525C382971799FF1F06
:109D100013090972994785442300A900231CF10007
:109D200097850100938585EC930740061775010020
:109D3000130505A5231CF1082308910097C9FF1FEF
:109D40009389A9A197500100E780604383D509005A
:109D500017850100130585E897500100E780204230
:109D6000294597500100E780604603D50900970018
:109D70000000E78080EC8327441710088545130511
:109D800050308297832744171796FF1F1306866C5F
:109D9000CD45130570308297832744171796FF1F10
:109DA00013064669B545130560308297832744172B
:109DB00030088945130510318297832744173009ED
:109DC0008945130520318297832744159305000A9E
:109DD0000D458297832744159305000A1145829704
:109DE000A30591002306910002CD23080100230C56
:109DF000010083278416300991451305704082972E
:109E0000832784161306B100854513050040829709
:109E10008327841670008545130510408297832799
:109E200084163008854513052040829783278416C1
:109E300010088545130550408297832704157D55EA
:109E40008297832744137D5582977D5597A0FFFF06
:109E5000E780A0838327440C82979790FFFFE780D9
:109E6000005F832784141796FF1F1306A65DD54550
:109E70000145829789471306700F814528092306FB
:109E8000F1009780FFFFE78080288D4713060008C8
:109E900081452808230CF1089780FFFFE7802027E1
:109EA0009147230CF100976701009387E77E984361
:109EB00083C747003AC8230AF10097D0FFFFE78025
:109EC000009670008545054597A0FFFFE780008359
:109ED00030099305700F094597A0FFFFE7800082C6
:109EE0003008930500080D4597A0FFFFE78000812B
:109EF00010089545114597A0FFFFE7802080C167B6
:109F000017C7FF1F130707EBF9171CC3232207000E
:109F10001795FF1F130585519790FFFFE780E07CA1
:109F20008327C41D17C5FF1F130545E782973C48CB
:109F300003450900854582978320C11A0324811AAD
:109F40008324411A0329011A8329C1195D61828082
:109F5000C16717C8FF1F0358E8E5F9176301F80840
:109F60003DCDB5CD011126CAB7E4040083A7841204
:109F700022CC2E862315B10006CE2A8401478146C5
:109F8000ED45428582972AC611ED1785010013051C
:109F900025C897500100E7806036F2406244D24401
:109FA00005618280FC440356A100A28582972C00A3
:109FB00017C5FF1F035505E09790FFFFE780A07FBF
:109FC00069DD178501001305E5C597500100E7809D
:109FD000E03283A7C412ED45280082977DBF8280BE
:109FE0000DC585471797FF1FA30BF7449797FF1FD2
:109FF0002388074435469795FF1F9385A54313058E
:10A000006030170300006700438C9797FF1FA388F9
:10A010000742E9BF97C7FF1F83C747DAA9EFC167A8
:10A0200017C7FF1F035707D9F9176306F704411134
:10A03000854722C417C7FF1F2302F7D837E404005F
:10A040007C4C06C689451795FF1F0345653E8297E0
:10A050000323841A2244B2409797FF1F83C7473DCA
:10A0600017C5FF1F035505D51307401F814631460D
:10A0700099454101028382806D712324811023263A
:10A08000111023229110328401CD8947630AF50211
:10A090008320C110032481108324411051618280E8
:10A0A000178501001305C5C6AE8497500100E780EF
:10A0B000E024A285268597B0FFFFE78020EEC9BF88
:10A0C000B7E70400FC4728008297178501001305B5
:10A0D000E5C497500100E78060228347810039C4BE
:10A0E0001307000B6380E7021387A7051377F70FA9
:10A0F0008D4663EDE602A285280097C0FFFFE7804A
:10A1000060F179B78547E3F587F8834591001775C6
:10A1100001001305659BB335B00097A7FF1F23858A
:10A12000B7F897500100E78080059DB7034791007D
:10A13000A207B966D98F1387E6556384E70C636D70
:10A14000F7042D671307B755638FE708636AF700B5
:10A1500029671307A755638FE708A2852800A1BFC9
:10A1600031671307C7556388E70635671307D75567
:10A17000E395E7FE8947E3FD87F097000000E7805D
:10A18000A0E99305E4FFC205C1811305A1009790E2
:10A19000FFFFE780E004EDBD3D671306F7556389D7
:10A1A000C706636DF6009386E665E398D7FAA28545
:10A1B000280097C0FFFFE780602BD9BD9306F766A4
:10A1C000638DD7041307F777E399E7F897C0FFFF8C
:10A1D000E780805675BD0146A285280097C0FFFF25
:10A1E000E780E00E75B5A285280097C0FFFFE780E5
:10A1F000201C79BDA285280097C0FFFFE780001DC5
:10A2000041BDA285280097C0FFFFE780201D49B50A
:10A2100097C0FFFFE780A02EA5BD97C0FFFFE78096
:10A220004034BDB5C16717C5FF1F0355A5B8F91761
:10A230006307F500B7E7040003A3C7170283828012
:10A2400017F3FFFF670023631783FFFFE70283E72E
:10A250002A8408452E89B28919C900C197150000C2
:10A260009385A586610597300100E78060048144ED
:10A270007D5A97100000E780E03963C7A404814449
:10A2800097100000E780003A63C8A40497C7FF1F37
:10A29000938707B39C43DC47B307F94091872302B8
:10A2A000F400638309048327C900B307F44095874A
:10A2B000A302F4001C4C89C79C4799C3228582974E
:10A2C0001783FFFF670043E35C4413971400850482
:10A2D000BA972390470171BF1C4813971400850457
:10A2E000BA972390070069BF832789000547B30702
:10A2F000F4409587A302F40083570400638EE702BD
:10A300008DC309476384E7040D47E395E7FA978710
:10A310000100938767F31CCC978701009387C7F3ED
:10A3200011A8978701009387A7B91CCC97870100D4
:10A33000938707BA5CC8BDBF97870100938747A57D
:10A340001CCC978701009387A7A5EDB797870100DD
:10A35000938747F41CCC978701009387A7F4D9BF54
:10A3600095E51783FFFFE70283D70046184483472C
:10A37000940075839D8B6317F70097100000E780AA
:10A3800060B448C41783FFFF6700A3D78280178398
:10A39000FFFFE70223D313893500C164420941114D
:10A3A000AA890144F11413590901054A2EC69710D0
:10A3B0000000E7802026B2456348A4000145410122
:10A3C0001783FFFF670043D383A709001317140007
:10A3D000BA9783D707006388B700639497006374C4
:10A3E0002A010504E1B70545D9BF1783FFFFE7023E
:10A3F00083CCAA892E89328BB6843A8ABE8A97A0EA
:10A400000000E78000FE71C9268597200000E780E4
:10A41000C00C8D4763E7A7007D551783FFFF6700DA
:10A4200003CD83DB440097100000E780A0242A843A
:10A4300097100000E78040259307740031443305EE
:10A44000850263CDA70297100000E780A022971035
:10A450000000E78020222A8497100000E780C022B5
:10A460009307740031443305850263C3A704971032
:10A470000000E78020209307450029A897100000DE
:10A48000E7808020330585021307F0179307C01774
:10A49000E35FA7FA2D55E3C277F963040B02D68672
:10A4A0005286A6854A8597200100E78000BDB5B792
:10A4B00097100000E780401D330585029307C5FF14
:10A4C000D1BF832749001385C90083D52700970092
:10A4D0000000E78000EC61F581B769553DBF97C783
:10A4E000FF1F2391A78E97C7FF1F9387678D904308
:10A4F00081470C463307F500420741836393B70059
:10A5000082805446139847008507C2962390E60040
:10A51000D5B797C7FF1F9387A78A9C4303C58700BA
:10A52000828017C5FF1F0355E58982801783FFFFCF
:10A53000E702E3BAC1671387D7FF630BE502636ADB
:10A54000A700F1176300F50201451783FFFF6700BD
:10A5500043BB1387E7FF6302E502FD171D8D13352B
:10A560001500E5B797500000E780A0297D15C5BF0D
:10A5700097500000E78020FED5BF97500000E7808D
:10A5800040FCEDB71783FFFFE70263B54111AA84D2
:10A5900001442EC697100000E780C008B24563480A
:10A5A000A400014541011783FFFF670083B59C4864
:10A5B000131514003E9583570500E385B7FE050487
:10A5C000C9BF03485500814693F7F60F63E50701BD
:10A5D00081473E858280584593975600BA9703D7A6
:10A5E00027006316B70003D70700E304C7FE8506FC
:10A5F000E1BF8346450001479377F70F63E4D70037
:10A60000814711A81C45131657000507B29703D6BA
:10A610000700E313B6FE3E8582801783FFFFE70243
:10A6200063AA93170501C18797BAFF1F938A4A79D6
:10A63000635BF00883A70A00C0479C4703570400E8
:10A64000198D420541816368F50001442285178315
:10A65000FFFF670063AA12052A94CDBFDC4713945D
:10A660004900014A3E94834744006341FA02014A8B
:10A67000834754006349FA028509C20993D9090145
:10A6800083A70A009847E3EBE9FCC1B71C44131900
:10A690005A00A6853E994A8597000000E780C0EEE3
:10A6A00005E1050AC9B75C4413195A00A6853E990D
:10A6B0004A8597000000E78020ED19E1050A4DBFAB
:10A6C000E30C09FA61B7AA8481495DBF1783FFFFD4
:10A6D000E702E3A01C452A8481E79307C5001CC557
:10A6E0001C44231204001CC09307F00F63EDB70055
:10A6F00093F5F50F228597200000E780C0E51783CA
:10A70000FFFF670003A093940501C167C18063F94F
:10A71000F500A685228597200000E780E0E8C5B710
:10A72000C18193F5F50F228597200000E780A0E214
:10A73000A685228597200000E780E0E3C9B797B798
:10A74000FF1F9387E767884382801C4599C797B7A7
:10A75000FF1F23A7A766014582807D55828097B79A
:10A76000FF1F9387E7659843834745004847920753
:10A770003E9582801783FFFFE70263966171004573
:10A780001C183EC6B70780013EC81C183ECA835736
:10A79000440002CE02D002CC231EF1008347840085
:10A7A0002A8902D22301F1023C083ED402D6970046
:10A7B0000000E78000FB835705002316F102975045
:10A7C0000000E78040C72307A1025C4003556400F6
:10A7D000F18313F717008347F10252055181F99B6A
:10A7E000D98FA307F10297100100E780607839CD77
:10A7F000AA840355050097A00000E78060BF83D7B7
:10A8000004002AD26800231CF10083D72400231DF2
:10A81000F1001C4803D647008C4397200000E780D6
:10A82000A0D08347B400CA86177601001306C64F2E
:10A830008117A305F4006C00481097200100E78001
:10A84000C0835D611783FFFF6700A38B2155D5BFD0
:10A850001C45B1CF03C5A700894613576500630B9C
:10A86000D7028D46630ED70285466300D7021307D1
:10A8700040063305E50203C7B700418B15CB83C7FC
:10A88000B700BD8B3355F54082801375F503130770
:10A89000803EC5B709671375F50313070771D1BF6C
:10A8A000372709001375F5031307077CD9B701454E
:10A8B00082801783FFFFE702838203A98500630C70
:10A8C00009048347B900AE8493F7070E85C3034597
:10A8D0009900930520030D810505B305B502884451
:10A8E000610597300100E780C0AC35A02E85970048
:10A8F0000000E78020F62A8419CD97000000E78049
:10A90000605C8325C900B307B54063FA87002E94C5
:10A91000B305A440E9F51773FFFF6700837E854503
:10A920007DBF1773FFFFE702837B2A8403D50500F1
:10A93000011132C636C43AC22EC002CA02CC02CEBF
:10A9400097A00000E780C0AA82452ACA22852ECCA3
:10A9500097000000E780E0E003570500231EE100B8
:10A9600097500000E78020ADA24632469247230F61
:10A97000A10036874C08B286228501469700000068
:10A98000E780E0A605611773FFFF67008377177301
:10A99000FFFFE702C37461711C183EC6B707800150
:10A9A0003EC81C183ECA3C0800453ED4AA8402CCCE
:10A9B00002CE02D002D202D697000000E78060DA11
:10A9C0008357050035592316F10297500000E780A0
:10A9D00080A62307A10209C48357440081EB2159B3
:10A9E0004A855D611773FFFF6700A371035564001B
:10A9F0005205518197100100E78080572A8965D15F
:10AA00008347B40093F7070E99C713058401973065
:10AA10000100E780409C83574400231EF1008347D8
:10AA200084002301F1025C4003550900D98313F728
:10AA3000070883471102231CA10093F7F707D98F5A
:10AA4000A300F10283572900231DF1005C40F1832C
:10AA500013F717008347F102F99BD98FA307F1027F
:10AA600097A00000E780C0982AD235D98347940088
:10AA70006800139757008347B400FD8BD98FA30557
:10AA8000F4001C4803D647008C4397200000E78061
:10AA9000A0A9A687177701001307072974000546A8
:10AAA0004C10268597000000E78060942A890DD914
:10AAB0008347B400A685FD8BA305F4009700000032
:10AAC000E78060DF31BF1773FFFFE7024361832434
:10AAD00085FE2A844111268597000000E78080D7F3
:10AAE000834734FF93F7070E8DCB2AC62685970040
:10AAF0000000E78060C809CD834734FFB245FD8B75
:10AB0000A309F4FE91C5228597300100E780608A91
:10AB100041011773FFFF6700C35E7DD98327C4FF20
:10AB20002685829775F5834734FF93F7070E91C703
:10AB3000228597300100E780008A032584FE970074
:10AB40000000E78000E5E9B71773FFFFE70223562F
:10AB50009C4141112A8903C7070089472E849356D7
:10AB600067006380F6040D466388C6049307F00708
:10AB70006304F7022E8597200000E78060ABAA846B
:10AB80008149C16B130C490097B7FF1F9387472377
:10AB90009C43984763E4E90441011773FFFF670092
:10ABA000C35403D745008547E3F8E7FE2E85972079
:10ABB0000000E78040ADE1B703D74500E3FEE7FCC6
:10ABC0002E8597200000E780A0A6AA8422859720E2
:10ABD0000000E78000A8C204C98C5DB7DC470355BC
:10ABE000A900139A49003E9A93170501C187635D36
:10ABF000F00083570A006397A70263E77403832773
:10AC0000CA00034D5A002DA0A1672167A98F130721
:10AC1000F7EFE374F7FE6397090097000000E78001
:10AC2000209161FD85098DB783278A00034D4A0075
:10AC3000835DA90003576900216A138BC7003AC6D8
:10AC4000814A33CA4D01631E5D0197B7FF1F938789
:10AC5000A7179C43E1DBA286628681452685829701
:10AC6000D1B7A1679387F7EF930C4BFF63F24703CC
:10AC7000B2455A8597F0FFFFE780A0710DC1032709
:10AC80008B00104709CE10436382C4023107D5BF41
:10AC9000EE85668597000000E780008F71F9938646
:10ACA0001A0093FAF60F130B0B0271BF8356440080
:10ACB0005C43E3E9F6F622853AC697200000E78078
:10ACC0002081A1679387D7042A8A035D4400324715
:10ACD00063E897008347D90093E707F8A306F900D4
:10ACE0001C4766852286E2858297C1670844FD1766
:10ACF000337AFA00529508C02312A40125B797B7FA
:10AD0000FF1F9387E70B9843814715C3144781477B
:10AD100063FFD500939745004C47BE9519C903C7FB
:10AD2000550081476375E600DC451606B2973E85FF
:10AD3000828003C745008147E37BE6FE16069C45FB
:10AD4000F5B71773FFFFE702E337AA892E8A81441C
:10AD500097BAFF1F938ACA0683A70A00984763E63B
:10AD6000E4001773FFFF67002339DC4713944400A6
:10AD700001493E9413BB140083474400634BF90020
:10AD8000014913BB140083475400634FF900850445
:10AD9000E1B70844931759005287DA860146A28525
:10ADA0003E9582990509C9BF4844931759005287B7
:10ADB000DA860546A2853E9582990509E9B717739B
:10ADC000FFFFE702C331814517F5FFFF1305054873
:10ADD00097B7FF1F239807FE97000000E780A0F6B3
:10ADE0001773FFFF6700E33197B7FF1F938747FD96
:10ADF0009C4395C31773FFFFE702632E814517F548
:10AE0000FFFF1305A54497000000E780C0F3177308
:10AE1000FFFF6700032F82801773FFFFE702832A7B
:10AE200037E404008327841241112315E100AE8921
:10AE30003289368A3A8681460147ED45AA8482974F
:10AE40002AC621C90356A100D28597400100E78098
:10AE5000A0278327C413CE8526858297058905C937
:10AE60008327440D2314210101462C002685829757
:10AE70002A8401C9B7E7040083A7C712ED4528005B
:10AE80008297228541011773FFFF6700E32649443B
:10AE9000D5B76554FDB75C41FD175CC1828017735F
:10AEA000FFFFE702C323B7E70400FC5F82979547E3
:10AEB0003305F50281450D811773FFFF6700632499
:10AEC0001773FFFFE702A321B7E70400FC5F829737
:10AED00095473305F5020D811773FFFF6700632265
:10AEE0001773FFFFE702A31FB7E7040083A7870BD1
:10AEF0000355050082971773FFFF670083201773C0
:10AF0000FFFFE702C31D035505003287AE86178693
:10AF1000FF1F0356465A97B5FF1F938525EB9700F1
:10AF20000000E780A0EF1773FFFF6700831D177312
:10AF3000FFFFE702C31AB7E7040083A7C71782978A
:10AF40001773FFFF6700E31B1773FFFFE702231967
:10AF5000B7E7040083A7871397B5FF1F938505E71D
:10AF6000829701451773FFFF6700A3191773FFFF4F
:10AF7000E702E316B7E7040083A7C71F81451785DB
:10AF8000FF1F0355454F82971773FFFF6700631735
:10AF90001773FFFFE702A314B7E7040083A7871323
:10AFA00097B5FF1F938585E3829701451773FFFFD0
:10AFB000670023151773FFFFE7026312B7E704006A
:10AFC00083A7C71F81451785FF1F0355C55082976B
:10AFD0001773FFFF6700E3121773FFFFE7022310E9
:10AFE0002E8597800000E780C0B297800000E78040
:10AFF000C0EF1773FFFF6700C3101773FFFFE7026F
:10B00000030E97800000E780C0F91773FFFF670009
:10B01000430F5C49E1175CC95CC583572501A10753
:10B020002319F50083570501A1072318F500828035
:10B03000F1473305F50297B7FF1F938727DC9C4341
:10B040003E9582808D476315F60803D746008547F5
:10B0500063F0E7081773FFFFE7026308368536845D
:10B060002E8997100000E780A05C29C9835744000F
:10B0700093140501C18063E39704228597100000B3
:10B08000E780005BFD14231294009307A002630085
:10B09000F5029307B0026307F50293079002631F5E
:10B0A000F500228597000100E780A08801A80146ED
:10B0B000CA85228597A00000E78040B31773FFFF81
:10B0C00067002304228597100000E7806007FDB722
:10B0D000828097B6FF1F9386A6D29C42014599CFE6
:10B0E0009843D44217B6FF1F232CE6D06396D700AF
:10B0F00097B6FF1F23A8E6D01385C7FE828017737B
:10B10000FFFFE702C3FD97000000E780A04B7144FA
:10B1100033058502914597900000E78000EC11E52A
:10B1200065551773FFFF6700C3FD97B7FF1F23A582
:10B13000A7CC97000000E780E048330585029145E1
:10B1400097900000E78060E961DD97B7FF1F23A7B4
:10B15000A7CA97000000E780E04697B7FF1F239734
:10B16000A7C897000000E780E04597B7FF1F23902E
:10B17000A7C897770100938767C017B7FF1F232BD6
:10B18000F7C697070000938707E917B7FF1F23212A
:10B19000F7C6014579B71773FFFFE70243F4AA85A5
:10B1A00017B5FF1F130585C497100000E780605F87
:10B1B0001773FFFF6700E3F41773FFFFE70223F243
:10B1C00097000000E78060FD97100000E780E05ED8
:10B1D00097B7FF1F9387C7C29C4391CF1387C7FEC2
:10B1E00019CB83D5C7FF17B5FF1F1305E5C19720FE
:10B1F0000100E780001C1773FFFF670083F01773DF
:10B20000FFFFE702C3ED97000000E780C0EC09CD27
:10B21000834785002A8493F7070499EB0355E500DB
:10B2200097000000E78080F91773FFFF670063ED68
:10B230008347C5009304450117B9FF1F130949BC93
:10B2400085E3832709005CC997B7FF1F23AA97BA34
:10B2500083274900F1FB97B7FF1F23A597BAE9B7EA
:10B26000FD172306F500610597800000E780A0D94F
:10B270008307840063CB07048347840093E707F8C0
:10B280002304F400B7E704009C5F82974205A947B6
:10B2900041813375F5028347840093F707FCC98F1A
:10B2A0002304F4008347D4003E951C402318A400D7
:10B2B00089CF984319CB8347C40050408145850707
:10B2C0003305F502420541810297832709005CC8D6
:10B2D00097B7FF1F23A697B28327490089E797B73F
:10B2E000FF1F23A197B28347C4009DDF835504014C
:10B2F00017B5FF1F130545B197200100E780600BCC
:10B3000025B71773FFFFE70283DD97B7FF1F93870A
:10B31000E7D49C4701448583858B85E3AE84B28561
:10B320003A8697100000E780204F2A8419C59710AD
:10B330000000E7806045829408CC22851773FFFFE8
:10B34000670023DC1773FFFFE702C3D741112E8983
:10B3500032C6AA8997000000E780C0313247130641
:10B360000502CA86970500009385C5CC17B5FF1F57
:10B370001305C5A797000000E780E0F82A8425C9D7
:10B380009304C50097000000E780E0411946AA85B4
:10B39000268597100000E78020198545268597109F
:10B3A0000000E7800015177501001305E59A4E951A
:10B3B00083450500268597100000E780C0195C488A
:10B3C00031468145A1075CC85CC483572401E1175D
:10B3D0002319F40083570401E1172318F4001C4CCF
:10B3E0003E859770FFFFE78080D2A3042501228568
:10B3F00041011773FFFF670023D01773FFFFE702B8
:10B4000003CE4111AA842EC632C497100000E780F3
:10B41000003A004DB2452246834784000CC050C01C
:10B4200093F7F70393E707042304F40023180400B9
:10B43000268597100000E780203583479400A946B1
:10B440002317A40013D7370005073307D7029D8BB6
:10B4500085072306F400A306E40083C70401D84847
:10B460008507230FF7FE17B7FF1F13076799584388
:10B47000232A04009307440129E317B7FF1F23235E
:10B48000F79817B7FF1F232DF79617B4FF1F130464
:10B49000A497228597200100E780E0E31C44858B78
:10B4A0005D8D19E58145228597200100E78060F0D8
:10B4B00041011773FFFF6700C3C41CC317B7FF1F09
:10B4C0002322F794D9B71773FFFFE70243C197050B
:10B4D0000000938565B7014597000000E78000B044
:10B4E00001451773FFFF6700C3C11773FFFFE70232
:10B4F00003BF97000000E78080B01773FFFF67006D
:10B5000043C08347C500A5E31773FFFFE70223BDD0
:10B510002A840355E50097000000E78000C821C198
:10B520008347840093F7F7FB2304F4001C4091C782
:10B53000DC4381C74C400145829797000000E780BB
:10B5400080B917B5FF1F1305258C97200100E780F0
:10B5500080E80355E40097000000E78020C61773D9
:10B56000FFFF670003BA82801773FFFFE70223B76C
:10B5700097B7FF1F9387C78897050000938565C815
:10B5800017B5FF1F1305458823A0070023A2070056
:10B5900097200100E780C0D11773FFFF670063B6F3
:10B5A0001C4D91CFDC4381CF1773FFFFE70223B31C
:10B5B0008345070082971773FFFF670083B482807B
:10B5C00097B7FF1F938787869C4303C50700828038
:10B5D00097B7FF1F938787859C4303C51700828019
:10B5E00097B7FF1F938787849C4303C527008280FA
:10B5F00097B7FF1F938787839C4303C547008280CB
:10B6000097B7FF1F938787829C4303C537008280CB
:10B6100097B7FF1F938787819C4303C5570082809C
:10B6200097B7FF1F938787809C4303C5670082807D
:10B6300097A7FF1F9387877F9C4303C5770082806E
:10B6400097A7FF1F9387877E9C4303C5870082804F
:10B6500097A7FF1F9387877D9C4303C59700828030
:10B6600097A7FF1F9387877C9C4303C5A700828011
:10B6700097A7FF1F9387877B9C4303C5B70011E102
:10B680001D45828097A7FF1F9387477A9C4303C578
:10B69000C700828097A7FF1F938747799C4303C504
:10B6A000D700828097A7FF1F938747789C4303C5E5
:10B6B000E700828097A7FF1F938747779C4303D5B6
:10B6C0000701828097A7FF1F938747769C4303C596
:10B6D0002701828097A7FF1F938747759C4303D557
:10B6E0004701828097A7FF1F938747749C4303D528
:10B6F0006701828097A7FF1F938747739C4303D5F9
:10B700008701828097A7FF1F938747729C4303C5D9
:10B71000A701828097A7FF1F938747719C4303C5AA
:10B72000B701828097A7FF1F938747709C4303C58B
:10B73000C701828097A7FF1F9387476F9C4303C56C
:10B74000D701828097A7FF1F9387476E9C43885736
:10B75000828097A7FF1F9387676D9C4303D5C7021D
:10B76000828097A7FF1F9387676C9C4303D5E702EE
:10B7700019E11305800C828097A7FF1F9387076B41
:10B780009C4303C50703828097A7FF1F9387076A1F
:10B790009C43C85B828097A7FF1F9387A768884355
:10B7A000828097A7FF1F938727688843828019E1CB
:10B7B0007D558280F5DE984265DFFDD917B7FF1F02
:10B7C0001307C7891847AA877155058B631D07247E
:10B7D00003C507001547E37DA7FC03C73700130522
:10B7E000F0057D171377F70FE364E5FC03C35700FB
:10B7F000E30003FC83C86700E38C08FA03C7770003
:10B80000494579171377F70FE364E5FA03C7A700F3
:10B8100011481305F7FF1375F50FE36BA8F803CE76
:10B8200097000D481305FEFF1375F50FE362A8F8A6
:10B8300003C8B7006309080065181378F80F1305EB
:10B84000600DE36705F703C5C700794879151375DF
:10B85000F50FE36FA8F403C8D7000D457D181378E2
:10B86000F80FE36705F503D80701930E4017511849
:10B87000420813580801E3ED0EF303C8E7007D18F2
:10B880001378F80FE36605F303C827017D181378D2
:10B89000F80FE36F05F103C88700C54E75181378DC
:10B8A000F80FE3E70EF103D86701856E938EBEE0D3
:10B8B0006D18420813580801E3EC0EEF03D8470156
:10B8C0006D18420813580801E3E40EEF03D887010E
:10B8D0007918420813580801E36C05ED03C8A70165
:10B8E0007D181378F80FE36505ED03C5B7011D4812
:10B8F0007D151375F50FE36DA8EA03C5D7017148EF
:10B9000079151375F50FE365A8EA03D5E701130868
:10B91000E00F7D1542054181E36CA8E803C50702ED
:10B92000494879151375F50FE364A8E8C85301C9B0
:10B9300037C834005915130858BFE36BA8E603A8AD
:10B94000870237C53400130555BF5918E36205E770
:10B9500017A5FF1F232AC54C03C6050117A5FF1F06
:10B960002326F54C0545E375C5E403D82501D049E8
:10B9700033760603E31E06E203C61501E30A06E278
:10B9800017A6FF1F2320B64A83C5270001466387F9
:10B99000A50003C61700F1453306B60283C70703A7
:10B9A0009305C00272971A071307C70516031A9763
:10B9B00096084697B387B70241553E97329742079C
:10B9C00041836362E8061763FFFFE7024371368530
:10B9D00097800000E780806B97000100E780004BB4
:10B9E0002A8497A00000E780605D2A9497F0000009
:10B9F000E78040292A9497900000E78080842A9469
:10BA000097F0FFFFE780E06F2A9497400000E780FF
:10BA100000972A9497700000E780809F2295176313
:10BA2000FFFF6700036E82801763FFFFE702236B4F
:10BA30004111A307A10097A00000E78080C89305EB
:10BA4000F100170500001305E5B597F0FFFFE7804B
:10BA5000802F014541011763FFFF6700836A176369
:10BA6000FFFFE702436517A4FF1F1304245F0328A9
:10BA7000840079599368180097A4FF1F23A4145FCA
:10BA80001378180063100802BA84BE89368B328A94
:10BA90002E89AA8A97F0FFFFE780E0A77D152695FB
:10BAA00019E531594A851763FFFF6700436497F032
:10BAB000FFFFE78040A67D152695A167E353F5FEBD
:10BAC00097B7FF1F9387879098433E8C814B01CB9C
:10BAD000014597F00000E7800047933B15004A8539
:10BAE000DA865686D28597900000E780A0502A8992
:10BAF00011CD1C44F99B17A7FF1F2325F756832759
:10BB00000C00CDD3E3800BFA829769BF268597A7F7
:10BB1000FF1F23A7075497F0FFFFE780809C414653
:10BB2000CE8517A5FF1F1305E55C97300100E78060
:10BB3000A05997D00000E780209C0325040B97D0E4
:10BB40000000E780E09F054597D00000E780E0A671
:10BB5000054597000000E78060EDA9B797A7FF1F94
:10BB60009387C74F9C47858BEDC71763FFFFE7029D
:10BB7000035717A5FF1F1305255697A7FF1F23AFD0
:10BB8000074C97A7FF1F23AD074C97A7FF1F23ABB9
:10BB9000074C97200100E780008497500000E78061
:10BBA000C0F897100100E780804F97100100E780F0
:10BBB000805597A7FF1F9387E7489C4391C705458A
:10BBC00097800000E780202397A7FF1F93874731C6
:10BBD0009C4399C741657D1597700000E78020A5BB
:10BBE00097F00000E780C04097D00000E7806092A7
:10BBF00097A7FF1F9387875B9C4313971701635693
:10BC0000070097F00000E780E0AF97A7FF1F23A38E
:10BC1000074E97A7FF1F23A1074E97A7FF1F23AF2C
:10BC2000074C97A7FF1F23AD074C97000000E78044
:10BC3000008C97000000E780A07597F0FFFFE78079
:10BC4000401897F00000E78020D91763FFFF6700D6
:10BC5000434B828097A7FF1F93874740884382808A
:10BC600097A7FF1F9387873FC8438280B7E7B0003D
:10BC70009387075063E1A70297A7FF1F9387073EAB
:10BC8000D843FD576367E50097A7FF1F23AAA73C8A
:10BC900081473E858280B957EDBF1763FFFFE702FA
:10BCA000034497800000E780A07497800000E7803D
:10BCB00000771763FFFF6700C3441763FFFFE702C6
:10BCC00063402A849304140201112E85B289A6854B
:10BCD000214636C63A8997300100E780803C0DE95D
:10BCE000B24638082686CE85130594049750000086
:10BCF000E780A04021462C084A8597300100E78064
:10BD0000403A1335150005611763FFFF6700C33E16
:10BD10000145D5BF1763FFFFE702633C9305450666
:10BD200017A5FF1F1305C51097100100E780606875
:10BD30001763FFFF6700E33C1763FFFFE702233A47
:10BD400041112EC697F0FFFFE780C017B24588C1AA
:10BD500041011763FFFF6700C33A1763FFFFE70264
:10BD60006336AA842E8497800000E780406BAA89FE
:10BD70008545228597000000E780E07D83C7E401C8
:10BD80001389940899E313890403CE8522859700CB
:10BD90000000E780407C2146930519022285970028
:10BDA0000000E780607897A7FF1F9387272B8C43BD
:10BDB000228597100000E780C08221469385840287
:10BDC000228597000000E78020761763FFFF670059
:10BDD000A3321763FFFFE702032E397197F00000CB
:10BDE000E78020B49305400661E997800000E78072
:10BDF000405F6302051497A7FF1F83C7270513B78A
:10BE0000170097A6FF1F2383E604014499CFC1645E
:10BE100017A9FF1F130989249309400EFD149700E9
:10BE20000000E78020836342A40A97F0FFFFE780C9
:10BE300060094169B7290900096AFD7A2A8B8144A2
:10BE40007D199389F97B130A0A71938A8AC797002F
:10BE50000000E780208063D7A4041304400EB3875A
:10BE6000840217A7FF1F1307671F0324070B3E94C5
:10BE70008357C4016382270B18403307EB4063EA02
:10BE8000E900834744008507B3874703D697636576
:10BE9000F70801468145094597F0FFFFE780C04A52
:10BEA000AA8B29E597400000E780C0828547631789
:10BEB000F50689659385057117A5FF1F130545F7DD
:10BEC00097100100E780E04E95A0B30734030327E5
:10BED000090BBA9703D7C7016308970003C7570038
:10BEE000A38207002382E700050415BF9305C50060
:10BEF000228597000000E78080E65E8522869765B0
:10BF000001009385A5E697F0FFFFE780404F5E852F
:10BF100097100000E780608A850415BF97A7FF1F70
:10BF20009387C7139C478D83858BC1F72161176366
:10BF3000FFFF6700C31B01468545094502D002D2B9
:10BF400002D402D697F0FFFFE7800040AA8479DD93
:10BF500097F00000E780209C1389C4002A84814563
:10BF60004A8597000000E780005F0C4041464A8503
:10BF700097000000E780405B832944006385090C3B
:10BF80004E8502D802DA02DC02DE97300100E7803B
:10BF900020382ACE141005462C0808184ECC97508D
:10BFA0000000E780200A1375F50F51ED83558400DA
:10BFB00093E525004A8597000000E780E05E114682
:10BFC0000C104A8597000000E780005601469765EF
:10BFD0000100938525DA268597F0FFFFE780204250
:10BFE000268597000000E780407D5C40A1D3014694
:10BFF00085450D4597F0FFFFE7800035AA841DD5E4
:10C0000048401389C40097300100E78060302AC699
:10C010004A8597000000E780404C3246636FC500B8
:10C020004C404A8597000000E7800050014681455A
:10C03000268597F0FFFFE780803C2685970000006B
:10C04000E780A077E5B583558400ADB71763FFFFA0
:10C05000E702E30897A7FF1F938747009C471DC18E
:10C0600093E7870017A5FF1F130585DC17A7FF1FA0
:10C07000232AF7FE97100100E78080311763FFFF46
:10C0800067002308DD9B17A7FF1F232DF7FC9730C0
:10C090000000E78020647DF117A5FF1F130545D937
:10C0A00097100100E7802033D1BF1763FFFFE7023D
:10C0B00083004169AA892E8AB28A368BBA8B814461
:10C0C00017ACFF1F130C8CF9930C400E7D1997F0E1
:10C0D000FFFFE780205863C4A40001443DA03384DF
:10C0E000940383270C0B3E948357C4016386270572
:10C0F0005A87D6865286CE85130504039700000022
:10C10000E780E0BB01C923800B0022851763FFFF96
:10C110006700E3FD8347F40185C35A87D6865286BC
:10C12000CE851305940897000000E78040B909C543
:10C1300085472380FB00D1BF850451BF835745004D
:10C140006380071E1763FFFFE702C3F701112A840C
:10C1500097000000E780C04D09C985476309F506CF
:10C1600005611763FFFF670023F997E00000E78090
:10C17000407B7DF5835744004947ED9BE392E7FE02
:10C18000C145228597000000E7804033AA842285BC
:10C1900097000000E780204F0357440002CE9147EC
:10C1A0002A89631AF700228597000000E780A051D2
:10C1B0003C082ACC3ECE97E00000E780C0755C5575
:10C1C000C5D374084A86A6850545829751BF035793
:10C1D0004400D147E3F6E7F8032A0400C1690149A6
:10C1E00097AAFF1F938A8AE7130B400EFD1997F059
:10C1F000FFFFE7802046634FA90E2285032A040033
:10C2000097000000E780C042A1452A892285970057
:10C210000000E780A02AAA84228597000000E7801A
:10C22000804A14402A86AA8978082685CA859700FC
:10C230000000E780C0E7AA8405D503C7F401894759
:10C240006315F7008347C10181DF5546D285138509
:10C25000640097300100E78020E7014597800000E7
:10C26000E780001901C583D7C401A5E797A7FF1F81
:10C270009387C7DE9C4793551900858913D73700EC
:10C28000058B01CF8983858B6399B70001452EC645
:10C2900097000000E780C0DBB2454E859780000024
:10C2A000E780A01E0346C1012A84937519002685E4
:10C2B00097900000E780203935C1268597800000DF
:10C2C000E7802018268511C0014597800000E7808F
:10C2D000404B97300000E780E03F8547E312F5E8E8
:10C2E00083C754001307F00FE38CE7E68507A382AA
:10C2F000F400BDB5B304690383A70A0BBE9483D7CA
:10C30000C401638B37015546D2851385640097308D
:10C310000100E78000D955DD0509D1BD5DD86DB7B5
:10C3200082801763FFFFE702E3D997800000E78070
:10C33000400B05C1C164014417A9FF1F130909D2AD
:10C340009309400EFD1497F0FFFFE780A030634E85
:10C35000A40017A5FF1F1305A5AD97100100E780E6
:10C3600020031763FFFF670023D9330534038327B6
:10C37000090B3E958357C50163889700231205007A
:10C3800097800000E780E00B050475BF97A7FF1FAB
:10C390009387C7CC9C478D83858B8DE31763FFFF05
:10C3A000E702E3D317A5FF1F130585A89710010027
:10C3B000E78060021763FFFF6700A3D482801763E2
:10C3C000FFFFE702C3D1970500009385C5A017A51D
:10C3D000FF1F1305E5A597100100E78060ED1763C7
:10C3E000FFFF670003D21763FFFFE70243CF8841D7
:10C3F000B7E70400BC5B050542054181829709C58A
:10C4000085472300F50005051763FFFF670063CF2D
:10C4100083C7F5FF2E858507A38FF5FE828083C72E
:10C42000F5FFFD1793F7F70FA38FF5FE99EF17634D
:10C43000FFFFE702C3CAB7E70400BC571385F5FF47
:10C4400082971763FFFF6700C3CB82801C410357AD
:10C4500045008D8FBA951CC12312B5003E858280A0
:10C4600093D78500A2051441DD8D835745001387BE
:10C47000E6FF18C189072312F50013D68500411184
:10C48000238FB6FEA38FC6FE410182801841930719
:10C49000F7FF1CC18357450085072312F500A30F42
:10C4A000B7FE8280835745008D8F2312F5001C4113
:10C4B000BE950CC12E858280AA8703D7470008410C
:10C4C0000D8FAA952392E7008CC3828018410845FE
:10C4D0003305A740828083574500035765001D8FB1
:10C4E0001C4108453385A7403305A7408280176368
:10C4F000FFFFE702C3BE41112EC62A849700000049
:10C50000E780A0FDB2456373B50001A083574400E6
:10C510000840BE952312B4003E9541011763FFFF0A
:10C52000670023BE1763FFFFE70263BB41112E8440
:10C53000B28532C697000000E780A0FB3246A28594
:10C5400097300100E78040B841011763FFFF6700A3
:10C5500043BB1763FFFFE70283B82E84854597002E
:10C560000000E78000F9230085001763FFFF6700E4
:10C5700043B91763FFFFE70283B641112317B100E8
:10C58000894597000000E780C0F68347E10023005B
:10C59000F5008347F100A300F50041011763FFFF99
:10C5A000670023B61763FFFFE70263B393D78500E5
:10C5B000A2054111DD8D2317B100894597000000C8
:10C5C000E78020F38347E1002300F5008347F10073
:10C5D000A300F50041011763FFFF670083B21763F3
:10C5E000FFFFE702C3AF1397850193D78501C166AB
:10C5F000938606F0D98F13D78500758FD98FA20542
:10C600003707FF00F98D4111DD8D2EC6914597004A
:10C610000000E78000EE6C00114697300100E780D3
:10C62000A0AA41011763FFFF6700A3AD1763FFFFD7
:10C63000E702E3AA1C41854503C4070097000000F8
:10C64000E78080E622851763FFFF670083AB1763EF
:10C65000FFFFE702C3A81C414111894503C707003A
:10C6600083C717002307E100A307F100970000002C
:10C67000E78080E30355E10041011763FFFF670096
:10C6800043A81763FFFFE70283A51C4141118945B9
:10C6900003C7070083C717002307E100A307F100C2
:10C6A00097000000E78040E08357E100410113D587
:10C6B0008700A2075D8D420541811763FFFF670078
:10C6C00043A41763FFFFE70283A10C4141112A84B1
:10C6D0001146680097300100E780009F9145228550
:10C6E00097000000E78040DCB247C166938606F001
:10C6F0001397870113D58701598D13D78700758F3D
:10C70000598DA2073707FF00F98F5D8D410117632F
:10C71000FFFF6700039F1C45BE950CC18280AE875A
:10C72000944391E6584101EF0CC15CC1828003C77C
:10C73000570013671700A382E700B687D5B70CC36D
:10C74000EDB7AA87084119CD1841D44398C36313A4
:10C75000D500D8C32A87034657009376160081E692
:10C76000232007008280944381CA8C4203A847009B
:10C770008CC363930601CCC3799A14C3A302C70088
:10C780003687D1BF1C45DC471D8DB777DBB6938755
:10C7900077DB09853305F502420541818280F14747
:10C7A000B385F50248452E9582808347450085076D
:10C7B0002302F50082801763FFFFE70243922A8479
:10C7C00009E41763FFFF6700C39383474400F5DB69
:10C7D000FD1793F7F70F2302F400E5F71C4403D786
:10C7E000270005072391E700DC4399C32285829740
:10C7F0004C4889CD83475400898B99E71C44228596
:10C800009C479C439C478297232A04000040232096
:10C8100004007DB71763FFFFE702638C8357250091
:10C8200041112EC681EB0144228541011763FFFFB0
:10C830006700238D035705008147F146E305F7FEA6
:10C84000B385D702404585072E948345440008C42C
:10C85000F5F5B247AA8481E7232A040009A81C45FC
:10C860006C0022859C439C43829748C84DDD8547D8
:10C870002312F400B24723200400231804002319D4
:10C88000F4005C485CC483D72400FD172391F400B6
:10C8900061BF1763FFFFE70283849797FF1F9387AA
:10C8A000275B8843232605002324050041059710B4
:10C8B0000100E78040B21763FFFF670083841763BE
:10C8C000FFFFE702C3811794FF1F130464581C4045
:10C8D000411199CF9C472300B5002AC65CC197003F
:10C8E0000000E78040FB1C40DC4399C3324582973F
:10C8F00041011763FFFF6700C3800347450029E339
:10C90000584DAA877D551DCF1753FFFFE702237DA2
:10C910001CC3DC479796FF1F23ACE652F156130564
:10C9200007012390D7009705000093850502971013
:10C930000100E780E09701451753FFFF6700637C24
:10C940007D55828082801753FFFFE70243790111F2
:10C950006146814528009750FFFFE780407B97970D
:10C96000FF1F9387E74E9C4328009305F00FDC4799
:10C970003EC697000000E780C0F405611753FFFF33
:10C98000670023789797FF1F9387874C9C43D8476E
:10C99000A1679387C702631EF70A397106DE22DC9E
:10C9A00026DA80004AD84ED652D456D23285B28486
:10C9B00097000000E780C0C7AA892685970000007D
:10C9C000E78020C92318A4FC268597000000E78093
:10C9D00040C82319A4FC268597000000E78060C7A3
:10C9E00083D744000A8A231AA4FC858393F7F70FA0
:10C9F000230EF4FC8607BD0793F7073F3301F14090
:10CA00008A8A01498347C4FD6367F902CE8513050D
:10CA100084FC232C54FD97000000E78080EA5281BB
:10CA2000130104FCF2506254D2544259B259225AB2
:10CA3000925A21618280268597000000E78060C1BC
:10CA400093171900D69705092390A7001379F90FBA
:10CA500055BF82809797FF1F9387873F9C43D84796
:10CA6000A1679387A702631AF70A397106DE22DCF1
:10CA700026DA80004AD84ED652D456D23285B284B5
:10CA800097000000E780C0BAAA89268597000000B9
:10CA9000E78020BCFD572318A4FC26852319F4FC4D
:10CAA00097000000E780E0BA83D744000A8A231A7F
:10CAB000A4FC858393F7F70F230EF4FC8607BD07CC
:10CAC00093F7073F3301F1408A8A01498347C4FD48
:10CAD0006367F902CE85130584FC232C54FD97006F
:10CAE0000000E78000DE5281130104FCF250625422
:10CAF000D2544259B259225A925A216182802685D3
:10CB000097000000E780E0B493171900D697050955
:10CB10002390A7001379F90F55BF82809797FF1FC5
:10CB2000938707339C43D847A16789076310F70AA7
:10CB3000397106DE22DC26DA80004AD84ED652D47D
:10CB400056D23285328997000000E78060AEAA890C
:10CB50004A8597000000E780C0AF835749000A8AE2
:10CB60002318A4FC858393F7F70F230CF4FC8607A6
:10CB7000BD0793F7073F3301F1408A8A8144834719
:10CB800084FD63E7F402CE85130584FC232A54FD5B
:10CB900097000000E780E0D25281130104FCF250BC
:10CBA0006254D2544259B259225A925A2161828017
:10CBB0004A8597000000E780C0A993971400D69794
:10CBC00085042390A70093F4F40F55BF82809797B4
:10CBD000FF1F9387E7279C43D847A1679387E70404
:10CBE000631EF70A397106DE22DC26DA80004AD895
:10CBF0004ED652D456D23285B28497000000E780D8
:10CC000020A3AA89268597000000E78080A4231826
:10CC1000A4FC268597000000E780A0A3231AA4FCAB
:10CC2000268597000000E780C0A283D744000A8AC7
:10CC30002319A4FC858393F7F70F230EF4FC8607D2
:10CC4000BD0793F7073F3301F1408A8A01498347C3
:10CC5000C4FD6367F902CE85130584FC232C54FDC3
:10CC600097000000E780E0C55281130104FCF250F8
:10CC70006254D2544259B259225A925A2161828046
:10CC8000268597000000E780C09C93171900D6976F
:10CC900005092390A7001379F90F55BF8280979754
:10CCA000FF1F9387E71A9C43D847A1679387C70460
:10CCB000631AF70A397106DE22DC26DA80004AD8C8
:10CCC0004ED652D456D23285B28497000000E78007
:10CCD0002096AA89268597000000E7808097FD5757
:10CCE0002318A4FC2685231AF4FC97000000E78093
:10CCF000409683D744000A8A2319A4FC858393F7BE
:10CD0000F70F230EF4FC8607BD0793F7073F3301A7
:10CD1000F1408A8A01498347C4FD6367F902CE85E1
:10CD2000130584FC232C54FD97000000E78060B9B4
:10CD30005281130104FCF2506254D2544259B25948
:10CD4000225A925A21618280268597000000E7804E
:10CD5000409093171900D69705092390A7001379DF
:10CD6000F90F55BF82809797FF1F9387670E9C43EB
:10CD7000D847A167DD076317F7041753FFFFE702E2
:10CD8000033679713285328497000000E780408A4B
:10CD90002AC6228597000000E780A08B2311A102FC
:10CDA000228597000000E780A088B2452300A102F9
:10CDB000280897000000E780C0B045611753FFFFC7
:10CDC0006700233482809797FF1F938767089C43EF
:10CDD000D847A167938787046317F7041753FFFFAA
:10CDE000E702E32F79713285328497000000E780F3
:10CDF00020842AC6228597000000E78080852311C1
:10CE0000A102228597000000E7808082B2452300BE
:10CE1000A102280897000000E780A0AA45611753E7
:10CE2000FFFF6700032E82809797FF1F93874702BB
:10CE30009C43D847A1679387A7046312F70217534F
:10CE4000FFFFE702C3290111280081459700000078
:10CE5000E78020A705611753FFFF6700832A8280C0
:10CE60009797FF1F9387C7FE9C43D847A167938777
:10CE700057026319F7021753FFFFE7024326011118
:10CE8000328597F0FFFFE780A07A2308A100814553
:10CE9000280097000000E780C0A205611753FFFF3C
:10CEA0006700232682809797FF1F938767FA9C432A
:10CEB000D847A1679387E702631BF7041753FFFF67
:10CEC000E702E32101113285328497F0FFFFE7800A
:10CED0004078AA84228597F0FFFFE7808077854716
:10CEE00009E9228597F0FFFFE78080744205B33798
:10CEF000A00028008145231891003ECA9700000039
:10CF0000E780209C05611753FFFF6700831F828025
:10CF10009797FF1F9387C7F39C43D847994763139D
:10CF2000F7081753FFFFE702831B797132853284BC
:10CF300097F0FFFFE780C06F2AC6228597F0FFFFBA
:10CF4000E78020712310A102228597F0FFFFE78080
:10CF5000206E2301A102228597F0FFFFE780406D3C
:10CF6000A301A102228597F0FFFFE780606C2302F6
:10CF7000A102228597F0FFFFE780806B2313A102B7
:10CF8000228597F0FFFFE780A06AB2452314A10233
:10CF9000280897000000E780C09245611753FFFF03
:10CFA0006700231682809797FF1F938767EA9C4349
:10CFB000D847A1679387C7036313F7081753FFFF89
:10CFC000E702E31179713285328497F0FFFFE78041
:10CFD00020662AC6228597F0FFFFE780806723102E
:10CFE000A102228597F0FFFFE780A0662311A1022E
:10CFF000228597F0FFFFE780A0632302A10222852C
:10D0000097F0FFFFE780C062A302A102228597F09C
:10D01000FFFFE780E0612303A102228597F0FFFF75
:10D02000E7800061B245A303A10228089700000031
:10D03000E780208945611753FFFF6700830C8280DA
:10D040001753FFFFE702A30901112A8497F0FFFF9E
:10D05000E780005EAA84228597F0FFFFE780605F8B
:10D06000228597F0FFFFE780C05E035744008D479D
:10D0700063F7E700228597F0FFFFE780805D228558
:10D0800097F0FFFFE780E05C2800A685970000008E
:10D09000E780208305611753FFFF6700830697979A
:10D0A000FF1F9387E7DA9C43D847A167FD07631FFB
:10D0B000F7001753FFFFE702830232859700000055
:10D0C000E78040F81753FFFF6700A303828097971C
:10D0D000FF1F9387E7D79C43D847A167E5076315F0
:10D0E000F7081753FFFFE70283FF79713285328417
:10D0F00097F0FFFFE780C0532AC6228597F0FFFF15
:10D10000E7802055228597F0FFFFE78080542310A9
:10D11000A102228597F0FFFFE780A05352055181BD
:10D120002311A10222852302010297F0FFFFE7806D
:10D130002050A302A102228597F0FFFFE780404F15
:10D140002303A102228597F0FFFFE780604EB245DE
:10D15000A303A102280897F0FFFFE78080764561CE
:10D160001753FFFF6700E3F982809797FF1F9387AC
:10D1700027CE9C43D847A1679387E703631FF70037
:10D180001753FFFFE702A3F5328597000000E78001
:10D1900060EB1753FFFF6700C3F682809797FF1F6E
:10D1A000938707CB9C43D847A16793874704631EA7
:10D1B000F7021753FFFFE70283F279713285328459
:10D1C00097F0FFFFE780C0462AC6228597F0FFFF51
:10D1D000E7802048B245280897F0FFFFE780606E9F
:10D1E00045611753FFFF6700C3F182809797FF1FC8
:10D1F000938707C69C43D847A1679387870263102C
:10D20000F7041753FFFFE70283ED7971328532840B
:10D2100097F0FFFFE780C0412AC6228597F0FFFF05
:10D22000E7800041B2452300A102280897F0FFFFE4
:10D23000E780206945611753FFFF670083EC828018
:10D240001753FFFFE702A3E9011197F0FFFFE78003
:10D25000203EAA85280097F0FFFFE78080660561E1
:10D260001753FFFF6700E3E99797FF1F938747BEB8
:10D270009C43D847A167D107631FF7001753FFFFEF
:10D28000E702E3E5328597000000E780A0FB175333
:10D29000FFFF670003E782809797FF1F938747BBD5
:10D2A0009C43D847A167C507631FF7001753FFFFCB
:10D2B000E702E3E2328597000000E780A0F8175309
:10D2C000FFFF670003E482809797FF1F938747B8AB
:10D2D0009C43D847A167B907631FF7001753FFFFA7
:10D2E000E702E3DF328597000000E780A0F51753DF
:10D2F000FFFF670003E182809797FF1F938747B581
:10D300009C43D847A167AD07631FF7001753FFFF82
:10D31000E702E3DC328597000000E780A0F21753B4
:10D32000FFFF670003DE82809797FF1F938747B256
:10D330009C43D84789476318F7021753FFFFE7025A
:10D3400003DA0111328532C897F0FFFFE780402EE3
:10D35000AA85280097F0FFFFE780A05605611753C4
:10D36000FFFF670003DA82809797FF1F938747AE1E
:10D370009C43D847A1678D076311F7041753FFFF3C
:10D38000E702E3D501113285328497F0FFFFE78091
:10D39000202A13066100AA844C00228597300000E1
:10D3A000E78000232800A68597F0FFFFE780605103
:10D3B00005611753FFFF6700C3D482809797FF1F53
:10D3C000938747A99C4381CFDC4391CB1753FFFF41
:10D3D000E702E3D082971753FFFF670083D2828072
:10D3E0001753FFFFE702A3CF79713C08AE843ED20A
:10D3F000A165B7070A002A843ED448103C08DD0521
:10D400003ED636C432C63AC297D0FFFFE780402CE2
:10D4100012474810BA8597F0FFFFE780C0133246E5
:10D420004810B28597F0FFFFE780E014A24648104D
:10D43000B68597F0FFFFE780001250100147814644
:10D44000A685228597D0FFFFE780E04D4561175301
:10D45000FFFF670003CB1753FFFFE70243C801112B
:10D460007C000329C501AE843ECAA165B707070049
:10D470002A843ECC48087C00C5053ECE97D0FFFFED
:10D48000E78000258345D900480897F0FFFFE78033
:10D49000800C500801478146A685228597D0FFFF62
:10D4A000E780604805611753FFFF670083C5175386
:10D4B000FFFFE702C3C283C7950093F7F707A38472
:10D4C000F50097000000E78040F91753FFFF670061
:10D4D00043C31753FFFFE70283C079713C08AE8452
:10D4E0003ED2A165B70709002A843ED448103C0803
:10D4F000938545043ED632C636C497D0FFFFE780F9
:10D50000201DA2464810B68597F0FFFFE780A004D3
:10D5100032464810B28597F0FFFFE780C0055010F3
:10D5200001478146A685228597D0FFFFE780A03F6F
:10D5300045611753FFFF6700C3BC1753FFFFE702A6
:10D5400003BA83C7950041112A8493F7F707A38490
:10D55000F50032852EC697F0FFFFE780800F8567C4
:10D560002AC46370F50297700000E78060E82246E5
:10D57000B24509ED11478146228597000000E780FA
:10D5800060E641011753FFFF6700A3B701478346D9
:10D59000F501DDB71753FFFFE702C3B201113C00ED
:10D5A0003ECAB7070A003ECC3C003ECE83C795007A
:10D5B000AA89328593F7F707A384F5002E8497F0A4
:10D5C000FFFFE78000098567637DF504A165AA84F4
:10D5D00093858504480897D0FFFFE780600F268574
:10D5E00097700000E780C0E02A8929E1914548084A
:10D5F00097F0FFFFE78020F6A685480897F0FFFF29
:10D60000E78060F7CA85480897F0FFFFE780A0F43D
:10D61000014781465008A2854E8597D0FFFFE780DD
:10D62000803005611753FFFF670003AD814548084F
:10D6300097F0FFFFE78020F20349090275BF1753F7
:10D64000FFFFE70223A879711C103ECAB7070F003D
:10D650003ECC404D1C10AA84AE894808994532C67C
:10D6600036893ECE97D0FFFFE780800632464808D5
:10D67000B28597F0FFFFE78000EE630C0902A54535
:10D68000480897F0FFFFE780C0E62546CA85972047
:10D690000100E78060A3500801478146CE852685BA
:10D6A00097D0FFFFE780202845611753FFFF6700F1
:10D6B000A3A48355C402480897F0FFFFE780A0EBBE
:10D6C0000355E402814505C5854785456301F5029B
:10D6D000C167FD179305F00F630BF5007D1597707B
:10D6E0000000E780608D9305150093F5F50F48085D
:10D6F00097F0FFFFE78020E683450403480897F092
:10D70000FFFFE78040E583451403480897F0FFFFDB
:10D71000E78060E483552403480897F0FFFFE78023
:10D7200080E583554403480897F0FFFFE780A0E4B5
:10D730009DB71753FFFFE702839A83C79500814681
:10D74000014693F7F707A384F50097000000E780F0
:10D7500040EF1753FFFF6700C39A1753FFFFE7021D
:10D76000039879713E841C103ECA2E89B7070F00BA
:10D77000A1653ECCFD051C10AA84480842C03AC2EF
:10D780003ECE36C432C697D0FFFFE78060F4324603
:10D790004808B28597F0FFFFE780E0DBA246480823
:10D7A000B68597F0FFFFE78000DD12474808BA858D
:10D7B00097F0FFFFE78020DC0248630C08029145E8
:10D7C000480897F0FFFFE780C0D21146A285972056
:10D7D0000100E780608F500801478146CA85268591
:10D7E00097D0FFFFE780201445611753FFFF6700C4
:10D7F00043918945480897F0FFFFE78080CF834732
:10D8000004002300F50083471400A300F500E1B7EE
:10D810001753FFFFE702038B83C7950001112A8A84
:10D8200093F7F707A384F5003285AE8432C697F0EC
:10D83000FFFFE78000E232462A89328597F0FFFF3A
:10D84000E78000DF85676373F902AA894A859770CC
:10D850000000E780E0B92A8419ED114781464A8625
:10D86000A685528597000000E780C0B70561175371
:10D87000FFFF670063889387E9FF93F7F70F05477A
:10D88000E366F7FE8347F50195EB8947E380F9FEF0
:10D890008346F401528501474A86A6859700000019
:10D8A000E78040B4A167D90748083ECC230A0100AD
:10D8B00002CE97000000E780A0B04DBF639EE70056
:10D8C0008947639EF90093071020231FF500977086
:10D8D0000000E78000B76DBF0947E39BE7FA8D477B
:10D8E000E398F9FA228597700000E780C0DE9787F9
:10D8F000FF1F938727759C4399E79787FF1F93879F
:10D90000275E9C4399C703D5040097800000E780F9
:10D91000E0CD231F040022855DBF1743FFFFE70210
:10D92000037C01113C003ECAB7070B003ECC3C0013
:10D930003ECE83C795002A89328593F7F707A384E3
:10D94000F500AE8497F0FFFFE780A0D093170501A4
:10D95000C187635AF006A1652A849385E5024808C9
:10D9600097D0FFFFE780C0D6A285480897F0FFFF59
:10D97000E78060C09787FF1F938787569C43A9EB7A
:10D9800001449375F40F480897F0FFFFE780A0BCAF
:10D990009355844093F5F50F480897F0FFFFE78013
:10D9A00080BB9355044193F5F50F480897F0FFFFAE
:10D9B000E78060BA014781465008A6854A8597D01E
:10D9C000FFFFE78040F605611743FFFF67006373C1
:10D9D000416585460546A2857D1597500000E78084
:10D9E000A0BC59DD510597000100E780C08E1304EB
:10D9F00040063344850271B71743FFFFE702236EE9
:10DA00000111B70706003EC683C7950021642A8925
:10DA100093F7F707A384F500AE8428009305A404C8
:10DA20000AC40AC897D0FFFFE78080CA30000147C8
:10DA30008146A6854A8597D0FFFFE780C0EE97E034
:10DA4000FFFFE780E01113049404480822CC230A66
:10DA5000010002CE97000000E78080960561174321
:10DA6000FFFF6700036A1743FFFFE702A365C16476
:10DA70002A8901449789FF1F9389495E130A80020E
:10DA8000FD1497E0FFFFE780E0BD6347A400014578
:10DA90001743FFFF67004366B307440303A7C90AA0
:10DAA000BA9703D707006306970083D727006384DC
:10DAB00027010504F9B70545E1BF1743FFFFE7025A
:10DAC00063602A8A2E8999C123A005008149814477
:10DAD000978AFF1F938A4A38614B97E0FFFFE780E0
:10DAE000A0BE63C7A4004E851743FFFF6700C36055
:10DAF0003384640383A70A003E948357040099E7A4
:10DB000063040900232089008504C1BF4146D285F2
:10DB10001305440097100100E780A05875F5A2890D
:10DB2000E5B71743FFFFE702E35939717C083ED49C
:10DB3000B7070A003ED67C083ED883C795002A8ADC
:10DB4000328593F7F707A384F5002E8932C697F044
:10DB5000FFFFE78000B085676373F5083246AA844B
:10DB6000328597F0FFFFE780A0AC8547AA8963E87C
:10DB7000A706A16593858504281097D0FFFFE7804D
:10DB800020B5268597700000E78080862A8429EDDD
:10DB90009145281097F0FFFFE780E09BA6852810AD
:10DBA00097F0FFFFE780209DCE85281097F0FFFFBC
:10DBB000E780609A014781463010CA85528597D028
:10DBC000FFFFE78040D6A1679387770448183EDCC3
:10DBD000230A010202DE97F0FFFFE780607E2161E9
:10DBE0001743FFFF670043518145281097F0FFFF5F
:10DBF000E7806096A685281097F0FFFFE780A09742
:10DC00009787FF1F9387477C9C4381CB228563893D
:10DC1000090097D00000E78080238345040271B794
:10DC200097D00000E7800022CDBF1743FFFFE70237
:10DC3000634983C795004111AA8993F7F707A38425
:10DC4000F5003285AE84328A97F0FFFFE78060A04E
:10DC50008567637FF5022A8997600000E780407935
:10DC60002A84914631C58347F50105476387E7025A
:10DC700091C70D476366F704AD461DA893050503DC
:10DC800003250A00414697100100E78080410DE915
:10DC900041011743FFFF67002346930595080325BD
:10DCA0000A00414697100100E780A03F814669F5D0
:10DCB0004A86A6854E8597000000E780C081C9BFCF
:10DCC00083250A001305940897700000E780E02878
:10DCD00019C1C146F1BF9787FF1F9387A7369C43A1
:10DCE00099E79787FF1F9387A71F9C4399C72285B2
:10DCF00097800000E780608969FD8547A30FF400E5
:10DD0000228597B00000E780A083228597600000FD
:10DD1000E78020734E8581464A86A68597F0FFFFEF
:10DD2000E780607BA1679387570448003EC42302C5
:10DD3000010002C697F0FFFFE780806891BF17439C
:10DD4000FFFFE702433783C795004111AA8993F784
:10DD5000F707A384F50032852E89B28A97F0FFFF7A
:10DD6000E780208F85676374F50EAA8497600000B2
:10DD7000E78000682A840DED416B014A978BFF1FF5
:10DD8000938BCB2D130C400E7D1B19A833048A03F3
:10DD900083A70B0B3E948357C40163836705050A71
:10DDA00097E0FFFFE780008BE342AAFE95460DA0B7
:10DDB0008357C501639697029305050303A50A00DF
:10DDC000414697100100E780C02D994611E1814638
:10DDD0002686CA854E8597F0FFFFE780C06F85A82D
:10DDE00083A50A001305040397700000E780E0167E
:10DDF000C14679FD2285231E940097A00000E7808C
:10DE00002074228597600000E780A0639787FF1F3A
:10DE10009387875B9C43A9C323000402228597D084
:10DE20000000E78080EF4E8581462686CA8597F000
:10DE3000FFFFE780406AA1679387070448003EC45C
:10DE40002302010002C697F0FFFFE78060574101FF
:10DE50001743FFFF6700A32989472300F402E1B7B6
:10DE6000397106DE22DC4AD8800052D456D25AD00C
:10DE700026DA4ED65ECE2E8A32892A8B97D0FFFFC5
:10DE8000E780407A0605710541998A8A3301A140ED
:10DE9000232224FC231404FC97D0FFFFE780807822
:10DEA00083479A000605350593F7F7072315A4FC69
:10DEB000A304FA004A85232624FC97E0FFFFE780AD
:10DEC000407993170501C1876340F0025681130121
:10DED00004FCF2506254D2544259B259225A925A16
:10DEE000025BF24B21618280AA844A8597E0FFFFA2
:10DEF000E7802076AA894A8597E0FFFFE780607572
:10DF0000A1659385C5022A89130544FC97C0FFFFCC
:10DF1000E780007C268597C0FFFFE780407085453D
:10DF200011C94A86CE8597C0FFFFE780C069AA8BDA
:10DF300021E98945130544FC97E0FFFFE780A061D4
:10DF4000A685130544FC97E0FFFFE780C062CE85FD
:10DF5000130544FC97E0FFFFE780E061CA851305E5
:10DF600044FC97E0FFFFE78000610147814613060C
:10DF700044FCD2855A8597D0FFFFE780C09AB9B795
:10DF80008145130544FC97E0FFFFE780C05CA68550
:10DF9000130544FC97E0FFFFE780E05DCE851305A5
:10DFA00044FC97E0FFFFE780005DCA85130544FC51
:10DFB00097E0FFFFE780205C814497D0FFFFE78078
:10DFC0006066E3D4A4FA83A70B0113971400BA97F1
:10DFD00083D5070099C5130544FC97E0FFFFE78050
:10DFE00080598504D9BF797106D622D44AD0001849
:10DFF0004ECE52CC56CA26D25AC8AE893289AA8A87
:10E0000097D0FFFFE78000620605690541990A8AFB
:10E010003301A140232A24FC231C04FC97D0FFFFDA
:10E02000E780406083C7990006052D0593F7F70741
:10E03000231DA4FCA384F9004A85232E24FC97E029
:10E04000FFFFE780006193170501C187634FF00070
:10E050005281130104FDB250225492540259F249E4
:10E06000624AD24A424B45618280AA844A8597E03F
:10E07000FFFFE780005EA1659385A5022A8913054D
:10E0800044FD97C0FFFFE780A064268597C0FFFF8F
:10E09000E780E058854509C9CA8597C0FFFFE7803A
:10E0A00080552A8B29E18945130544FD97E0FFFF40
:10E0B000E780604AA685130544FD97E0FFFFE780EF
:10E0C000804BCA85130544FD97E0FFFFE780A04A17
:10E0D00001478146130644FDCE85568597D0FFFF44
:10E0E000E7806084B5B78145130544FD97E0FFFFE5
:10E0F000E7806046A685130544FD97E0FFFFE780B3
:10E100008047CA85130544FD97E0FFFFE780A046DE
:10E11000814497D0FFFFE780E050E3DBA4FA832738
:10E120000B0113971400BA9783D5070099C51305FF
:10E1300044FD97E0FFFFE78000448504D9BF174303
:10E14000FFFFE702C3F983474500404DD5EFFD5778
:10E150005DC48346940009476363D70A0346B4004D
:10E16000854663EEC6088306E40063CA06085C457C
:10E17000F9562390D7009787FF1F83C727CE99E3CF
:10E18000A304E4009787FF1F938787D59C4381E70B
:10E190008947A306F4009787FF1F9387E7229C43D4
:10E1A00081E789472306F40097050000938545061B
:10E1B000AA841305040197F00000E780600FFD5763
:10E1C000231AF40281471CDC01489787FF1F23A311
:10E1D00087C89787FF1F938727C8232E040304C08F
:10E1E000804397D0FFFFE780204E61463306C5028B
:10E1F000814522859740FFFFE78060F181473E859A
:10E200001743FFFF6700E3EFFD57D5BF1743FFFF3D
:10E21000E702E3EC2A840355450297600000E7809B
:10E22000201D19E5231E04001743FFFF670063ED5F
:10E230008357E401F5DB930504FF1745010013053F
:10E2400025ED97E00000E7802014F9BF1743FFFF9A
:10E25000E702E3E82E89A16541119385E5032A844D
:10E2600036C432C6BE843AC297C0FFFFE78040463C
:10E2700012472285BA8597E0FFFFE780C02D32461E
:10E280002285B28597E0FFFFE780E02EA246228537
:10E29000B68597E0FFFFE780002E630309029145F2
:10E2A000228597E0FFFFE780C0241146A6859710DE
:10E2B0000100E78060E141011743FFFF670063E46D
:10E2C0008945228597E0FFFFE780A02283C70400ED
:10E2D0002300F50083C71400A300F500E9BF17432E
:10E2E000FFFFE702C3DF83C79500444D054793F75F
:10E2F000F707A384F5001C42411183C70700636739
:10E30000F7062E842A89B1C003C7D400630FF70231
:10E310001787FF1F1307C7BC184305C3A386F40064
:10E3200097A00000E780804983C7D40099E7416542
:10E330007D1597400000E780802F83D72403918BC1
:10E3400089C797E00000E78000134A85A28597F00F
:10E35000FFFFE7808010A167C10748003EC4230289
:10E36000010002C697F0FFFFE780800541011743D7
:10E37000FFFF670003D91743FFFFE70243D603D728
:10E3800045008D47AA8441112E8432892E8563E38E
:10E39000E70297E0FFFFE780C02BAA852300090072
:10E3A000268597C0FFFFE780002541011743FFFF47
:10E3B000670023D597E0FFFFE780A0292AC62285C2
:10E3C00097E0FFFFE780E028B24585472A862300D3
:10E3D000F900268597C0FFFFE780E01EF9B7397185
:10E3E00006DE22DC26DA80004ED652D456D24AD837
:10E3F0005AD05ECEAE89B284AA8A97D0FFFFE7805A
:10E40000602106051305250241990A8A3301A140BE
:10E41000232224FC231404FC97D0FFFFE780801FF5
:10E4200083C7990006054D0593F7F7072315A4FC4C
:10E43000A384F9002685232624FC97E0FFFFE780CC
:10E44000402193170501C1876340F00252811301F7
:10E4500004FCF2506254D2544259B259225A925A90
:10E46000025BF24B21618280AA8B03AB040097C050
:10E47000FFFFE780C01A51E583D744000149854476
:10E48000F11793B71700A301F4FC834734FCA1658F
:10E49000C9C79385E504130544FC97C0FFFFE780D7
:10E4A0002023A685130544FC97E0FFFFE780A00A20
:10E4B000DE85130544FC97E0FFFFE780C00B834730
:10E4C00034FC114691E30946DA85130544FC97E0D4
:10E4D000FFFFE78060058144630A0900416B7D1BF3
:10E4E00097D0FFFFE780001363CCA4020147814669
:10E4F000130644FCCE85568597C0FFFFE780A042F7
:10E50000B1B7A685130634FC97000000E780E0E66B
:10E51000933415002A8986048DBF9385C504A5BF51
:10E520008327C90013971400BA9783D5070063881F
:10E530006501130544FC97E0FFFFE780C0038504F5
:10E5400045B71743FFFFE70203B779711C103EC4BC
:10E55000B7070F003EC61C103EC883C79500AA8AA5
:10E56000328593F7F707A384F500AE89328497E0EC
:10E57000FFFFE780000E93170501C187635AF0067D
:10E580002A8A228597E0FFFFE780A00C2A8952851E
:10E59000032B040097C0FFFFE780600839ED835725
:10E5A000440081440544F11793B71700A303F10019
:10E5B00083457100DA872287CA8652862800970031
:10E5C0000000E780E0C8014781463000CE855685CF
:10E5D00097C0FFFFE7802035A1679387D7034808DE
:10E5E0003ECC230A810026CE97F0FFFFE78040DD76
:10E5F00045611743FFFF670083AFA28513067100D3
:10E6000097000000E78060D7AA84094455D13544BB
:10E61000E30055FB4A8597F0FFFFE78000450D4476
:10E6200041D9014497D0FFFFE780C0FE634DA400AD
:10E63000C16B0144FD1B97D0FFFFE780A0FD634E37
:10E64000A4001544B5B7DC4413171400BA9783D758
:10E650000700638327030504F1B7D8449317140018
:10E66000BA9703D70700631B7701239027012685FC
:10E6700097A00000E780C0DA01441DBF050465BF14
:10E680001743FFFFE70203A483C7950041112A8ABD
:10E6900093F7F707A384F50032852E89328497E03B
:10E6A000FFFFE78000FB93170501C1876353F00666
:10E6B000AA89228597E0FFFFE780A0F92311A10036
:10E6C0004E85832A040097C0FFFFE78040F539E5B7
:10E6D0008357440085440144F11793B71700A30002
:10E6E000F1000348110003572100D6875285CE86DA
:10E6F0002686CA8597F0FFFFE7806006A167F107CD
:10E7000048003EC42302910022C697F0FFFFE78035
:10E7100020CB41011743FFFF6700039EA28513062C
:10E72000110097000000E78040C52A84894455D92C
:10E730008357210011678544BA97C2071167C183C7
:10E740001307F7EFE36FF7F89787FF1F9387878F1C
:10E750009C4381CB85451305210097500000E7803D
:10E760006074835521002285814497C0FFFFE780B4
:10E77000A0E125D923100500228597A00000E7809D
:10E7800080CC85B71743FFFFE702E39283C795006C
:10E7900041112A8B93F7F707A384F50032852E8A5F
:10E7A000328497E0FFFFE780C0EA93170501C18735
:10E7B0006351F006AA8A228597E0FFFFE78060E9AF
:10E7C0002A895685832B040097C0FFFFE78020E548
:10E7D00031E58357440081440544F11793B717008E
:10E7E000A301F10003483100DE875A854A87D686A7
:10E7F0002286D28597F0FFFFE78060F6A167ED07DC
:10E8000048003EC42302810026C697F0FFFFE78040
:10E8100020BB41011743FFFF6700638DA2851306EC
:10E82000310097000000E78040B5AA8409445DD913
:10E830009167CA97C2071167C1831307F7EF0544B1
:10E84000E362F7FACA8597C0FFFFE780E0D301448F
:10E8500051F9814997D0FFFFE780C0DC63DBA90055
:10E86000984893971900BA9703D7070005EF2390AC
:10E87000270197D0FFFFE780E0DA1544E384A9F68B
:10E88000268597A00000E78000BC9777FF1F93873D
:10E89000677B9C430144B9D74A8597500000E780C5
:10E8A000005889B785097DB71743FFFFE7028381C9
:10E8B00079713E847C083EC82E8AB7071400A16592
:10E8C0003ECAE5057C08AA89080836C4428932C6D2
:10E8D000BA8AC6843ECC97C0FFFFE78060DFCA8556
:10E8E000080897E0FFFFE78000C732460808B285B6
:10E8F00097E0FFFFE78020C8A246630A09049D4510
:10E90000080897E0FFFFE780C0BE1D4681459730AD
:10E91000FFFFE780C07F63890A089145080897E0F8
:10E92000FFFFE78000BD1146A68597000100E78044
:10E93000A079100801478146D2854E8597C0FFFF18
:10E94000E78060FE45611733FFFF6700E37AB68515
:10E95000080897E0FFFFE78000C21C400808D84382
:10E960009355C701858912075183B205D98D97E068
:10E97000FFFFE78040C01C40080883C5870097E080
:10E98000FFFFE78040BD1C40080883C5A70097E053
:10E99000FFFFE78040BC1C40080883C5970097E054
:10E9A000FFFFE78040BB85BF8945080897E0FFFF70
:10E9B000E78020B483C704002300F50083C7140058
:10E9C000A300F500BDB71733FFFFE702A36F83C7AE
:10E9D00095004111AA8993F7F707A384F5003285C2
:10E9E000AE84328497E0FFFFE780A0C6931705014D
:10E9F000C187635DF0042A89032A040097C0FFFFE2
:10EA0000E780E0C119E9835744000548F11793B73F
:10EA10001700A307F100814631A81306F100A28573
:10EA200097000000E78060951DC51C459DC783D6F3
:10EA3000470001480347F10093078500D2884A86C2
:10EA4000A6854E8597000000E78040E64101173318
:10EA5000FFFF6700636A09487DBF1D486DBF17331C
:10EA6000FFFFE702236665715C083EC4B7077B01C0
:10EA70003EC65C083EC883C795002A8A328593F754
:10EA8000F707A384F500AE8997E0FFFFE78040BA5F
:10EA90008357E100E1C78945280097C0FFFFE78061
:10EAA00020C38145280097E0FFFFE780C0AA97C0F8
:10EAB000FFFFE78000C99787FF1F9387E7909C437C
:10EAC0001774FF1F03448439AA843334800099C328
:10EAD000136424009777FF1F938787409C4399C353
:10EAE000136444009777FF1F9387C7559C4399C3CE
:10EAF0001364840083D504002800014997E0FFFFD8
:10EB0000E78060A783D52400280097E0FFFFE78017
:10EB100080A683D54400280097E0FFFFE780A0A5EA
:10EB200097D0FFFFE78000AB93150501C181280056
:10EB300097E0FFFFE78020A4A285280097E0FFFF71
:10EB4000E78060A39C446360F9020147814630007E
:10EB5000CE85528597C0FFFFE780E0DC596117330F
:10EB6000FFFF67006359DC441314490028003E94FA
:10EB700097E0FFFFE7806096834744000347540017
:10EB800089070607BA978607E36AF5FC83552400D0
:10EB90002800814A97E0FFFFE780E09D834544001D
:10EBA000280097E0FFFFE780009B83455400280082
:10EBB00097E0FFFFE780209A8347440063C9FA008B
:10EBC000814A8347540063C1FA020509A5BF1C446A
:10EBD00013975A002800BA9783D50700850A97E053
:10EBE000FFFFE7804099C9BF032BC40093975A00E9
:10EBF00028003E9B83552B00850A97E0FFFFE780A6
:10EC0000809783550B00280097E0FFFFE780A096D0
:10EC10004DBF1733FFFFE702834C5C4993E71700B2
:10EC20005CC997A00000E78060B51733FFFF67005D
:10EC3000434D1733FFFFE702834A2E84814597F047
:10EC4000FFFFE780C0E705C583570500FD172310C8
:10EC5000F50009C4835725002310F4009700000035
:10EC6000E78060FB01451733FFFF670083493145AB
:10EC70007DD823100400C5BF1733FFFFE70283448C
:10EC800083C7950041112A8A93F7F707A384F500FB
:10EC900032852E89328497E0FFFFE780809B9317AF
:10ECA0000501C1876356F006AA89C145228597E010
:10ECB000FFFFE780A0802A8B4E85832A040097C03F
:10ECC000FFFFE780C09531E983574400231101001D
:10ECD0000544F11793B71700A300F10081440348DE
:10ECE000110003572100D6875285CE862286CA8519
:10ECF00097F0FFFFE780A0A6A1679387170248005F
:10ED00003EC42302810026C697E0FFFFE780406BE8
:10ED100041011733FFFF6700233E13061100A28550
:10ED200097F0FFFFE7806065AA8409E523110100E1
:10ED3000094475B7930521005A8597000000E780C4
:10ED400080EF835721002A84D9DB9777FF1F9387B1
:10ED5000672F9C4381CB8545130521009750000008
:10ED6000E7804014835521002685314497C0FFFF7A
:10ED7000E78080812DD5231005002685979000001F
:10ED8000E780606C0144A1BF1733FFFFE702233522
:10ED900041112E896C00AA8402C697F0FFFFE7801C
:10EDA00000D20DC10357050005072310E5009700A9
:10EDB0000000E78040E681473E8541011733FFFFB1
:10EDC000670023343247954765DBCA85268597302F
:10EDD0000000E780800CC147E34005FE32448547D0
:10EDE00041462310F40083570900A685130544000B
:10EDF0002311F40097000100E780002D228545BF14
:10EE00001733FFFFE702032C83C795004111AA8A3D
:10EE100093F7F707A384F5003285AE89328497E033
:10EE2000FFFFE780008393170501C1876356F00653
:10EE30002A8AC145228597D0FFFFE7802068AA84EF
:10EE40005285032B040097B0FFFFE780407D31E936
:10EE500083574400231101008544F11793B717002D
:10EE6000A300F10001440348110003572100DA8791
:10EE70005685D2862686CE8597F0FFFFE780208EC6
:10EE8000A1679387070248003EC42302910022C66F
:10EE900097E0FFFFE780C05241011733FFFF670093
:10EEA000A325A2851306110097F0FFFFE780E04C31
:10EEB0002A8409E523110100894475B72685930545
:10EEC000210097000000E78060ECAA8449FD83558B
:10EED0002100228597B0FFFFE780006B49F50149CB
:10EEE00097C0FFFFE7800074635DA900184893177F
:10EEF0001900BA9703D707000DEF0357210023909D
:10EF0000E70097C0FFFFE780E0716306250397776E
:10EF1000FF1F938727139C4399C7035521009750E0
:10EF20000000E780C0EF228597900000E780A051A5
:10EF30001DBF050975B795443DB705C19307F00F8F
:10EF4000630FF500C547630CF5009307F5FF054512
:10EF50003315F5004205418182800145828041657B
:10EF60007D158280B9E91733FFFFE7024317034598
:10EF70000603328497000000E78060FC9305803E22
:10EF8000B305B502C205C18181CD0357E4028547AF
:10EF900063F8E7001305040197E00000E780604193
:10EFA0008357E40241677D176385E700FD17231748
:10EFB000F4021733FFFF6700C31482801733FFFF8B
:10EFC000E702630F004283C79500444D03491400D4
:10EFD00093F7F707A384F50083470400220911671C
:10EFE0003369F900A167B347F90041112A8BAE8A52
:10EFF00063ECE70E834724001307C00EB91793F79D
:10F00000F70F6373F71003473400C14763EEE70E51
:10F01000834744001307E00793C707086371F70CA1
:10F020008349840083477400A209B3E9F900856726
:10F0300063F7F90A034A6400834754004E85220AA5
:10F04000336AFA0097500000E780803A61C1239646
:10F050002403834B3400137AFA00239A3403238861
:10F0600074032399440393890401631C090023A6B4
:10F070000402239804024E8597E00000E780A03543
:10F080003DA0034924004A8597000000E78020EB5B
:10F090002397A402834744004E85A388F402E38D9E
:10F0A0000BFCE30B09FC97E00000E780602E9790D3
:10F0B0000000E780407281460146D6855A8597E078
:10F0C000FFFFE7800058A167938797033EC42302A0
:10F0D0000100480002C697E0FFFFE780602E410173
:10F0E0001733FFFF6700A3008544A2862686D685D6
:10F0F0005A8597E0FFFFE780C054A1679387970385
:10F100003EC423029100F1B7BD44C5B79144F1BF9D
:10F110001733FFFFE70203FB01111C08404D3EC2FD
:10F12000B7070F003EC41C083EC62A89AE8997C0A7
:10F13000FFFFE78000D7585C1C5C6346B70E639402
:10F14000E50063E2A70E3385A740B3B7A700B30578
:10F15000B7401306803E81469D8D97000100E780F1
:10F16000C0B693140501C180A1659385C50348000D
:10F1700097B0FFFFE780C0558145480097D0FFFF5B
:10F18000E780603D83550404480097D0FFFFE78087
:10F19000803E83552404480097D0FFFFE780A03DC0
:10F1A000814589CCC167FD179305F00F6388F40092
:10F1B000268597500000E78020E0AA85480097D078
:10F1C000FFFFE780403903554404814501CDC16705
:10F1D000FD179305F00F6307F50097500000E780D7
:10F1E000A0DDAA85480097D0FFFFE780C0368345A1
:10F1F0006404480097D0FFFFE780E035834574043E
:10F20000480097D0FFFFE780003550000147814656
:10F21000CE854A8597B0FFFFE780E0700561173320
:10F22000FFFF670063ED814481B71733FFFFE702FB
:10F2300003EB83C7950093F7F707A384F5009700C6
:10F240000000E78020ED1733FFFF670083EB1733E3
:10F25000FFFFE70223E783C795004111404D93F775
:10F26000F707A384F5002A8A3285B284AE8997D045
:10F27000FFFFE780003E2A8B268597D0FFFFE780BF
:10F28000403D2A89268597D0FFFFE780603A931793
:10F290000B0163CA0702E177CA97C207C1831167EE
:10F2A00063E3E70293070910C207C1831307B00F96
:10F2B000637BF70093170901C187AA8A634AF000AC
:10F2C000C54763FE570141011733FFFF6700C3E2E3
:10F2D00097B0FFFFE7802025E31725FFD5B7630828
:10F2E0000B0263060902814463890A02B7077F00A3
:10F2F00023106405231124057CC056859700000067
:10F30000E780E0C39304803EB304950239A0B707B9
:10F310007F00232004047CC081440355240497E02B
:10F320000000E780E0A2A1C497C0FFFFE78060B7BC
:10F33000269593D7F44133379500AE97BA9708DCFA
:10F340005CDCCE85528597000000E780A0DC99E068
:10F3500023220404A1679387B70348003EC4230215
:10F36000010002C697E0FFFFE7808005A9BF814743
:10F3700001481CDC232E0403E9B71733FFFFE70223
:10F3800003D697C0FFFFE7802034E1473305F5023D
:10F39000914597500000E78040C4E55711C5977725
:10F3A000FF1F23ABA7AA81473E851733FFFF6700E6
:10F3B00043D51733FFFFE70283D29777FF1F938769
:10F3C00067A980433DC0835704046390A706835711
:10F3D0002404639CB7043689B28497C0FFFFE7809A
:10F3E00040AC5C5C63C3B7046395B7001C5C63EE20
:10F3F000A7028347640463F3F400A6872303F4049D
:10F400008347740463F39700A687A303F404835728
:10F41000440441677D176385E70085072312F404E0
:10F420003C4481C7CA85268582971733FFFF670052
:10F4300043CD9777FF1F9387E7A19C43014599C36D
:10F4400003C5870082801733FFFFE70243C901111C
:10F45000B70707003EC683C79500584D0AC493F707
:10F46000F7070AC8A384F5002A89AE8411CB1C4291
:10F4700083C707002304F70097900000E78000345B
:10F48000216493055402280097B0FFFFE7804024D1
:10F4900097000000E78020FAAA85280097D0FFFF98
:10F4A000E780600B300001478146A6854A8597B00A
:10F4B000FFFFE780404713044402480822CC230A98
:10F4C000010002CE97E0FFFFE78080EF0561173370
:10F4D000FFFF670003C31733FFFFE70243C00111BB
:10F4E0007C003ECAB70707003ECC7C003ECE83C7F7
:10F4F00095002E84AA8493F7F707A384F500A165ED
:10F5000093855502480897B0FFFFE780601C97007D
:10F510000000E78040F2AA85480897D0FFFFE78007
:10F520008003500801478146A285268597B0FFFFDA
:10F53000E780603F05611733FFFF670083BC977763
:10F54000FF1F938727919C43094599C303C59700E3
:10F5500082809777FF1F9387E78F9C43094599C364
:10F5600003C5D70082809777FF1F9387A78E9C43A0
:10F57000014599C303C5A70082801733FFFFE70247
:10F5800063B40111B70708003EC683C79500404D1C
:10F590000AC493F7F7070AC8A384F5002A89AE8442
:10F5A00029C41442854703C7060063E0E70A83477E
:10F5B0009400094681496380C702B307F740A3045A
:10F5C000E400B339F00083C716002305F4009790D8
:10F5D0000000E780A01E03572403058B19C763862C
:10F5E000090097D00000E78000E9216493058402B8
:10F5F000280097B0FFFFE780A00D97000000E7808C
:10F6000040F4AA85280097D0FFFFE780C0F4970058
:10F610000000E78080F5AA85280097D0FFFFE780EB
:10F6200080F3014781463000A6854A8597B0FFFFE9
:10F63000E780602F13047402480822CC230A0100DB
:10F6400002CE97E0FFFFE780A0D705611733FFFFE9
:10F65000670083AA1733FFFFE70263A801117C004C
:10F660003ECAB70708003ECC7C003ECE83C795005B
:10F670002E84AA8493F7F707A384F500A1659385E8
:10F680008502480897B0FFFFE780800497000000DC
:10F69000E78020EBAA85480897D0FFFFE780A0EB22
:10F6A00097000000E78060ECAA85480897D0FFFF2C
:10F6B000E78060EA500801478146A285268597B019
:10F6C000FFFFE780402605611733FFFF670063A354
:10F6D0009767FF1F938707789C43014599C303C52C
:10F6E000B70082801733FFFFE702639F0111B7075E
:10F6F00007003EC683C79500404D0AC493F7F7073D
:10F700000AC8A384F5002A89AE8405C81C420547AF
:10F7100083C707006368F7060347B400630FF70069
:10F72000A305F40097900000E78040098347B400E8
:10F73000B9CF97D0FFFFE78000BF21649305B400E5
:10F74000280097B0FFFFE780A0F897000000E7804F
:10F7500060F8AA85280097D0FFFFE780C0DF014747
:10F7600081463000A6854A8597B0FFFFE780A01B41
:10F770002904480822CC230A010002CE97E0FFFFAB
:10F78000E78000C405611733FFFF6700839797D0B8
:10F79000FFFFE780E0BF55B71733FFFFE702239471
:10F7A00001117C003ECAB70707003ECC7C003ECE6C
:10F7B00083C795002E84AA8493F7F707A384F500E6
:10F7C000A165AD05480897B0FFFFE78060F097009E
:10F7D0000000E78020F0AA85480897D0FFFFE78067
:10F7E00080D7500801478146A285268597B0FFFF44
:10F7F000E780601305611733FFFF67008390976709
:10F80000FF1F938727659C43094599C303C5C7001C
:10F8100082801733FFFFE702838C01117C00AE84E6
:10F820003ECAA165B70707002A843ECCD1057C00FB
:10F8300048083ECE97B0FFFFE78080E997000000C0
:10F84000E78020FCAA85480897D0FFFFE780A0D07A
:10F85000500801478146A685228597B0FFFFE780C3
:10F86000800C05611733FFFF6700A3891733FFFF83
:10F87000E702E38683C7950093F7F707A384F500B3
:10F8800097000000E78020F91733FFFF67006387C8
:10F890001733FFFFE702038383C795000329C501E0
:10F8A000411193F7F707A384F5001C4283C90700B1
:10F8B000854763E637079777FF1F9387E7B09C4339
:10F8C0002E84AA8485CF97000000E78080F38947C3
:10F8D0006306F502630409028347C90063803703A6
:10F8E0002306390197900000E78040ED83572903F4
:10F8F000898B89C797D00000E780E0B72685A2856D
:10F9000097000000E78020F1A167CD0748003EC4C2
:10F910002302010002C697E0FFFFE78060AA4101D1
:10F920001723FFFF6700437D9767FF1F9387875269
:10F930009C431D4599C303C5E70082801723FFFF41
:10F94000E702E3790111B70707003EC683C79500B8
:10F95000584D0AC493F7F7070AC8A384F5002A890B
:10F96000AE8415C71C4283C7070093968701E186C2
:10F9700063C4060685466381D7068346E70063882D
:10F98000F6002307F70097900000E78020E321644A
:10F990009305E400280097B0FFFFE78060D397004D
:10F9A0000000E780A0F8AA85280097D0FFFFE78035
:10F9B00080BA014781463000A6854A8597B0FFFF8F
:10F9C000E78060F63504480822CC230A010002CE05
:10F9D00097E0FFFFE780C09E05611723FFFF6700E8
:10F9E00043721723FFFFE702836F01117C003ECAB9
:10F9F000B70707003ECC7C003ECE83C795002E841F
:10FA0000AA8493F7F707A384F500A165B905480810
:10FA100097B0FFFFE780C0CB97000000E78000F1C0
:10FA2000AA85480897D0FFFFE780E0B25008014759
:10FA30008146A285268597B0FFFFE780C0EE05616D
:10FA40001723FFFF6700E36B1723FFFFE7028367BE
:10FA5000AA8401441769FF1F13090940E14997C0AF
:10FA6000FFFFE78060C66344A400014519A8330581
:10FA70003403832709003E95835725006397970039
:10FA800011051723FFFF670023670504C9BF032E75
:10FA90008500630A0E121763FF1F1303A35A032383
:10FAA00003006315030029436390061203234E01EC
:10FAB000631503001D43639907101723FFFFE70237
:10FAC000835FC689428A3E89BA8AB684328BAE8BFE
:10FAD0002A84B5E103554E0019E501431A85172321
:10FAE000FFFF6700C360A167A98F116763FBE70091
:10FAF00097000000E78080F5814597F0FFFFE780E1
:10FB000080130844B70700E05841F98F18455CC1DD
:10FB1000B707001FF98F1CC55C4991C7610597E0C5
:10FB20000000E780408BE38A09FA22859790000065
:10FB3000E78060C65DB7328597C00000E78040432C
:10FB40000D4349DD1C44116703D54700A167A98F08
:10FB500063FBE70097000000E78040EF814597F0E6
:10FB6000FFFFE780400D0323840093164B01D182F1
:10FB70008347B300035663008588FD8BA305F3001C
:10FB8000FD777D8E558EFD76FD16B204F18E8327AE
:10FB90004301C58E231273012313D30023045301A1
:10FBA00023052301A3044301BDDF228597B0FFFF96
:10FBB000E78040CAAA850844B5D1610597D0000006
:10FBC000E780207F8DB71D431A8582801723FFFFB2
:10FBD000E702434F0569AA84AE89328A0144FD5A7F
:10FBE0007D1997C0FFFFE780E0A26347A4000145AD
:10FBF0001723FFFF67004350D84493171400BA97A8
:10FC000003D70700631F37032390570163070A00D8
:10FC1000268597900000E780A0809C449DC383D7F1
:10FC20006700B3F72701639E3701D28801488147F7
:10FC30000147814601468145268597000000E780FF
:10FC400040E5050479BF1723FFFFE702A347797159
:10FC50001C103EC4B7070F003EC61C103EC883C729
:10FC60009500AA8A328593F7F707A384F5002E89B9
:10FC7000328497D0FFFFE780C09D93170501C187AD
:10FC8000635AF006AA89228597D0FFFFE780609C1F
:10FC90002A8A4E85032B040097B0FFFFE780209847
:10FCA00039ED8357440081440544F11793B7170099
:10FCB000A303F10083457100DA872287D2864E863E
:10FCC000280097E0FFFFE780A058014781463000F9
:10FCD000CA85568597B0FFFFE780E0C4A167938788
:10FCE000F70348083ECC230A810026CE97D0FFFFB9
:10FCF000E780006D45611723FFFF6700E33FA285A2
:10FD00001306710097E0FFFFE7802067AA8409448B
:10FD100055D1528597E0FFFFE78020D50D4459D992
:10FD20000546D285268597000000E78060EA2A8490
:10FD300051B71723FFFFE702833A835507000346B5
:10FD4000270041112A842E8532C62EC497E0FFFF7A
:10FD5000E780A0D101C93246A24522859700000064
:10FD6000E78000E741011723FFFF6700833917236E
:10FD7000FFFFE702433483C795004111AA8A93F736
:10FD8000F707A384F5003285AE89328497D0FFFF50
:10FD9000E780208C93170501C1876357F00AC1459E
:10FDA0002A8A228597C0FFFFE78040712A8D22852D
:10FDB00097D0FFFFE780E0892A89228597D0FFFF4F
:10FDC000E7800087930705F893F7F70F1307E0071D
:10FDD000AA8B637BF706228597D0FFFFE7804085DB
:10FDE0002A8C228597D0FFFFE7808084AA8C5285D9
:10FDF000032B040097B0FFFFE780608239E9835747
:10FE00004400231101008144F11793B71700A300A8
:10FE1000F1000544034711008356210093878400B5
:10FE20005685DA8822885286CE8597F0FFFFE780D4
:10FE3000E0A7A167E90748003EC42302810026C667
:10FE400097D0FFFFE780C05741011723FFFF6700EE
:10FE5000032A13061100A28597E0FFFFE780E05117
:10FE6000AA8409E52311010009446DB79305210017
:10FE70006A8597F0FFFFE78060F12A8441FD835592
:10FE800021009356C9001316490185486688E28708
:10FE90005E87858A5182268597000000E78060BFD3
:10FEA0002A848DBF1723FFFFE702E32083C7950055
:10FEB00041112A8B93F7F707A384F5003285AE89A9
:10FEC000328497C0FFFFE780C07893170501C18790
:10FED0006352F00A2A8A228597C0FFFFE780607785
:10FEE000AA8A228597C0FFFFE780A0762A8922850B
:10FEF00097C0FFFFE780C073930705F893F7F70FEC
:10FF00001307E0072A8C6377F706228597C0FFFF67
:10FF1000E7800072AA8C228597C0FFFFE7804071BE
:10FF20002A8D5285832B040097A0FFFFE780206F66
:10FF300039E58357440085440144F11793B717000E
:10FF4000A301F10003473100930784005A85DE883E
:10FF50002688D6865286CE8597F0FFFFE7800095EB
:10FF60008D4748003EC42302910022C697D0FFFF70
:10FF7000E780004541011723FFFF67004317A28573
:10FF80001306310097E0FFFFE780203F2A84894471
:10FF900055D99356C9001316490185486A88E687E2
:10FFA0006287858A5182D68597000000E78060AE1F
:10FFB000AA8449BF1723FFFFE702C3102A8981449F
:10FFC0000144617A916A176BFF1F130BAB0797B05F
:10FFD000FFFFE780206563C7A40022851723FFFF8A
:10FFE000670083118327090093991400CE9703D5E6
:10FFF000070033074501420741836364570305C186
:020000040001F9
:1000000003270B0019C785453E8597400000E78010
:1000100060E9832709000504CE9723900700850433
:100020007DB797000000E78060A2832709000504E0
:10003000CE972390070065D5814597F0FFFFE780B5
:1000400080BFF1BF1723FFFFE702C30783C79500F7
:1000500041112A8A93F7F707A384F50032852E8988
:10006000328497C0FFFFE780C05E93170501C18708
:10007000635AF004AA89832A040097A0FFFFE7804F
:10008000005A31E58357440085440144F11793B782
:100090001700A301F10003483100D68752850147BC
:1000A000CE862686CA8597D0FFFFE780406BA16782
:1000B000F50748003EC42302910022C697D0FFFFF7
:1000C000E780003041011723FFFF6700E302A285AC
:1000D0001306310097E0FFFFE780202A2A84894435
:1000E0005DD99767FF1F9387E7F59C4381CF04494C
:1000F00097B0FFFFE7800053AA8526859740000050
:10010000E78040DA1305040197000000E780C0EAA9
:10011000228597800000E78000338144ADBF17231C
:10012000FFFFE70243F983C795004111AA8A93F7BD
:10013000F707A384F5003285AE89328423110100CC
:1001400097C0FFFFE780E05093170501C187635414
:10015000F0062A8AC145228597C0FFFFE780003656
:10016000AA8B5285032B040097A0FFFFE780204B4A
:1001700021E98357440085440144F11793B71700E0
:10018000A300F1000348110003572100DA875685C8
:10019000D2862686CE8597D0FFFFE780405CA16798
:1001A0009387270248003EC42302910022C697D0BD
:1001B000FFFFE780E02041011723FFFF670023F3E3
:1001C000A2851306110097E0FFFFE780001B2A8439
:1001D00089444DD99767FF1F9387C7E698433E89A7
:1001E00001CF044997B0FFFFE780C043AA85268569
:1001F00097400000E78000CB130504019700000042
:10020000E78080DB97B0FFFFE780C04195443DD990
:10021000930521005E8597F0FFFFE78020B7AA8451
:1002200035F11C480357210022852390E700978071
:100230000000E780402183270900A9D7035521004A
:1002400097400000E780A0BD35BF1723FFFFE702FE
:1002500083E683C795004111AA8A93F7F707A38421
:10026000F5003285AE89328497C0FFFFE780603E9B
:1002700093170501C1876351F0062A8A228597C02A
:10028000FFFFE780003D2A895285032B040097A0D9
:10029000FFFFE780C03831E58357440085440144BF
:1002A000F11793B71700A301F10003483100DA8773
:1002B00056854A87D2862686CE8597D0FFFFE7806F
:1002C000004AA167F90748003EC42302910022C6F4
:1002D00097D0FFFFE780C00E41011723FFFF6700A3
:1002E00003E1A2851306310097E0FFFFE780E008F5
:1002F0002A8489445DD99167CA97C2071167C1836F
:100300001307F7EF8544E362F7FA9767FF1F9387B8
:1003100067D39843BE8B01CF044997B0FFFFE780B6
:100320006030AA85268597400000E780A0B71305B6
:10033000040197000000E78020C897B0FFFFE78026
:10034000602E95443DD11C4822858144239027018D
:1003500097800000E780200F83A70B00B9D74A855C
:1003600097400000E780A0AB89B71723FFFFE702A3
:1003700003D72A844105B28497000000E780C0C3F8
:1003800011C5228597800000E780E00B8146014679
:10039000A685228597800000E780C04E1C4C89C747
:1003A000DC4799C3228582971723FFFF670063D537
:1003B0009767FF1F938707AA9C43014599C313853D
:1003C000070182809767FF1F9387C7A888438280B1
:1003D0001723FFFFE702A3D09317C600DD8DC205E8
:1003E0004111C1812A8432C697C0FFFFE780A0185F
:1003F0003246228511829375F60F97C0FFFFE78082
:10040000801541011723FFFF6700A3CF1723FFFFCC
:10041000E70243CB79713C083ED2B7070C003ED4CB
:100420003C083ED683C79500AE842A8993F7F70728
:10043000A384F500A16593853504481097A0FFFFBC
:10044000E7800029C165FD150144176AFF1F130AE3
:10045000EAC0930A400EAE892E8B2EC697B0FFFFDE
:10046000E780401F4205931704014181C183B245D3
:1004700063E9A702C167FD176387F500481097C0BD
:10048000FFFFE780400F501001478146A6854A854F
:1004900097A0FFFFE780204945611723FFFF670012
:1004A000A3C53307540383270A0BBA9703D6C701A2
:1004B000630A3601638A3501481097000000E7801F
:1004C00060F1DA85050451BFB285EDBF1723FFFF48
:1004D000E70263BE79717C083EC8B70711003ECAC7
:1004E0007C083ECC83C79500AA89328593F7F7072D
:1004F000A384F5002E8997C0FFFFE78080158567EC
:100500006378F504A165AA848905080897A0FFFF10
:10051000E780001C268597400000E78060ED1334DB
:1005200015000A04A285080897C0FFFFE780A00213
:10053000A685080897C0FFFFE780E00325CC0147A8
:1005400081461008CA854E8597A0FFFFE780A03D31
:1005500045611723FFFF670083B9B30754030327DF
:10056000CA0ABA9703D70700631C970003D627006F
:1005700063806505080897000000E780A0E5DE8538
:1005800005042EC697B0FFFFE780C00D4205931704
:1005900004014181C183B245E3E1A7FCC167FD17B6
:1005A000E38FF5F8080897C0FFFFE780C0FC41BF64
:1005B000B285F9B7C165FD150144176AFF1F130A1B
:1005C000EAA9930A80022E8BAE8B65BF1723FFFF2B
:1005D000E702E3B018418347170083460700A207EC
:1005E000D58FD207D1832390F50083472700034797
:1005F00017008D45A207D98F91832310F60097C06D
:10060000FFFFE78060EA1723FFFF670083AF172330
:10061000FFFFE70223ABC16401441769FF1F130901
:10062000E9A393098002FD1497B0FFFFE7808003E0
:100630006347A40001451723FFFF6700E3AB3305C1
:1006400034038327C90A3E9583570500E38597FE47
:100650000504D9BF1723FFFFE702C3A62A8AAE8984
:10066000B284B68A97400000E78080D819E59147A8
:100670003E851723FFFF670023A82A894E8597C070
:100680000000E780E08E2A84638E0A048D476DD1D6
:1006900003570500C547E31D47FD0347F90185469C
:1006A000AD47E317D7FC8347450081CF4146A68578
:1006B0005D0597F00000E780C09E814755D9AD47A2
:1006C00045BF130965012302E500CA8526859710F9
:1006D0000000E780606231C1A547E38B0AF823027E
:1006E000040079B705C183570500E39247F94146F5
:1006F000A685190597F00000E780A09A81472DD9BB
:100700009947BDB74E8597000000E78080F02A84A6
:10071000954739DD130955004DBF4146A685231085
:100720004401231134011305190097F00000E780FC
:10073000A099228597800000E780A0EA81470DBF3D
:100740001723FFFFE702A39979717C003ECCB7071E
:100750000A003ECE7C003ED083C79500B2842E8432
:1007600093F7F707A384F5001306A1002A892C004C
:10077000268597000000E780A0E5A16528088D0583
:1007800097A0FFFFE780C0F490408355A100035578
:100790008100854697000000E78000ECAA84AA85C6
:1007A000280897C0FFFFE78000DB0356A1008355B0
:1007B0008100280897000000E780C0C13008014789
:1007C0008146A2854A8597A0FFFFE780C01585472F
:1007D00048103ED42302910202D697D0FFFFE78053
:1007E00020BE45611723FFFF6700A3911723FFFF7A
:1007F000E702E38E79717C003ECCB7070A003ECE5B
:100800007C003ED083C79500B2842E8493F7F7070F
:10081000A384F5001306A1002A892C0026859700E1
:100820000000E780E0DAA16528088D0597A0FFFFAA
:10083000E78000EA90408355A1000355810081467E
:1008400097000000E78040E1AA84AA85280897C0A5
:10085000FFFFE78040D00356A100835581002808A0
:1008600097000000E78000B7300801478146A28565
:100870004A8597A0FFFFE780000B481023029102F2
:1008800002D402D697D0FFFFE78080B345611723DB
:10089000FFFF670003871723FFFFE70243849700EA
:1008A0000000E78060DB1723FFFF67008385975711
:1008B000FF1F9387675A884382801723FFFFE70251
:1008C0000382835725004111AE842A842307B10097
:1008D00017F5FFFF130525466C002316F10097A0BE
:1008E000FFFFE780404691C4228597800000E780A3
:1008F000E0D6FD572310F4001306200281451305AE
:1009000054009720FFFFE780808041011713FFFF0D
:100910006700237F1713FFFFE702C37A79717C001A
:100920003ECCB7070A003ECE7C003ED083C7950080
:10093000AA89AE8493F7F7073285A384F5001306DE
:10094000A1002C0097000000E78080C803558100BB
:10095000114497400000E780A0A915C50355A100E8
:10096000014497B00000E780A06011CD0357050057
:100970008357810045446318F700854597000000C0
:10098000E780E0F30144216993053900280897A026
:10099000FFFFE780E0D3A285280897C0FFFFE7802C
:1009A00080BB0356A10083558100280897000000F2
:1009B000E78040A2300801478146A6854E8597A072
:1009C000FFFFE78040F648104AD42302810202D696
:1009D00097D0FFFFE780C09E45611713FFFF6700B8
:1009E000A3711713FFFFE702E36D9757FF1F93876C
:1009F00067462A8488432E8915C5035745038357C4
:100A0000C4016311F70223260502231805024105DC
:100A100097D00000E780209C6306090097800000C3
:100A2000E78060DB81449759FF1F93892963130A8C
:100A3000800297B0FFFFE780E0C263C4A404975729
:100A4000FF1F9387E7499C4399C70355C40197202B
:100A50000000E780C0BD6307090022859780000081
:100A6000E780C0A01306400E814522859710FFFF46
:100A7000E780E069FD57231EF4001713FFFF6700AE
:100A8000A3673385440383A7C90A3E95035705002E
:100A90008357C4016317F700CA8597000000E780F9
:100AA00000E2850479B71713FFFFE702A36183C74C
:100AB00095004111AA8993F7F707A384F5003285C1
:100AC000AE8497C0FFFFE780C0B885676378F50400
:100AD0002A8997400000E780A091014401CD83D787
:100AE0000400314463882701854597000000E780B2
:100AF00080EF01444E85A2864A86A68597D0FFFFE7
:100B0000E780609DA1679387170448003EC42302D5
:100B1000810002C697D0FFFFE780808A410117134A
:100B2000FFFF6700635D1713FFFFE702A3599757A5
:100B3000FF1F93872732804329C4014597C00000D7
:100B4000E780002181470148C1641CDC232E040397
:100B5000232004041759FF1F130949500144930926
:100B6000400EFD1497B0FFFFE780C0AE634FA400B6
:100B7000814517F5FFFF1305857F97A0FFFFE780ED
:100B8000801C1713FFFF67002357330534038327A7
:100B9000090B3E958357C5016387970085459700EC
:100BA0000000E78040E4050475BF9357050113D7A3
:100BB0008700A380F50093170501C183A1832380DB
:100BC000E5002381F500A381A50082801713FFFFB4
:100BD000E702E3502300050083C71500A300F500DA
:100BE00083C725002301F50083C73500A301F50065
:100BF00083C745002302F50083C75500A302F50013
:100C000083C7650093059500A30305002303F50042
:100C100023040500328597000000E78040F9171390
:100C2000FFFF6700034E1713FFFFE702A3494111BF
:100C3000E9540DCD85CD93F9C5FF2E842A89AA8468
:100C4000338AA900B7EA040063189A020D88854424
:100C500011CCB7E704009C5F82972AC622866C00FD
:100C60003305390197E00000E78000462685410101
:100C70001713FFFF6700434883A78A0391048297F5
:100C800093170501C183A183A38EF4FE9357050139
:100C9000238FF4FEA183238EA4FEA38FF4FE6DB7F1
:100CA00063E6D5021713FFFFE7026343B2874111E2
:100CB0003686BE8536C697E00000E780E040B24643
:100CC000410136851713FFFF6700A3438146368530
:100CD0008280838705001387F5003D05FD8793F724
:100CE0007708834607007D158606B58FA300F500BB
:100CF0006307B7007D17834717009D83DDB78280A8
:100D00001713FFFFE702A33DB7E7040083A7070916
:100D100032872A863A858297133515001713FFFF0D
:100D20006700233E15C181478DC11713FFFFE702FE
:100D3000033B414697E00000E780003985473E8548
:100D40001713FFFF6700E33B81473E8582801DCD7F
:100D50001713FFFFE702A338414681452A84971005
:100D6000FFFFE780C03A4146814513050403971011
:100D7000FFFFE780C0390147C1672322040438C858
:100D80007CC805451713FFFF6700A3370145828024
:100D900081473DCDB5CD1713FFFFE7024334B28441
:100DA0002E891306800581452A849710FFFFE7806E
:100DB0000036CA8524C4268597000000E780C0F667
:100DC0004146814522859710FFFFE780403430443B
:100DD000A285228597000000E780C0F293040401F9
:100DE000A285268597000000E780E0EEA685130522
:100DF000040297000000E78000EE228597000000C3
:100E0000E78020F585473E851713FFFF6700632FB6
:100E10003E8582801713FFFFE702C32A4111E95480
:100E20000DCD85CD93F9C5FF2E842A89AA84338AF6
:100E3000A900B7EA0400639844030D88814411CCEB
:100E4000B7E704009C5F82972AC622866C003305B0
:100E5000390197E00000E78020272685410117131C
:100E6000FFFF6700632983A78A0391048297931782
:100E70000501C183A183A38EF4FE93570501238F3F
:100E8000F4FEA183238EA4FEA38FF4FE6DB765CD7F
:100E90001713FFFFE7020323B28411E6054517137A
:100EA000FFFF670063252A842E890145EDD93C4860
:100EB0007848B3E6E700E5D69386F7FFB3B7F600C8
:100EC0007D17032A4404BA9734C87CC863050A0610
:100ED000C14913050A03B38949412295637D36014F
:100EE000B2862E86A68597000000E780A0DB7C40B6
:100EF000BE9464C065B7CE862E86CE85970000006E
:100F0000E78040DAC114D2944E9923220404A287C8
:100F10009306040103C7070003C607038507318F43
:100F2000A38FE7FEE398F6FE3044A2852285970062
:100F30000000E78020DD2699C1493306994063EC23
:100F40009900A9DCA686A685130504039700000076
:100F5000E78040D579BF8147B306F4003307F60038
:100F60000347070083C5060085072D8F2380E60011
:100F7000E39437FF3044A285228597000000E78084
:100F800060D8C1145DBF014582800DC11713FFFFFA
:100F9000E702E3141306800581459710FFFFE78001
:100FA000001705451713FFFF6700A3150145828051
:100FB000814749C5C1C51713FFFFE7024312FC4132
:100FC00041462E84AA846399C70413860501A2872B
:100FD0008146C14503C7070003C507038507298F5D
:100FE0003305D600034505008506298FA38FE7FE4C
:100FF000E392B6FE3044A285268597000000E78084
:1010000060D0228597000000E78060F885473E8524
:101010001713FFFF6700E30E138507031D8E81453D
:1010200022959710FFFFE780800E7C40130700F8A1
:1010300013060402A2972388E70251BF3E858280EF
:101040001713FFFFE702A3096D712E84B284AA85EE
:1010500090102800368997000000E780A0D309EDA2
:10106000D55725A050400C40280097000000E7808D
:1010700040E27DD5FD142104F5F42C004A8597004B
:101080000000E78020F3814761DD3E855161171341
:10109000FFFF670003071713FFFFE7024304411137
:1010A0002EC432C62C00054697000000E78080F968
:1010B00041011713FFFF6700C3041713FFFFE70287
:1010C000030201112A842EC602C802CA02CC02CE33
:1010D00097E00000E780C023B2462A86A285080870
:1010E00097000000E78060FB1375F50F056117138B
:1010F000FFFF670003011713FFFFE70243FE79714B
:10110000B2872A8421462308B10013051101BE8548
:101110003AC436C697E00000E78000FBB24693056C
:101120009101368597000000E78060A822851410A1
:1011300035460C0897000000E78020F62A842247F5
:1011400001E921460C103A8597E00000E780C0F7DE
:10115000228545611713FFFF6700A3FA1713FFFFEE
:10116000E702E3F77171AE84AA850A85328497009D
:101170000000E78060BB11C90A86A685228597001A
:101180000000E78020B8814711E1C5473E854D61E9
:101190001713FFFF6700E3F61713FFFFE70223F1C2
:1011A0001D712A8AB289BE8435468547130511010F
:1011B0002E8CB68A3A8BC28C468D2308F10097E0BC
:1011C0000000E78060F010100C085285231F01001A
:1011D00097000000E780C0F82A843DEDA147631323
:1011E000FD089307900591E0E5473546E285130534
:1011F000110113990A012308F1001359090197E01D
:101200000000E78060EC1357890093978A00D98F1C
:1012100090080C085285231FF10097000000E7801A
:1012200020F42A8415E9A1E49387FA0091831379C5
:10123000F9003EC6631309004149668B8144C14BE6
:10124000854DB247639F970C6A868C0033855C019D
:1012500097E00000E78040E7228525611713FFFF34
:101260006700A3E893079004C9F0A547BDBF834773
:1012700001050947C14B2308F10083471105A58FDC
:10128000A308F10093872400814463E1FB04014734
:1012900014083386E6008C08B386E400BA95DA9623
:1012A00083C6060083C505000507AD8E2300D60062
:1012B000E390E7FE4147639CE70490080C085285E1
:1012C00097000000E780C0E925D181A0B3069B000C
:1012D000BA871008B305F60090083E9603C50600CD
:1012E0000346060085078506298E2380C500E39204
:1012F00077FF998F90080C085285BE9497000000E4
:10130000E78000E68947014749D12A84B1B79008B0
:101310003E96034606001408BE962380C600850745
:1013200059BFB24785046387971481471808B306ED
:10133000F70098083E973386F900034707000346F5
:1013400006008507318F2380E600E39177FF900840
:101350000C08528597000000E78080E05DF5354677
:10136000E285130511012308B10197E00000E78031
:10137000A0D5139704014183939784002183D98FCB
:1013800010180C085285231FF10097000000E78019
:1013900020DD25FD814710183387F9003E9603476D
:1013A000070003460600B306FB008507318F238044
:1013B000E600E39277FF65A81808B306F7009808DF
:1013C0003E973386F900034707000346060085076A
:1013D000318F2380E600E3E127FFCA87639E770908
:1013E00090080C08528597000000E78060D711FD37
:1013F00081479800B306F700900818103E973E9674
:1014000003470700034606008507318F2380E60067
:10141000E39177FF3546E285130511012308B101F9
:1014200097E00000E78040CA139704014183939737
:1014300084002183D98F10180C085285231FF100D6
:1014400097000000E780C0D1E31105EC8147101838
:101450003387F9003E960347070003460600B306AC
:10146000FB008507318F2380E600E3E227FFC109F7
:10147000410BC1BB814785B79408BE9683C6060061
:1014800018083E972300D700850789BF638006327E
:101490001713FFFFE702A3C159712A84BE89B28BDB
:1014A00085473546130511022E8B468C4289BA8A30
:1014B000368A2300F10297E00000E780E0C01018B0
:1014C0000C1022852317010297000000E78040C915
:1014D00063180512A147631FFC06930790056393E9
:1014E0000900E5473546DA851305110293140A0110
:1014F0002300F102C18097E00000E780E0BC931771
:101500008A0013D78400D98F90080C1022852317E6
:10151000F10297000000E780A0C47DE16392090416
:101520009307FA00BD88918391E0C144C207C1834B
:10153000DE8C814A3EC6414DB24763E2FA0E6286B6
:10154000B3854B01881097E00000E78080B54DC956
:101550003D557DA093079004E39609F8A54759B738
:10156000834701050947C14C2300F1028347110558
:10157000B3C7F900A300F10293872900814963E111
:10158000FC04814618103306D7008C083387D90035
:10159000B69556970347070083C5050085062D8F2E
:1015A0002300E600E390D7FE41476390E7069008EA
:1015B0000C10228597000000E78080BA35D189A001
:1015C000B3863A01BA871010B305F60090083E962C
:1015D00003C506000346060085078506298E23807D
:1015E000C500E39297FF3387EC4090080C102285EA
:1015F000BA9997000000E780A0B68947014741D11A
:1016000065611713FFFF670043AE90083E960346DF
:1016100006001410BE962380C600850779B7B2472E
:10162000850A93990A01939D8A0093D909016391D0
:10163000570F85473546DA85130511022300F1025D
:1016400093D9890097E00000E78000A8B3ED3D0141
:1016500090000C1022852317B10397000000E7804B
:1016600020B059FD8147A68963EA970626860C08B3
:101670004A8597E00000E78020A581471810B3064F
:10168000F700100898083E973E9603470700034668
:1016900006008507318F2380E600E3E197FE639F14
:1016A000A90590080C10228597000000E78040AB48
:1016B00021F981479810B306F700900818183E9753
:1016C0003E9603470700034606008507318F2380B7
:1016D000E600E391A7FF4109C10CB9BD18089000CD
:1016E000B306F7003E963387FC0003470700034626
:1016F00006008507318F2380E600B5B798084E971E
:10170000034707001C10CE972380E700850941BFDF
:1017100085473546DA85130511022300F10293D976
:10172000890097E00000E780209AB3ED3D0190002A
:101730000C1022852317B10397000000E78040A218
:10174000E31005EC814718089000B306F7003E96B9
:101750003387FC0003470700034606008507318FE7
:101760002380E600E391A7FF41460C084A8597E0F5
:101770000000E780609581471810B306F700100855
:1017800098083E973E9603470700034606008507E4
:10179000318F2380E600E391A7FF90080C1022858B
:1017A00097000000E780C09B1DD599BD7D558280C4
:1017B0001713FFFFE702A39201112A842E859305D8
:1017C0005100328902C002C202C402C693047400EE
:1017D00097F0FFFFE780A03D1D46A6851305910009
:1017E00097E00000E780408E10088A854A859700C0
:1017F0000000E780E09619ED93071400180883C6EF
:1018000007000346070085070507B18EA38FD7FEA3
:10181000E397F4FE05611713FFFF6700838E17132C
:10182000FFFFE702238A2E848C414111AA89838716
:1018300015003289914463D30700A1449757FF1FD5
:10184000938787B89C43A1C7C1CA8D472310F10075
:1018500083C725004A852301F10083C73500A30112
:10186000F10083C745002302F10083C75500A3029E
:10187000F10083C7650093059100A30301002303D2
:10188000F1002304010097F0FFFFE78040320C4095
:101890004A860A8597F0FFFFE7808033032804001B
:1018A00083564400A6881D0881470147E5164286F5
:1018B0008A854E8597000000E780408E2A8919E5C9
:1018C000A685228597B0FFFFE780A0C24A85410127
:1018D0001713FFFF670043824A860A8597F0FFFFD0
:1018E000E780002F6DB71703FFFFE702A37D2E846B
:1018F0008C414111AA89838715003289914463D3B1
:101900000700A1449757FF1F938707AC9C43A1C7CB
:10191000C1C68D472310F10083C725004A852301E6
:10192000F10083C73500A301F10083C745002302FE
:10193000F10083C75500A302F10083C7650093053A
:101940009100A30301002303F1002304010097F099
:10195000FFFFE780C0250C404A860A8597F0FFFF0D
:10196000E780002783564400032804008A85858E7B
:10197000C2061D08C1822312D400A68881470147F0
:10198000E51642864E8597000000E78060B0410171
:101990001703FFFF670043764A860A8597F0FFFF2B
:1019A000E78000234DBF1703FFFFE7024373B33502
:1019B000B000011185052A891315F601336515015B
:1019C0002308B1009305110136843AC632C03EC4E3
:1019D00042C297F0FFFFE780801DA24712484255A0
:1019E00093D68700230BF10093059101935788004C
:1019F000A30AD100A30BF100230C010197F0FFFF14
:101A0000E780E01A3247024603280400B337E000BB
:101A1000835644009207914411C2A1444A85A68886
:101A200042860C0897F0FFFFE78040772A8919E586
:101A3000A685228597B0FFFFE780A0AB4A850561A8
:101A40001703FFFF6700E36B1703FFFFE7028367DE
:101A500001113EC68647B335B0008505AA89131526
:101A6000F6015D8D2308B1009305110136843A8992
:101A7000B28442C446C297F0FFFFE7804013224879
:101A80009248164593578800A30AF10093059101E7
:101A900093D78800230B0101A30BF100230C110144
:101AA00097F0FFFFE780A0103247104083564400B4
:101AB000B337E000920703280900914891C0A1487C
:101AC0000C084E8597000000E780809CAA8401E9FD
:101AD000835544004A8597B0FFFFE78080A12685A3
:101AE00005611703FFFF67002361AA959307F00FB5
:101AF00017070100130747656317B50013C5F7FF04
:101B00001375F50F828005058346F5FFB58FBA97EB
:101B100083C70700D5B70357450014419307F00F5B
:101B20001706010013064662369742074183139554
:101B300006014181631BE500AD8FB29703C5070025
:101B4000130515F3133515008280850603C5F6FFCE
:101B5000A98FB29783C70700D9BF1703FFFFE7021A
:101B60000358B28736842E86BA86AA853E85BA8403
:101B700097F0FFFFE7806052634F0500228597D002
:101B80000000E780E0782A86A686A285268597F061
:101B9000FFFFE78080501703FFFF6700835617039E
:101BA000FFFFE70223525D712A8BAE8A1705010001
:101BB000130505572C00B284368ABA893E8997F0FE
:101BC000FFFFE780C04F2A845DE134104146DA858B
:101BD000280097F0FFFFE780404C2A8449E98547B9
:101BE000A303F100A6C2930771002408BEC4A68611
:101BF00085470D462C18281002DC02DED6C0BEC672
:101C000097F0FFFFE78000442A8435E183477102A3
:101C1000A6860D4693F7F7072300FA00C1473EDE7C
:101C20002C188947281026DCA303F10097F0FFFF4A
:101C3000E78040412A8405ED4146A6854E8597D030
:101C40000000E78060488D47A6860D462C182810B6
:101C5000A303F10097F0FFFFE780C03E2A8401E96B
:101C60004146A6854A8597D00000E780E045228559
:101C700061611703FFFF670023481703FFFFE702B7
:101C8000034697F700009387A7A1984383C74700AF
:101C900079712A89AE84170501001305E5480C08FF
:101CA0003AC42306F10097F0FFFFE78040412A8401
:101CB00005ED14104146CA85080897F0FFFFE7803C
:101CC000C03D2A8415E1140815462C00081097F031
:101CD000FFFFE780803C2A8401E921462C08268505
:101CE00097D00000E780403E228545611703FFFF43
:101CF000670023411703FFFFE702633E97F70000E9
:101D00009387079A9C477971AA842E84170501004E
:101D1000130505420C083EC697F0FFFFE780203A06
:101D20000DE914104146A685080897F0FFFFE780EB
:101D3000C03605E1140811466C00081097F0FFFF4B
:101D4000E780A03519E58347F10193F7F7032300F6
:101D5000F40045611703FFFF6700A33A1703FFFF75
:101D6000E702E3373688A14881470147E54697F007
:101D7000FFFFE780A0421703FFFF670083381703C8
:101D8000FFFFE702C3353688A14881470147E54692
:101D900097F0FFFFE780C06F1703FFFF6700633610
:101DA0001703FFFFE702A33301112A842E850C08D5
:101DB00032C697F0FFFFE780803009ED3247970683
:101DC0000100938666351008C14522859700000002
:101DD000E780E0D805611703FFFF67008332170330
:101DE000FFFFE702C32F4111C1472EC032C48A85CD
:101DF00009463EC23EC697F0FFFFE780A02441019E
:101E00001703FFFF6700E32F1703FFFFE702232DF0
:101E10004111AE8613061009AA850A8502C002C2C6
:101E200002C402C697F0FFFFE78020274101170395
:101E3000FFFF6700032D1703FFFFE702432A3287E6
:101E4000970601009386462F2E8693050002970081
:101E50000000E780C0D01703FFFF6700832A170345
:101E6000FFFFE702C3277971C1472ACC2ED032D4B5
:101E70002C080D4628003ECE3ED23ED602C402C6F5
:101E800002C802CA97F0FFFFE780C01B4561170335
:101E9000FFFF670003271703FFFFE7024324011139
:101EA000AA842E8417050100130585298A8597F0D9
:101EB000FFFFE780C02015E514084146A6850A8586
:101EC00097F0FFFFE780601D09ED8347E1010347BD
:101ED000F101A207D98FCA07C9836177D98F23106F
:101EE000F40005611703FFFF6700A32115CD170359
:101EF000FFFFE702C31E9747FF1F938767FA9043D0
:101F00009745FF1F938505FA1745FF1F130545F5F4
:101F100097D00000E78000C51745FF1F130545F463
:101F20001703FFFF6700E31D1745FF1F130545F368
:101F300082808DCD1703FFFFE702631A9747FF1FCB
:101F4000938707F6944301112E840A869745FF1F55
:101F5000938545F597D00000E78040C60A85029436
:101F6000014505611703FFFF6700A3197D558280B6
:101F70001703FFFFE702A31697D00000E78080D188
:101F80009747FF1F23AEA7F017F5FFFF1305E5C91D
:101F900097B00000E780C0741703FFFF6700631667
:101FA0001747FF1F130707F29317150008433E95C5
:101FB000FD572310F50082801703FFFFE70223126D
:101FC0002A84084009E51703FFFF670083131C41BB
:101FD00058401CC06313E5005CC0834755002320B4
:101FE0000500F99BA302F50097A0FFFFE780E07CC6
:101FF000C9BF1703FFFFE702E30C9747FF1F938753
:1020000067EE98432A8411CB8347350093F7070284
:1020100089C703550500894502971305440197B008
:102020000000E780403B835504000355E4009730EF
:102030000000E780A00C485819C597A0FFFFE78073
:10204000C077232A04021305840397000000E78069
:10205000E0F68144B1499790FFFFE780E06A63CBE7
:10206000A402834734002320040493F727FCA30130
:10207000F40000489790FFFFE780006A13161500F0
:10208000814522859700FFFFE78060081703FFFF67
:1020900067008306B38734030329040385043E994C
:1020A0004A8597000000E78060F12304090065B7C6
:1020B0008347350093F7070299E3014582808357F0
:1020C000E500E39CB7FEC167FD176316F600054502
:1020D0008280054599A81703FFFFE7024300931785
:1020E0000601C187B2842A8401496359F0028357EB
:1020F00005009DCB01456367F600034584003E95CE
:102100003325A6001375F50F0DA01C4813171900F1
:10211000BA9783D70700E38E97FA05099790FFFFD8
:10212000E780805FE343A9FE01451703FFFF6700D7
:1021300043FD1703FFFFE702E3F8AE89AA849790F7
:10214000FFFFE78020532A8497D0FFFFE780A02E6F
:10215000AA8601471306840197050000938585E44C
:102160001745FF1F130545D69790FFFFE780A0197D
:102170002A8925C98C441304C50022859E0593F540
:10218000050897A0FFFFE780003DCC4083877400DF
:10219000E18163DD070493E50508228597A0FFFF31
:1021A000E780603B0D4693854400228597A0FFFFA2
:1021B000E780803783D50400228597A0FFFFE78062
:1021C000A03E83D52400228597A0FFFFE780C03D75
:1021D00003D6490083A50900228597A0FFFFE78069
:1021E000A0344A851703FFFF670003F193F5F50755
:1021F0006DB71703FFFFE70283EE01112A843285D2
:1022000032C697A0FFFFE780A0289780FFFFE780F6
:102210008031835704001747FF1F130727E4324616
:10222000231BF100930700F8A30DF1001C4718438E
:10223000231AA1008983858BB307F740B28548082C
:102240003ECE231C0100230D010097000000E78013
:1022500080EE05611703FFFF6700A3EA1703FFFF86
:10226000E70243E6004101453DC49304C4002685CE
:102270003289AE8997A0FFFFE780802595452A8A9D
:102280002685035B040197A0FFFFE780E0212685F8
:1022900097A0FFFFE780203F8D45AA8A268597A05B
:1022A000FFFFE7806020268597A0FFFFE780A03D25
:1022B0005C48420A135A0A01D2975CC4231864018D
:1022C000814763983A0146054D813306254193378E
:1022D000160013F5F70F1703FFFF6700E3E117037D
:1022E000FFFFE70243DD89692A8BAE8B328AB68A0B
:1022F00081440144314CFD199790FFFFE780C040B5
:1023000063CDA4009790FFFFE7800043018D33B5B4
:10231000AA001703FFFF670083DD33898403832747
:102320000B003E9963170A008347890085043E9499
:10233000E1B703560A00DE854A8533F6C9009700E7
:102340000000E780E0F16DD10545E1B71703FFFF1D
:10235000E702E3D801112A847C000355E5003ECA58
:10236000B70707003ECC7C003ECE97200000E780F8
:1023700020082A898545480897A0FFFFE780E039B3
:102380009945480897A0FFFFE780A016AA844A85D0
:1023900097200000E780A0082380A4009747FF1F34
:1023A0009387C7CB9C434166130606F0939687013B
:1023B00013D78701558F93D68700F18E558FA207CB
:1023C000B706FF00F58FD98F11462C001385140036
:1023D0003EC497D00000E78020CF5008A3820400BD
:1023E0008945228597000000E780E0E019C9AA85A9
:1023F0001305840397A0FFFFE780A0323C408507C8
:102400003CC005611703FFFF6700A3CF1703FFFF61
:10241000E702E3CC9790FFFFE78000322A840504AF
:102420009790FFFFE78040303305A402F1479145C4
:102430003305F50297200000E78020BA11E56555C5
:102440001703FFFF6700E3CB9747FF1F23A4A7A84D
:102450009790FFFFE780402E2A8405049790FFFFA6
:10246000E780802C3305A4028945060597200000EB
:10247000E780A0B669D59747FF1F23A5A7A497902B
:10248000FFFFE780602B2A8405049790FFFFE78019
:10249000A0293304A4029747FF1F239787A2979090
:1024A000FFFFE78060292A849790FFFFE780C0271D
:1024B000930714003385A7029747FF1F2397A7A010
:1024C000970701009387878B1747FF1F2322F7A0E9
:1024D0000145BDB71703FFFFE702C3BEAA842E89DB
:1024E00001449749FF1F938969B7130A80069790A3
:1024F000FFFFE78060236347A40001451703FFFF48
:10250000670083BF3305440383A709024A86A68573
:102510003E9597000000E780E0B919E10504C1BFCE
:102520000545E9BF1703FFFFE702E3B8AA8A2E8B30
:10253000B28B368C3A8A814401448149974CFF1F03
:10254000938CCCB1130D80069790FFFFE780C01DE0
:1025500063C9A40011E085494E851703FFFF67009A
:1025600003B93389A40383A70C025E86D6853E99FE
:102570004A8597000000E780E0B31DC19790FFFFF8
:10258000E780801B0544636D4501D2866286DA854B
:102590001305090397000000E780A0D411C1854905
:1025A00085045DB71703FFFFE702C3B1C1644111A2
:1025B0002A8901449749FF1F938949AA130A800673
:1025C000FD1436C632C42EC29790FFFFE780C015B7
:1025D00092452246B2466348A400014541011703D3
:1025E000FFFF670063B13305440383A709023E95EB
:1025F00009C683473500C18B9DC791C68347350007
:1026000093F707028DC3630699008357E500639C27
:1026100027010357050001CB63E7E50083478500E9
:10262000BA97E3CDF5FA050469BF1703FFFFE70288
:1026300063A9C1642A8901449749FF1F938909A2AC
:10264000130A8006FD149790FFFFE780E00D6346B4
:10265000A4001703FFFF670023AA3305440383A7E1
:1026600009023E958357E500638A97006304990049
:102670006396270197000000E780E0970504E1B723
:102680001703FFFFE702A3A289692A8AAE8A328B69
:10269000B68B8144174CFF1F130C4C9C930C800687
:1026A000314DFD199790FFFFE780000863C6A40035
:1026B0001703FFFF670063A33389940383270C028A
:1026C0008355CA015A863E994A8597000000E780E3
:1026D000609E31C1814D15A03384AD03832709036A
:1026E00003D60B00D68533F6C9003E9422859700A9
:1026F0000000E780E0B609E9850D9790FFFFE780CD
:10270000A000E3CBADFC01A8228597000000E78084
:10271000E08A23040400850471B71703FFFFE70272
:1027200083994169AA8A014A174BFF1F130B0B9328
:102730007D19C14B054C9790FFFFE780E0FE634693
:10274000AA001703FFFF6700839A93098006B30767
:102750003A0383290B02BE9983D7E900638E2701D0
:1027600063842A01639A570103A4890301E84E8513
:1027700097000000E780C0BD050A75BF83570401BC
:10278000639977099304C400268597A0FFFFE7802B
:1027900020D485452A8D2685835C040197A0FFFF00
:1027A000E78080D0268597A0FFFFE78060E862057C
:1027B0006185635905048D45268597A0FFFFE78055
:1027C000A0CE8945268597A0FFFFE780E0CD89450B
:1027D000268597A0FFFFE78020CD8545268597A019
:1027E000FFFFE780A0CD83470500094793F7F70770
:1027F000639AE7009945268597A0FFFFE78000CC04
:10280000A30285014848337D2D01231894016A9560
:1028100048C40040A1BF1703FFFFE702438C37E421
:1028200004008327041D82979737FF1F83C7077013
:102830001715FF1F130585CFA300F5008327441C40
:1028400082978327841C81461306F00F814501453A
:1028500082971703FFFF6700C38A1737FF1F13070D
:10286000E75C18439735FF1F83C5456C9737FF1FFB
:102870009387476A83468703034697036397D50088
:102880009737FF1F2384C76A828083C58701034768
:10289000A7036317B6009737FF1F2389E768828075
:1028A00003C687016317C7009737FF1F2380D768C8
:1028B000828083C68701130750026319D7009307EC
:1028C00060021737FF1F2303F766828083C68701E4
:1028D000130660026315D60093077002DDB783C745
:1028E000870155BF9737FF1F9387C762D44B0947AE
:1028F000638DE60817F3FEFFE702637E1739FF1FBB
:102900001309895E3E8483470900918B9DCFB7E40C
:10291000040083A7041D829783A7441C1735FF1F5B
:102920001305055D829783A7841C81461736FF1F18
:102930000346065E81450145829721C5834709000C
:10294000ED9B1737FF1F2301F75A8347040093F7C6
:10295000F70F85CB91471737FF1F2327F75C9700A9
:102960000000E78080EB97000000E78040EFB7E7CA
:102970000400BC4F414691451735FF1F0345055ADA
:10298000829717F3FEFF6700C377828017F3FEFF7D
:10299000E702E3748D4741116306F504C5476308F8
:1029A000F50285476310F5029737FF1F2382A7586A
:1029B000B7E70400BC4B930500101735FF1F034514
:1029C000E5558297410117F3FEFF67008373854742
:1029D0001737FF1F230EF754B7E70400BC4B9305CE
:1029E0000020E1BF9737FF1F9387C752D44B114791
:1029F000638DE600B7E7040083A7071D8297B7E75A
:102A00000400BC4B930500044DBF05491737FF1F59
:102A1000232C275183C7070032C62E8493F7F70F64
:102A2000D5D3B7E4040083A7041D7D141374F40FF9
:102A30008297E37689FCB245994703C61500E3F017
:102A4000C7FCFC4409061735FF1F1305A54E8297E6
:102A5000BC48930500081735FF1F0345254C829796
:102A600079BF17F3FEFFE70283671737FF1F1307CE
:102A7000674A4047184B1C409736FF1F23A2F64A6F
:102A80006316E4001737FF1F232EF748130584FE53
:102A90009790FFFFE78020A7035564FF9780FFFF13
:102AA000E780A06F97A0FFFFE78020D117F3FEFF1C
:102AB0006700236517F3FEFFE70263629737FF1F86
:102AC00093874745D84BDC4789C797000000E780CC
:102AD00080F985471737FF1F2328F7449737FF1FD3
:102AE0009387C7349C43930500021735FF1F0345A6
:102AF000E54283C787031737FF1F2309F742B7E76C
:102B00000400BC4B829717F3FEFF6700835F973783
:102B1000FF1F23A3A740828017F3FEFFE702835A1B
:102B200037E404007C4CA1451735FF1F0345053FE2
:102B300082977C48A1451735FF1F0345253E9734F2
:102B4000FF1F9384243D8297DC4489EB97000000AB
:102B5000E78080D917F3FEFF6700035A03D567FFAC
:102B60009780FFFFE7806063AA896DD1D8489147BD
:102B70006310F7027C4C91451735FF1F0345053A5A
:102B800082977C4891451735FF1F03452539829769
:102B900003A9490103D409018947B7E9040017379C
:102BA000FF1F2323F73883A7091D210442048297BE
:102BB00083C784011715FF1F130545976119171760
:102BC000FF1FA305F79683A7491C4180829797377B
:102BD000FF1F238F073483A7C91C814609469375BD
:102BE000F40F4A85829711E99737FF1F83C78744FF
:102BF00089C79700FF1FE780E0FFB7E70400BC4FDD
